:020000040800F2
:1000000050EA0120CD020008B97F0008956E000873
:10001000597E0008E5210008D5A200080000000074
:10002000000000000000000000000000B186000891
:100030007534000800000000318200088593000834
:10004000E7020008E7020008E7020008E7020008EC
:10005000E7020008E7020008B1370008E7020008DD
:10006000E7020008BD370008C9370008E7020008AA
:100070000D330008E7020008E7020008E702000865
:10008000E7020008E7020008E7020008092200086A
:10009000E9210008F9210008E7020008D537000827
:1000A000E702000851940008E7020008E702000890
:1000B000E7020008E7020008E7020008E70200087C
:1000C000E7020008E7020008E7020008E70200086C
:1000D000E7020008E7020008E7020008A5A20008FE
:1000E000E7020008E7020008E7020008E70200084C
:1000F000E7020008E7020008E7020008E70200083C
:10010000E7020008E7020008E7020008E70200082B
:10011000E7020008E7020008E7020008E70200081B
:10012000E70200081D3300082D3300083D330008A6
:10013000E7020008E7020008E70200083922000889
:100140001922000829220008E7020008E702000837
:10015000E70200084D330008E7020008BDA20008CE
:10016000E7020008E7020008E7020008E7020008CB
:10017000E7020008E7020008E702000800000000AC
:10018000E7020008E702000800F002F800F074F847
:100190000AA090E8000C82448344AAF10107DA45E2
:1001A00001D100F069F8AFF2090EBAE80F0013F0C0
:1001B000010F18BFFB1A43F00103184794F3000026
:1001C000D4F300000A444FF0000C10F8013B13F088
:1001D000070408BF10F8014B1D1108BF10F8015BA0
:1001E000641E05D010F8016B641E01F8016BF9D193
:1001F00013F0080F1EBF10F8014BAD1C0C1B09D1EA
:100200006D1E58BF01F801CBFAD505E014F8016B5B
:1002100001F8016B6D1EF9D59142D6D370470000ED
:10022000103A24BF78C878C1FAD8520724BF30C822
:1002300030C144BF04680C607047000000230024F4
:1002400000250026103A28BF78C1FBD8520728BFE6
:1002500030C148BF0B607047752900F0F9806329F1
:1002600000F06782002070471FB50EF064FF00F0B9
:1002700040F91FBD10B510BD00F070FA1146FFF730
:10028000F3FF0AF0E1F900F08EFA03B4FFF7F2FF92
:1002900003BC00F091FA00000B49D1F800C04A6895
:1002A0005CF8043B1068184442F8040B8C4528BFE6
:1002B000A1F1DC0C8A4228BFA1F1DC02C1F800C028
:1002C0004A6020F0004070470C0100200948804738
:1002D00009480047FEE7FEE7FEE7FEE7FEE7FEE728
:1002E000FEE7FEE7FEE7FEE704480549054A064B40
:1002F000704700003D9400088901000850A80120C3
:1003000050EA012050AA012050E6012053EA020CD5
:1003100000F069802DE9F04B4FF00006002B1FBF65
:10032000B3FA83F503FA05F424FA05F65E4012BF2A
:100330001643B2FA82F502FA05F4C5F120051EBF94
:1003400022FA05FC44EA0C04203556EA044C4FEA34
:10035000144418BF641C4FF000084FF0000990428D
:1003600071EB030C39D3002919BFB1FA81F701FAF7
:1003700007F6B0FA80F700FA07F6C7F120071EBFAC
:1003800020FA07FC46EA0C062037B6FBF4FCA7EB84
:100390000507103F07F01F0BCBF120062CFA06F6DD
:1003A0000CFA0BFB44BFB3460026202FA4BF5E46C9
:1003B0004FF0000B5BEA060C08BF4FF0010B19EB86
:1003C0000B0948EB0608ABFB027C06FB02CC0BFBDF
:1003D00003CCC01B71EB0C01C1E70B460246414642
:1003E0004846BDE8F08B13B5084318BF4FF0FF3007
:1003F0000146AFF30080BDE81C40704770B50C4665
:100400000546012A05D02878800600D5EA69002330
:1004100002E0012305E05B1C934202D2E05C00286D
:10042000F9D1A869E618C01AA861286A1844286298
:100430002846AFF3008004E0D5E9012114F8010B50
:100440009047B442F8D32846AFF3008070BD000057
:100450002DE9F0410646002410687529314616A59D
:1004600010D0AFF30080002802DA404213A507E065
:1004700031688A0701D512A502E0490704D511A504
:10048000012401E0AFF3008000210A2206F12407D5
:1004900009E0B0FBF2FCB0FBF2F302FB1C003030D1
:1004A00078541846491C0028F3D123462A46304682
:1004B000BDE8F04100F0DAB8000000002D000000B7
:1004C0002B000000200000000B4910B5A1F17C02B8
:1004D0000A4CC2E93712372106E000EB104342F81C
:1004E0002130074B00FB03400B1EA1F10101F4DC9E
:1004F00010BD0120E8E70000AC000020E119D6663D
:10050000CD0D0100032A40F2308010F0030C00F002
:10051000158011F8013BBCF1020F624498BF11F83D
:1005200001CB00F8013B38BF11F8013BA2F10402F6
:1005300098BF00F801CB38BF00F8013B11F003036E
:1005400000F02580083AC0F0088051F8043B083AD2
:1005500051F804CBA0E80810F5E7121D5CBF51F874
:10056000043B40F8043BAFF30080D20724BF11F8EE
:10057000013B11F801CB48BF11F8012B24BF00F853
:10058000013B00F801CB48BF00F8012B704710B5C4
:10059000203AC0F00B80B1E81850A0E81850B1E83C
:1005A0001850A0E81850203ABFF4F5AF5FEA027C7B
:1005B00024BFB1E81850A0E8185044BF18C918C0AB
:1005C000BDE810405FEA827C24BF51F8043B40F84C
:1005D000043B08BF7047D20728BF31F8023B48BF31
:1005E00011F8012B28BF20F8023B48BF00F8012B6F
:1005F000704702F0FF0343EA032242EA024200F09E
:1006000002B84FF0000200B51346944696462039D2
:1006100022BFA0E80C50A0E80C50B1F12001BFF4BB
:10062000F7AF090728BFA0E80C5048BF0CC05DF821
:1006300004EB890028BF40F8042B08BF704748BF6F
:1006400020F8022B11F0804F18BF00F8012B7047E3
:1006500070477047704710B500F078F8006810BD1B
:1006600010B5044600F072F8046010BD2DE9F047A3
:100670000D4699469246044600F124080168880612
:1006800004D5E06921F01001216000E00120A842BA
:1006900001DD471B00E00027A1697A1902EB090080
:1006A000081AA0612078C00602D42046AFF300806B
:1006B000002608E0D4E901211AF806009047206AD4
:1006C000401C761C20624E45F4DB2078C0060AD51B
:1006D0002046AFF3008006E0D4E9012130209047A6
:1006E000206A401C2062381EA7F10107F4DC07E0F5
:1006F000D4E9012118F805009047206A401C2062C7
:10070000281EA5F10105F3DC2046AFF30080207818
:10071000000602D50220BDE8F0870120FBE710B5F6
:10072000436913B1AFF3008001E0FFF767FE0120DA
:1007300010BD127800F124010A7000224A700122D3
:10074000EDE711684FF0FF32E9E70000004870471D
:10075000F8C3012000487047F8C301207546FFF731
:10076000F9FFAE4605006946534620F0070085466E
:1007700018B020B5FFF7B8FDBDE820404FF00006E7
:100780004FF000074FF000084FF0000BAC46ACE80C
:10079000C009ACE8C009ACE8C009ACE8C00921F068
:1007A00007018D46704710B50446AFF30080204620
:1007B000BDE81040FFF769BD01491820ABBEFEE758
:1007C0002600020070470000B0B52DED028B0446F4
:1007D00000284FF0FF0061D00D4600295ED095ED56
:1007E000000A95ED011A95ED022A95ED033A20EEE7
:1007F000010A22EE033A21EE011A22EE022A31EE1C
:10080000021A30EE030A31EE011AB7EE008A30EE1A
:10081000000A78EE410A0DF00FF9B0EE401A95ED9E
:10082000000A95ED012A95ED023A95ED034A20EE76
:10083000030A24EE022A30EE420A30EE000AB0EE3D
:10084000C02AB4EE482AF1EE10FA84ED011A02DA59
:100850000CF0EEFD01E009F085FE84ED020A95ED55
:10086000000A95ED011A95ED032A95ED023A20EE66
:10087000020A21EE031A30EE010A23EE031A22EED9
:10088000022A32EE011A31EE011A30EE000A78EE39
:10089000410A0DF0D1F8002084ED000A40B2BDEC11
:1008A000028BB0BD70B52DED028B00284FD0B7EE96
:1008B000001A81EE000A0D4604464FF07E51002DCD
:1008C00080ED040A4FF00000C4E90010A060E06071
:1008D00000F09F80D5E900600EF062FB41EC180B40
:1008E00030460EF05DFB41EC110BB0EE480AF0EE25
:1008F000680A0CF0A1FF51EC100B0DF059FD95EDBD
:10090000000AB5EE400AF1EE10FA22D195ED010A87
:10091000B5EE400AF1EE10FA1BD195ED020AB5EEE4
:10092000400AF1EE10FA14D140F2C560C3F64D70E2
:1009300044F62D214AF2564244F2AD73C3F60D41FE
:10094000CBF63932C3F619730FC4002061E0FF20E3
:100950005FE09FED321A00EE100AB4EE410AF1EEAC
:1009600010FA1EDCB5EE400AF1EE10FA19DB9FED2D
:100970002C2AB4EE420AF1EE10FA25DCB4EE410A5C
:10098000F1EE10FA20DB9FED271AB4EE410AF1EEEA
:1009900010FA2CDCB4EE420AF1EE10FA27DB00204C
:1009A00037E045F66E10C3F67F7045F20C3148F61D
:1009B000AB0249F28553C3F6B011CBF6BB32C3F696
:1009C00097530FC4002024E040F2C560C3F64D7079
:1009D00044F62D214AF2564244F2AD73C3F60D415E
:1009E000CBF63932C3F619730FC4002011E040F280
:1009F000C560C3F64D7044F62D214AF2564244F2CA
:100A0000AD73C3F60D41CBF63932C3F619730FC47B
:100A1000002040B2BDEC028B70BD00BFDB0FC9BF30
:100A2000DB0F49C00000B4C20021C0E900118160A1
:100A300070470000B0B52DED108B8EB00446002835
:100A40004FF0FF0018BF002904D140B20EB0BDEC3A
:100A5000108BB0BD002AF8D040F200054EF69E7013
:100A6000C2F20005C3F627502860C3B193ED00EA37
:100A700093ED01FAD3ED028AB5EE40EAF1EE10FAF9
:100A800011D1B5EE40FAF1EE10FA0CD1F5EE408A34
:100A9000F1EE10FA07D1204600F094FAD5E720468F
:100AA00000F090FAD1E792ED000A92ED011A94ED70
:100AB000014A94ED025A92ED022A94ED036A94EDF4
:100AC000003A24EE407A61EE050A37EE607A62EE73
:100AD000060A37EE607A60EE030A62EE051A71EEDE
:100AE000A00A61EE061A70EEE10A61EE031A62EEE8
:100AF000042A22EE032A21EE041A91ED00DA71EEA7
:100B0000E21A20EE066A31EE021A20EE050A36EEEF
:100B1000216AD1ED019AD1ED02AA31EE400AB6EE7A
:100B2000001AB5EE40DA27EE015A60EE810A26EE91
:100B3000017AF1EE10FA20EE016A0AD1F5EE409A40
:100B4000F1EE10FA05D1F5EE40AAF1EE10FA00F040
:100B5000EC812DEE0D0A29EEA91A30EE010A2AEEDB
:100B6000AA1A30EE010A8DED0D6A8DED0C7ACDEDED
:100B70000B0A8DED0A5A06F08FF92DEE001A8DED55
:100B8000071A29EE801A2AEE800A8DED081A8DEDDB
:100B9000090A2EEE0E0A2FEE0F1A30EE010A28EE89
:100BA000A81A30EE010A06F077F994ED001A6EEEFD
:100BB00000DA6FEE00AA94ED034A31EE01EA68EE26
:100BC000808A94ED012A94ED023A2AEE8E6A61EE53
:100BD00001EA8DED026A28EE8E0A2DEEAE5A26EE5F
:100BE000046A62EE02BA35EE465A20EE036A36EE29
:100BF000055A2DEEAB6A32EE02FA36EE055A2AEEAF
:100C00008F6A23EE066A36EE055A28EE8F6A26EEC4
:100C1000046A63EE03FA36EE055A2DEEAF6A24EE4F
:100C2000048A35EE465A2DEE886A2DEE8E9A35EE00
:100C3000465A29EE046A2AEEAE7A37EE066A22EEAA
:100C4000000A2DEE8FAA36EE400A23EE0A6A36EE2F
:100C5000000A2AEEAB6A30EE460A2AEEAF6A73EE5D
:100C6000039A36EE000A28EEA96A24EE066A36EEEA
:100C7000000A2AEE886A30EE460A25EE055A20EE72
:100C8000000A35EE000A21EE02BA21EE035A21EEE7
:100C9000041A8DED051A22EE031A8DED031A23EEC8
:100CA000041A8DED041A34EE041A8DED015A22EE69
:100CB00004CA6EEE03CA8DED061A29EE84DA06F038
:100CC000EBF894ED013A94ED022A9DED021A29EE1B
:100CD000024A21EE031A31EE444A94ED031A28EE3B
:100CE000AE5A35EE044A2AEE015A35EE044A28EE91
:100CF000AB5AF7EE001A34EE454A2AEEA95A81EEB5
:100D0000800A25EE015A35EE044A28EEAF5A34EE39
:100D1000454A28EE885A75EE042A3CEE0C4A9DEDB1
:100D2000075A34EE6C4A34EE454A3BEE0B5A9DEDC1
:100D3000086A35EE0D5A35EE465A2FEE056A29EE51
:100D4000847AF6EE007A76EE470A37EEEF6A36EEF0
:100D5000486A9DED018A20EE066A3CEE487A27EE4D
:100D6000227A36EE076A36EE6D7A22EE226A66EE57
:100D7000073A70EEE33ADDED050ADDED034A60EE79
:100D8000015A74EEE00ADDED044A60EE200A7BEEC3
:100D9000244A64EEA24A70EEA40A63EE224A70EE80
:100DA000EA0A74EEE56A66EEA06A77EEEB7A76EE12
:100DB000A33A78EE0C6A77EEEF7A60EE266A67EE79
:100DC000A27A76EEA76A76EEE86A60EE027ADDED48
:100DD000068A27EEA68A38EE23CA68EE843A2EEEFB
:100DE000058A78EE233A3BEEAB8A71EEC81A3FEEE5
:100DF000AF8A71EEC81A9DED098A21EE22AA71EE22
:100E0000C81AB1EE008A23EE089A21EE899A73EE91
:100E1000C93A94ED009A2AEE07BA73EE8B3A29EE9E
:100E200022BA77EE8B7A67EEA07A72EEA22A77EE7C
:100E3000A33A63EE227A75EEE75A65EEA65A35EECE
:100E4000A3DA68EE853A6EEE045A73EEE53A62EE86
:100E5000085A65EEA11A73EEE11AF8EE003A60EE58
:100E6000233A62EE235A75EECB5A65EE875A20EE8E
:100E7000033A71EEA51A73EE0A5A20EE090A22EE21
:100E8000222A65EEA05A30EE422A75EEA11A22EE11
:100E9000262A23EE811A32EE218A2FEE042A29EE29
:100EA000854A31EE241A34EE022A21EE071A36EE74
:100EB000400A32EE011A20EE200A30EE010A23EE3B
:100EC000261A31EE009A2CEE0C0A2DEE0D1A30EE99
:100ED000010A28EE081A31EE000A29EE091A31EE4D
:100EE000000A05F0D9FF95ED004A9DED0A5A20EE63
:100EF0000C1ADDED0B0A20EE0D2A24EE011A9DEDF1
:100F00000C7A9DED0D6A20EE083A20EE090A35EEC6
:100F1000415A24EE021A70EEC10A24EE031A24EE9E
:100F2000000A37EE417A36EE406A94ED043A94EDC9
:100F3000000A94ED011A25EE035A94ED022A30EED0
:100F4000050A20EE835A94ED034A35EE011A27EE86
:100F5000035A35EE022A26EE033A84ED000A84EDA8
:100F6000011A20EE000A21EE011A33EE043A30EEA7
:100F7000010A22EE021A30EE010A23EE031A30EEC5
:100F8000010A84ED022A84ED033A05F085FF94ED11
:100F9000001A94ED012A94ED023A94ED034A20EEF2
:100FA000011A20EE022A20EE033A20EE040A002065
:100FB00084ED001A84ED012A84ED023A84ED030ADF
:100FC00043E50000B0B52DED108B044600284FF02E
:100FD000FF0018BF002900F06981002A00F0668137
:100FE00040F2000542F60230C2F20005C3F6075097
:100FF000286092ED000A92ED011A94ED014A94EDF9
:10100000025A92ED022A94ED036A94ED003A24EE1E
:10101000407A61EE050A37EE607A62EE060A37EE34
:10102000607A60EE030A62EE051A71EEA00A61EEC4
:10103000061A70EEE10A61EE031A62EE042A22EE4D
:10104000032A21EE041A91ED00CA71EEE21A20EE95
:10105000066A31EE021A20EE050A36EE216A91ED9B
:1010600001DA91ED02EA31EE400AB6EE001AB5EE71
:1010700040CA27EE01BA20EE81AA26EE019AF1EECF
:1010800010FA20EE018A0AD1B5EE40DAF1EE10FA3C
:1010900005D1B5EE40EAF1EE10FA00F0BC802CEE7E
:1010A0000C0A2DEE0D1A30EE010A2EEE0E1A30EE5D
:1010B000010A05F0F1FE94ED003A94ED025AF1EECA
:1010C000001A2CEE001A94ED014A75EE050A63EE43
:1010D000212A65EE053A62EEA34A61EE205A74EECB
:1010E000A54A64EE045A2DEE002A94ED036A34EE0C
:1010F000047A62EEA52A72EEA42A62EE074A32EE64
:10110000E4CA76EE062A64EE214A66EE066A64EECA
:10111000A67A21EE22DA77EECD7A23EE03DA2DEEEF
:1011200021DA2EEE000A24EE0DEA33EE033A7EEECB
:10113000277A22EE03EA77EECE7AB2EE00EA24EEC8
:101140000E4A77EEE47A24EE25FA7FEE277A24EE33
:10115000234A34EE274A60EE244A34EE84FA2DEE18
:10116000054A21EE033A33EE043A25EE0E4A25EE07
:10117000215A65EE264A33EE243A62EE222A33EEF5
:10118000623A33EE453A65EE842A32EE833A24EE33
:10119000234A34EE033A20EE050A30EE03DA21EE5C
:1011A000070A25EEA11A21EE061A31EE400A23EEB7
:1011B000A11A26EE011A30EE010A22EE201A30EEB4
:1011C00041EA2CEE0C0A2FEE0F1A30EE010A2DEE3A
:1011D0000D1A31EE000A2EEE0E1A31EE000A05F05D
:1011E0005BFE95ED004A20EE0C1A20EE0F2A24EE4D
:1011F000011A20EE0D3A20EE0E0A3BEE41BA24EE23
:10120000021A3AEE41AA24EE031A24EE000A39EE3D
:10121000419A38EE408A94ED043A94ED000A94ED38
:10122000011A2BEE035A94ED022A30EE050A2AEE3B
:10123000035A94ED034A35EE011A29EE035A35EEAE
:10124000022A28EE033A84ED000A84ED011A20EE0A
:10125000000A21EE011A33EE043A30EE010A22EEC2
:10126000021A30EE010A23EE031A30EE010A84ED71
:10127000022A84ED033A05F00FFE94ED001A94ED76
:10128000012A94ED023A94ED034A20EE011A20EE71
:10129000022A20EE033A20EE040A002084ED001A10
:1012A00084ED012A84ED023A84ED030A40B2BDECDC
:1012B000108BB0BDB1EE601AB4EE600AF1EE10FA18
:1012C000B4EE401AC8BFB0EE600AF1EE10FAC8BF23
:1012D000B0EE410A7047000080B54DF61030C2F202
:1012E00001000068082109F049FC80BD80B54CF27E
:1012F000E442C2F2010200201221132300F086F919
:10130000002080BD80B5022001214FF0FF3209F09E
:1013100075FC80BD9FED010A704700BF0000C84307
:1013200080B54DF61030C2F201000068102109F0BE
:1013300025FC80BD80B54CF2E440C2F20100C21D24
:1013400001200221062300F061F9002080BD000089
:1013500080B5042001214FF0FF3209F04FFC80BD21
:10136000F0B581B000284FF0FE0700F097800C46E2
:10137000002900F0938040F65016C2F200060546A0
:10138000307808B1FD2789E009F096FC4DF6103160
:10139000C2F20101002808607BD000207E21B62225
:1013A000EC6200F08FF901201421B62200F08AF9D6
:1013B0001E2000F07BFE00201E2100F04DF90020D1
:1013C000002100F049F91E2865D1012000210124E7
:1013D00000F042F90F2860D1052000F04FFD0620F3
:1013E00000F04CFD41F2BD52C0F600020020012188
:1013F000002700F031FE41F2D921C0F6000105209E
:1014000000F086FD41F22131C0F60001062000F017
:101410007FFD00204021AA2200F054F90020412144
:10142000012200F04FF900205321082200F04AF970
:1014300000205821042200F045F900207D210422DB
:1014400000F040F9322000F031FE01200F2101228E
:1014500000F038F901201021032200F033F90120B7
:101460001621002200F02EF901201821012200F09F
:1014700029F901201521802200F024F90A2000F02A
:1014800015FE0520347000F013FD062000F010FD5D
:1014900004E0FE2702E0FC2700E0FC2778B201B060
:1014A000F0BD0000002841D04CF2E441C2F201013D
:1014B000B1F901209FED1F3A00EE102AB8EEC00AE4
:1014C00080EE030AB1F90330B1F905C001EE103A1C
:1014D00002EE10CAB8EEC11AB8EEC22A81EE031AA3
:1014E00082EE032A4FF60003CFF6FF7380ED040A65
:1014F0004A7C897CD20042EA51120021B1EB922F42
:1015000080ED051A80ED062A18BF1A4300EE102A56
:10151000B8EEC00AB4EE001A20EE010AB3EE071AC4
:1015200030EE010A80ED0A0A48B27047FE2148B247
:10153000704700BF00A0AA45C0B34CF2E441C2F21C
:101540000101B1F90720B1F90930B1F90B1000EE32
:10155000102A01EE103A9FED172A03EE101AB8EE8A
:10156000C00AB8EEC11AB8EEC33A80EE020A81EEA4
:10157000021A83EE022A9FED103AC16A91ED014AE8
:1015800091ED025A20EE030A21EE031A22EE032AFD
:1015900091ED003A31EE441A30EE430A32EE452A1C
:1015A00080ED070A80ED081A80ED092A6FF001002E
:1015B000704700BF6F12034235FA8E3C10B5012010
:1015C00000F090FC4DF61034C2F2010438B901204D
:1015D000012100F0C3FC2068022109F0CFFA0220AB
:1015E00000F080FC002818BF10BD0220012100F08F
:1015F000B5FC2068042109F0C1FA10BD80B518209F
:1016000001214FF0FF3209F0F9FA80BD002A08BF2E
:10161000704770B51C4615460E4618B1012805D115
:10162000022000E00120002100F098FC4CF2F7417C
:1016300046F08000C2F20101087000200122002360
:1016400000F01AFD002029462246012300F0EAFCA2
:10165000BDE8704070470000F0B581B0044601203D
:101660000D46012600F022FD14B1012C04D1022602
:101670003046002100F072FC4CF2F746C2F201063F
:1016800045F08000374607F8010B00203146012263
:101690000023012500F0F0FC002031460222002347
:1016A00000F0C0FC34B1012C09D14CF2F747C2F272
:1016B000010702252846012100F050FC3878C0B20D
:1016C00001B0F0BDB0B5044601F07F004CF2F74127
:1016D000C2F20101087001204A70012500F0E6FC09
:1016E00014B1012C04D102252846002100F036FC5B
:1016F0004CF2F741C2F2010100200222002300F067
:10170000BBFC24B1012C18BFB0BD022000E00120B9
:10171000012100F023FCB0BD2DE9F04381B040F67B
:10172000B818C2F200080646D8F8000014460D4664
:101730006421002A08BF0A2409F08AF908B1FB24B1
:101740002FE04DF28039C2F20109D9F8000000E023
:10175000006930B10178B142FAD14168A942F7D1AC
:101760001AE0142000F012FC88B1074620461C2124
:10177000002209F0C3F8B86058B1D9F800003C73F2
:1017800000243E707D603861C9F8007005E0FE24D9
:1017900003E0384600F06EFBFF24D8F8000009F0A3
:1017A000CDF960B201B0BDE8F083000070470000E1
:1017B0004DF28032C2F20102126800E01269002A82
:1017C00004BF0020704713788342F7D153688B42DF
:1017D000F4D1906870470000D0E90212081FB0FAF7
:1017E00080F14FF0020008BF0320022A18BF480909
:1017F000704700004CF650424CF62841C2F20102FC
:101800000128C2F2010118BF0022002818BF1146AA
:10181000012888BF00210846704700002DE9F041EB
:1018200015464CF66862C2F201021278012A11D103
:10183000A5B140F6B818C2F200080746D8F8000073
:101840000E4664211C4609F003F958B1FB2040B252
:10185000BDE8F081FD2040B2BDE8F081FE2040B23D
:10186000BDE8F08138463146FFF7A2FFD8F80010F6
:101870000646084609F062F966B13046294600225C
:10188000234608F0F7FF002818BF4FF0FF3040B2A2
:10189000BDE8F081FC2040B2BDE8F0812DE9F047C1
:1018A0008AB04CF66867C2F20107387808B1FD24A7
:1018B0008AE04CF25840C2F201006821FEF7A1FE16
:1018C000002400BFE0B200F03BFA0134012CF9D053
:1018D0004CF6646041F2AD71C2F20100C0F6000145
:1018E00001600020002409F0DDF840F6B811C2F2D2
:1018F00000010028086066D0E8464FF00109404624
:10190000282187F80090FEF77CFE4CF62846C2F2AC
:1019100001064FF00E0A30464146CDE90244CDE9BA
:101920000799CDF824A0049402F036FC304603F069
:1019300003F841F64922C0F600020020062100F01B
:1019400051F841F6DD45C0F60005002000212A4689
:1019500000F048F8002001212A4600F043F800205A
:1019600002212A4600F03EF83046032102F0B6FB81
:101970004CF65046C2F2010630464146CDE9049A83
:1019800002F00AFC304602F0D7FF41F60D32C0F6F5
:1019900000020120082100F025F8012000212A463C
:1019A00000F020F8012001212A4600F01BF8012058
:1019B00002212A4600F016F83046112102F08EFB73
:1019C00087F8009000E0FF2460B20AB0BDE8F0871D
:1019D00080B54CF66462C2F201021268002A18BF98
:1019E000904780BD4CF66863C2F201031B78012B5F
:1019F0001EBFFD2358B270473AB101284FF0FF03D4
:101A000098BF0C2904D958B27047FE2358B27047CA
:101A10004CF2584CC2F2010C342310FB03C00023DB
:101A200040F8212058B2704780B54CF66863C2F286
:101A300001031B78012B03D1FFF76EFE40B280BD7E
:101A4000FD2040B280BD00002DE9F04F93B003A807
:101A50000D3001904FF0000A0CAE002005E000BFF1
:101A60000298002800F101004CD15FFA80FB02903F
:101A70005846FFF7BFFE0028F2D0044609E000BF39
:101A800003F0CAFA0990384603A90022002308F09F
:101A900085FF2046002102F001FC0028E0D020460E
:101AA000002132460AAB02F009FC0028F1D10E9861
:101AB0000028304618BF043005683046FFF78CFE1A
:101AC000804628464146FFF783FF814658464946EF
:101AD000FFF76EFE0028DCD00746DDE90F02CDF8E7
:101AE0000CA00028CDE908AACDE906AA8DF80C8043
:101AF000CDE904598DF81820C2D101980AA9FEF742
:101B000001FDBDE713B0BDE8F08F00002DE9F04FF7
:101B100093B003A80D3001904FF0000A0CAE0020E6
:101B200005E000BF0298002800F101004CD15FFAE7
:101B300080FB02905846FFF75DFE0028F2D0044675
:101B400009E000BF03F068FA0990384603A90022B3
:101B5000002308F023FF2046012102F09FFB00280C
:101B6000E0D02046012132460AAB02F0A7FB002854
:101B7000F1D10E980028304618BF04300568304671
:101B8000FFF72AFE804628464146FFF721FF81469F
:101B900058464946FFF70CFE0028DCD00746DDE931
:101BA0000F02CDF80CA00028CDE908AACDE906AABD
:101BB0008DF80C80CDE904598DF81820C2D1019818
:101BC0000AA9FEF79FFCBDE713B0BDE8F08F000047
:101BD0002DE9F04389B017464CF66862C2F2010263
:101BE0001278012A04D10446012806D9FF2000E01A
:101BF000FD2040B209B0BDE8F08301F0FE001D46B3
:101C00000E46022802D00DB9FE20F2E7DDF8408032
:101C1000B8F1080F01D9FF20EBE72046FFF7EAFDF6
:101C200098B181460020032E0890CDE90600CDE949
:101C30000400CDE90200019009D8DFE806F0020AAD
:101C40000D110197002100200DE0FE20D1E7FF20BB
:101C5000CFE70297002005E001970220002102E073
:101C6000022002970421CDE903100020002DCDF8B9
:101C700014808DF8180018BFB8F1000F05D001A826
:101C8000183029464246FEF73DFC484602F0A8FBC4
:101C900038B101A901F118026B46484602F032FA48
:101CA00028B101A9204600F0A5F80138A1E70020DD
:101CB0009FE7000079B180B582B00A6891F804C04E
:101CC0004B1D0021CDF800C0FFF782FF02B0BDE838
:101CD000804040B27047FE2040B270472DE9F0438B
:101CE00089B001AC04F118090025E84604E000BF02
:101CF000002D05F1010520D1EFB23846FFF77AFD3E
:101D00000028F5D0064600BF384600F027F8002826
:101D1000EED1304602F064FB0028E9D03846214677
:101D200000F02EF80028E3D0304621464A464346CC
:101D300002F0E8F90028E7D0DAE709B0BDE8F0835F
:101D40004DF6183100EBC010C2F2010101EBC000EA
:101D50000021C0F80014C0F8041470474DF6183183
:101D600000EBC010C2F2010101EBC000D0F800147A
:101D7000D0F80404081AB0FA80F040097047000057
:101D8000002904BF002070472DE9F0414DF6183CB2
:101D900000EBC012C2F2010C0CEBC202D2F800E45C
:101DA000D2F804349E451FD002F204452C6800EBA3
:101DB000C0100CEBC00000EB4412640150F804C0EA
:101DC000D2E901805769D2E90364C1E900C8C1E9D9
:101DD0000447C1E90206D2E90620C1E906202868C5
:101DE000013000F01F002860BEEB030018BF012087
:101DF000BDE8F08101284FF0000238D8B9B32DE9D1
:101E0000F0474DF6183C00EBC012C2F2010C0CEB8F
:101E1000C202D2F80034D2F804E4013303F01F0305
:101E200073451ED002F58069D9F8004000EBC01060
:101E30000CEBC00000EB44124FEA441AD1E904C68F
:101E4000D1E90078D1E9025440F80A705661C2E93C
:101E5000034CC2E90185D1E90610C2E90610C9F8B0
:101E60000030B3EB0E0218BF0122BDE8F047104668
:101E70007047000080B509F0F9FD80BD07284FF0DC
:101E8000FF0212D801460620DFE801F0090F0F0F0C
:101E90000F0406080A2002E0172000E0092080B5A0
:101EA00003F06EFA0022BDE8804050B27047000097
:101EB00007284FF0FF0212D801460620DFE801F0A4
:101EC000090F0F0F0F0406080A2002E0172000E098
:101ED000092080B503F058FA0022BDE8804050B2D6
:101EE00070470000082884BF0020704780B54FF27B
:101EF0003821C0F6000101EBC002526831F8301001
:101F0000104603F07DF80138B0FA80F0400980BD3A
:101F1000B9B1082882BFFF2040B270474FF2382283
:101F2000C0F6000232F830C0002000232CFA00F284
:101F3000D20709D10E2B03F1010300F10100F5D9FD
:101F400008E0FE2040B2704740F21412C2F20002D4
:101F500042F82010002040B270470000082882BFDD
:101F6000FF2040B2704780B50A464FF23821C0F6D4
:101F7000000101EBC0035B6831F83010184603F034
:101F800045F80020BDE8804040B2704780B509F0B8
:101F9000DFFB80BD00281EBFFF2040B27047B7EEB8
:101FA000001A4CF68C50B4EE410AC2F20100F1EE78
:101FB00010FAC8BFB0EE410A00689FED0C1AC16A62
:101FC000B5EE400A0131F1EE10FAB8BFB0EE410AA9
:101FD00001EE101AB8EE411A20EE010ABCEEC00A5A
:101FE00080ED0D0A002040B2704700BF00000000E5
:101FF00010B510B1FF2460B210BD4CF68C50C2F287
:1020000001000021002404F085FB60B210BD000037
:1020100040F62C01C2F20001002818BF002108463A
:102020007047000070B510B1FF2040B270BD1E4671
:1020300014460D46FFF7ECFF0028F5D0294622464E
:1020400016B103F029FE02E0142303F06BFD002813
:1020500018BF012040B270BD002A0FBFFE204CF215
:10206000C443C2F2010303EB40101CBF40F821201F
:10207000002040B27047000070B510B1FF2040B2A0
:1020800070BD1E4614460D46FFF7C2FF0028F5D06E
:102090002946224616B104F0EDF802E0142303F0BD
:1020A00095FE002818BF012040B270BD70B50446EF
:1020B00008F076FB0546FF2608F054FB411C052975
:1020C0000BD80120884010F0310F0BD110F0060F13
:1020D0000AD0204602F08EFE11E06FF000418842E7
:1020E00018BF002670B270BD4FF47A70B0FBF5F1E6
:1020F000B4FBF1F0A14288BF012008F009FB0026E3
:1021000070B270BD2DE9F04108F04AFB04460AF0B8
:102110008DFE4FF47A784EF21806B8FBF4F4CEF246
:102120000006376804FB00F50AF080FE6043316862
:10213000854208BF394656F8042C01FB08F10132EC
:10214000B1FBF2F100FB08F0401A00F57A700021B3
:10215000BDE8F08103288FBF002040B201A151F8F3
:1021600020007047D4CD0120840800201CCE01201F
:10217000CC08002080B582B001680A68D20614D568
:10218000002201920A68019249680191019907F0C1
:102190000DFF40F25C1100EBC000C2F2000101EB48
:1021A0008000006A002818BF804702B080BD000090
:1021B0003AB103284FF0FF0398BF082904D958B259
:1021C0007047FE2358B2704740F25C1300EBC0002A
:1021D000C2F2000303EB8000002340F8212058B234
:1021E00070470000FEE7000080B54CF62840C2F2C0
:1021F000010002F009F980BD80B54CF62840C2F21A
:10220000010002F001F980BD80B54CF62840C2F211
:10221000010002F0F9F880BD80B54CF65040C2F2E2
:10222000010002F0F1F880BD80B54CF65040C2F2DA
:10223000010002F0E9F880BD80B54CF65040C2F2D2
:10224000010002F0E1F880BD4FF0030160B146F2F9
:1022500000420068C4F2000202F58063984208BFA1
:102260000121801A08BF0146C8B2704780B50246F6
:1022700003284FF0FF000BD851B140F26830C2F292
:10228000000050F8220028B102691AB18068904716
:1022900040B280BD007900220A54FC2040B280BDCB
:1022A000B0B540F21000C2F2000000F017F840F2A2
:1022B00068350024C2F2000503E000BF0134042C9D
:1022C00009D055F824000028F8D0C1680029F5D0BD
:1022D00080688847F2E70020B0BD000010B10179A6
:1022E000032902D9FF2040B2704740F26832C2F29F
:1022F000000242F82100002040B2704750B380B580
:1023000090F88010022902D80144097CB1B900215B
:102310000FF2480C1CF8012083181B7C002B08BF0F
:10232000042203D1022901F10101F3D180F88020B8
:1023300080F8842080F8A82080F8C02000F11001E7
:1023400000F14802012300F0F5F80020BDE88040CC
:1023500040B27047FF2040B2704700BF000102004A
:102360000146006891ED241A90ED030A91ED252AAB
:1023700020EE011A20EE020A002081ED241A81EDE0
:10238000250A7047002070470146006891ED251A24
:1023900090ED020A002031EE400A81ED250A7047D7
:1023A00090F88010012902D051B9012100E00021EC
:1023B00080F8801080F8841080F8A81080F8C01091
:1023C000002070470146006891ED241A90ED040A40
:1023D00091ED252A20EE011A20EE020A002081ED5F
:1023E000241A81ED250A704701460122002081F858
:1023F000C3207047014690F8C100013000F003028D
:10240000002081F8C12070470146006891ED251A2F
:1024100090ED020A002030EE010A81ED250A704796
:102420000146006891ED241A90ED020A002031EE79
:10243000400A81ED240A70470146006891ED241A94
:1024400090ED020A002030EE010A81ED240A704767
:102450000146052081F88C000222002081F8AC2082
:10246000704700000020704710B5864600284FF0E6
:10247000000018BF002A00D110BDD2F804C08CF0B3
:1024800000404FEACC0343EA5073062B10D80020DB
:10249000DFE803F0050E0E0E04222B00ECE79EF899
:1024A0002600002818BF0120E1B391F8261024E08F
:1024B000DEF82C0000EA0C00A0EB0C00B0FA80F073
:1024C0004FEA501081B3C96A01EA0C01A1EB0C017B
:1024D000B1FA81F1490913E09EF82800002818BFDD
:1024E000012019B391F8281007E09EF82700002872
:1024F00018BF0120E1B191F82710002918BF012170
:10250000127A002A08BF10BD022A05D0012A07D17D
:1025100081F00101084010BD80F00100084010BDAD
:10252000002010BD0021EBE70021E9E70021E7E7EB
:102530000021E5E72DE9F047804600284FF0FF0035
:102540001ED00E46E1B14FF21C4A1C4691460025B2
:10255000C0F6000A03E000BF1035B02D0FD00AEB23
:102560000507787A2042F7D0304649463A46FFF7C9
:102570007BFF0028F0D0F96840468847ECE7002050
:1025800040B2BDE8F08700002DE9F0410022C1E92A
:102590000022C1E90222C1E904228A61034653F8FC
:1025A00001EF40F2013C1C7CC0F2020C013CE4B2A1
:1025B000E500032C4FF0000438BF2CFA05F493F823
:1025C0003C505E689F68D3F80C800C755C7C0D7085
:1025D000013CE4B2E500032C4FF0000438BF2CFAB4
:1025E00005F44C759C7CC1F804E0651EEDB2EC006E
:1025F000032D4FF0000538BF2CFA04F58D75DD7CF6
:102600008E606E1EF6B2F500032E4FF0000638BF46
:102610002CFA05F6CE751B7DCF60013BDBB2022B99
:10262000C1F810809EBFDB002CFA03F30B76837D8C
:10263000013BDBB2DF00032B4FF0000338BF2CFA65
:1026400007F34B76C37D013BDBB2DF00032B4FF07A
:10265000000338BF2CFA07F38B76007E0138C0B236
:10266000C30003284FF0000038BF2CFA03F2CA76EB
:10267000BDE8F08180B505F00DFE80BD90F83D000D
:102680007047000070B52DED028B20B30446FFF7B4
:1026900039FD05460E460CF0D8FC9FED1F8A00EE72
:1026A000100A80EE080AE068281A66F1000184ED3D
:1026B000010A0CF0CAFC00EE100A80EE080A94F839
:1026C0008000E560042884ED020A06D3204600F06D
:1026D000F1F8FC201BE0FF2019E094F8A8004CF270
:1026E000B435C2F2010505EB001081682046884729
:1026F00094F8840005EB001041682046884794F860
:10270000C00005EB0010C16820468847002040B299
:10271000BDEC028B70BD00BF00247449B0B5054606
:1027200000284FF0FF000BD00C4649B12846C421C9
:10273000FDF767FF2C60FFF7B3FDFFF793FE002066
:1027400040B2B0BD80B5417C69B1042280F88C20D4
:10275000002200F11001C0E9242200F14802022306
:10276000FFF7E8FE80BD032180F88C1080BD0000DB
:1027700080B5417C61B3012280F8AC20B0F93020F3
:102780000368524200EE102AB0F9322090ED021A8E
:1027900003EE102AB8EEC00A93ED012AB8EEC33A50
:1027A00021EE000A21EE031A22EE000A22EE011A9F
:1027B000B7EE082A00F1100121EE021A00F14802DA
:1027C000042380ED2C0A80ED2D1AFFF7B3FE80BDA7
:1027D000002180F8AC1080BD80B5417C71B190F8CB
:1027E0003630012200F1100180F8C22080F8C33099
:1027F00000F148020823FFF79DFE80BD002180F80C
:10280000C11080BD90F824200168032A05D0022A57
:1028100005D0012A06D1143102E0163100E015314D
:10282000097800E0032180F88C10D0E90512C0E996
:102830002412704790F825200168032A05D0022A47
:1028400005D0012A06D1173102E0193100E0183114
:10285000097800E0002190ED070A90ED081AB8EE23
:10286000002A20EE020ABFEE082A21EE021A80F8A2
:10287000AC1080ED2C0A80ED2D1A704790F82710CF
:10288000027C0139CBB2022B80F8C12088BF70478F
:102890004FF4FF6202EAC10140F20012C0F20102ED
:1028A0004FF48033CA4023FA01F180F8C22080F847
:1028B000C3107047032180F88C10002180F8AC1001
:1028C00080F8C1107047000010B5044600F00AF807
:1028D000002818BF10BD2046FFF710FD2046FFF767
:1028E000D1FE10BD78B32DE9F04F83B0044654F803
:1028F000100F0190606B04F11C0B029001989BE893
:10290000C00F04F1040EA06304F154009EE82E50A1
:1029100080E8C00F0298A5640025E1632264636427
:10292000C4F84CC0C4F850E0E06600BFE8B22146ED
:10293000FFF79CFC0135042DF8D1002003B0BDE861
:10294000F04F40B27047FF2040B2704700000000D7
:1029500080B500EE100AB8EE400A10EE100A0CF036
:102960001FFB9FED110B53EC102B0CF055F80BF0E7
:102970001FFD00EE100A0BF0B5F99FED0D1A9FED4B
:102980000E2A20EE010A9FED0B1AB0EEC00A30EEBF
:10299000010AB4EE420AF1EE10FAC8BFB0EE420AE4
:1029A00080BD00BF00BF00BFFCA9F1D24D62503F07
:1029B000CDCC4C3E9A99193FCDCC4C3F2DE9F047F8
:1029C0002DED028B804600284FF0FE0000F0DD80E8
:1029D0000D46002900F0D980FFF794FBD8F80020BD
:1029E000801A61F100010CF030FB9FED6A0A01EEE4
:1029F000100A81EE000A88ED010AFFF783FB2979AE
:102A00000246C8F80000404600F0C8F808B1FD20B2
:102A1000BBE098F8080005280AD8DFE800F0030BAF
:102A2000030333220020C8E90300C8F814003FE084
:102A3000FD20AAE095ED020A95ED031A95ED052A11
:102A400095ED043A20EE020A22EE011A22EE033A34
:102A500088ED030A88ED041A88ED053A88ED062A08
:102A600026E0E869C8F80C0008F21460A96990ED46
:102A7000008AD8F80000C8F81010FFF769FF28EEA8
:102A8000000A13E0E869D8ED011AC8F80C00A8693B
:102A9000D8ED3F0A9FED401AC8F8100008F5747091
:102AA000B0EE000A05F0A0FAB1EE400A88ED050A82
:102AB00098ED030A08F2844004F022FA88ED030A34
:102AC00098ED040A08F2A44004F01AFA88ED040A0A
:102AD00098ED050A08F2C44004F012FA404688ED69
:102AE000050A00F0BDF89FED2C8A6FF00F0940F247
:102AF000E44A40F264544FF4807600BF08EB0907C3
:102B000097ED170AD7ED370A87ED1B0AD8ED011AA2
:102B100008EB06052846B0EE481A05F065FAD7ED31
:102B2000330AD8ED011A05F1F000B0EE481A05F0AD
:102B30005BFA08EB040087ED230A04F0E1F907F2E1
:102B4000146080ED000A97ED0F0AD7ED2B0A87ED90
:102B50001F0AD8ED011A05F5F070B0EE481A05F01D
:102B600043FA08EB0A0087ED270A04F0C9F907F2D7
:102B7000046019F104090AF1200A04F1200406F1A5
:102B80003C0680ED000AB9D1002040B2BDEC028BBA
:102B9000BDE8F08700007A4400000000F0B581B085
:102BA00030B10446007A0D46884203D100202BE064
:102BB000FE2029E0052D13D1052811D01046FDF780
:102BC00083FCFDF769FBC0074FF0FF3008BF012011
:102BD00000EE100AB8EEC00A04F2146080ED000A9C
:102BE0004FF48077E61906F5F07005F0FDFA06F16E
:102BF000F00005F0F9FA304605F0F6FA3C37B7F583
:102C0000F87FEFD10020257240B201B0F0BD000086
:102C1000F0B581B0044600F5BE668025D4F86004A6
:102C200096ED010A2844371D04F0B4FDD4F8600481
:102C300096ED050A2844203004F0ACFD0835A02D9F
:102C40003E46EBD1D4F86004803004F06FFCD4F839
:102C50006004A03004F06AFC01B0F0BD0000000088
:102C60002DE9F04F81B02DED028B8AB0077A044632
:102C7000012F3AD1E06820F000400CF091F99FED6F
:102C80002E0B55EC106B32462B460CF0C9F960BB8D
:102C9000206920F000400CF083F932462B460CF0FE
:102CA000BFF910BB606920F000400CF079F93246A2
:102CB0002B460CF0B5F9C0B994F80C0404F13C0CA7
:102CC000002804BF012084F80C040020C4E9070098
:102CD000C4E90900D4F8E405D4F8E815D4F8EC25E3
:102CE000D4F8F0358CE80F0027E2002084F80C04BB
:102CF0006FF00F002118CA6C0430C1F8F425F9D127
:102D0000052F00F21A820120B84010F00D0F1FD0DD
:102D10000020C4E90700C4E9090048F200000021CE
:102D2000C4F29D30C4F23421C4E90F01C4E9110199
:102D300003E200BF00BF00BF9A9999999999B93FE2
:102D4000CC3B7F669EA0E63FCD3B7F669EA0E63FE4
:102D5000D4E9030A65690CF023F9804628468946C0
:102D60000CF01EF91FED0A0B06465BEC102B5B46C0
:102D70000F460292CDF814B00BF04EFE42464B4681
:102D80000BF048FB02460B460BF046FE81465046D0
:102D900088460CF005F91FED140B05468A4653ECE6
:102DA000102B30463946CDE903230BF035FE2A4679
:102DB00053460BF02FFB02460B460BF02DFE02464E
:102DC0000B46484641460BF025FB41EC100B0BF03F
:102DD00051F851EC100B0BF0EBFAE061D4E9030869
:102DE00065690CF0DDF8074628468A460CF0D8F8ED
:102DF000029A5B46064689460BF00EFE3A4653465B
:102E00000BF008FB02460B460BF006FE82464046DE
:102E10008B460CF0C5F8DDE9032305460F46304626
:102E200049460BF0F9FD02460B46284639460BF0A1
:102E3000C9FF02460B460BF0EFFD02460B4650461B
:102E400059460BF0E7FA41EC100B0BF013F851EC7C
:102E5000100B0BF0ADFA2062D4E903016569019112
:102E60000CF09EF80746284689460CF099F8DDF8E4
:102E70000880059B424606468B460BF0CDFD024678
:102E80000B46384649460BF09DFF02460B460BF0B9
:102E9000C3FD814601988A460CF082F8DDE90323E0
:102EA00007460D46304659460BF0B6FD02460B4626
:102EB000384629460BF086FF02460B460BF0ACFD68
:102EC00002460B46484651460BF0A4FA41EC100B63
:102ED0000AF0D0FF51EC100B0BF06AFA6062D4E9F3
:102EE000030A65690CF05CF80746284689460CF031
:102EF00057F8059B424606468B460BF08DFD024671
:102F00000B46384649460BF05DFF02460B460BF078
:102F100083FD8146504688460CF042F80D465946DE
:102F2000DDF80CA0DDF810B00746304652465B468F
:102F30000BF072FD3A462B460BF06CFA02460B463C
:102F40000BF06AFD02460B46484641460BF062FA1A
:102F500041EC100B0AF08EFF51EC100B0BF028FA2D
:102F6000A062D4E9038066690CF01AF80546304681
:102F700089460CF015F852465B4606460F460BF0A4
:102F80004BFD2A464B460BF045FA41EC180B4046E8
:102F90000CF006F8029A059B0546884630463946ED
:102FA0000BF03AFD2A4643460BF034FA41EC110B84
:102FB000B0EE480AF0EE680A0AF03EFC51EC100B45
:102FC0009FED9F0B53EC102BCDE900230BF024FD5C
:102FD0000BF0EEF9E063D4E903A066690BF0E0FFC3
:102FE000054630468B460BF0DBFFDDF80C90049B6A
:102FF0004A4606460F460BF00FFD02460B46284692
:1030000059460BF0DFFE41EC180B50460BF0C8FFA1
:10301000DDF80880059B05468A463046394642461B
:103020000BF0FAFC2A4653460BF0F4F941EC110B75
:10303000B0EE480AF0EE680A0AF0FEFBDDE9002374
:1030400051EC100B0BF0E8FC0BF0B2F92064D4E962
:1030500003A066690BF0A4FF054630468B460BF0D3
:103060009FFF4A46DDF8109006464B460F460BF090
:10307000D3FC02460B46284659460BF0A3FE41EC12
:10308000180B50460BF08CFF4246DDF814800546C5
:103090008A463046394643460BF0BEFC02460B4694
:1030A000284651460BF08EFE41EC110BB0EE480A5B
:1030B000F0EE680A0AF0C0FBDDE9002351EC100BCA
:1030C0000BF0AAFC0BF074F96064D4E903A0666904
:1030D0000BF066FF054630468B460BF061FF039A06
:1030E0004B4606460F460BF097FC2A465B460BF014
:1030F00091F941EC180B50460BF052FF029A05462D
:103100008A463046394643460BF086FC02460B465B
:10311000284651460BF056FE41EC110BB0EE480A22
:10312000F0EE680A0AF088FBDDE9002351EC100B91
:103130000BF072FC0BF03CF9A0649FED430A04F124
:103140003C000021421892ED001A0431B5EE401AFD
:10315000F1EE10FABCBF31EE001A82ED001A102910
:10316000F0D19FED3A1A9FED3A2A9FED3A3A9FED42
:103170003A4A9FED3A5A002006A90AE0F1EE600AA9
:1031800036EE076AC2ED0B0A0130042882ED136A9D
:103190004DD004EB800292ED0F7A92ED336A01EB91
:1031A000800337EE467AB4EE417AF1EE10FA83ED01
:1031B000007A08DD37EE027AB4EE417AF1EE10FAC9
:1031C000F8DC83ED007A93ED007AB4EE437AF1EE09
:1031D00010FA08DA37EE007AB4EE437AF1EE10FA1C
:1031E000F8DB83ED007AB4EE447AF1EE10FA0BDDF1
:1031F000B4EE417AF1EE10FA06DCD36936EE076AD6
:10320000D36236EE036ABFE7D2ED070AB4EE457A21
:10321000F1EE10FAB2DAB4EE437AF1EE10FAADDB69
:1032200036EE076AC2ED0B0A36EE016AACE70AB069
:10323000BDEC028B01B0BDE8F08F00BF00BF00BF46
:1032400000000000DCA54C400000B4430000344303
:103250000000B4C3000034C30000B4420000B4C294
:1032600090ED001AF5EE400AF1EE10FA31EE000A88
:1032700010DDB4EE600AF1EE10FAA2BF30EE600A83
:1032800080ED000A7047B5EE400AF1EE10FAB8BFC3
:1032900030EE200A80ED000A70470000B5EE401ABB
:1032A000F1EE10FA30EE600AD8BF7047B6EE002A91
:1032B00021EE022AB4EE420AF1EE10FAC4BF30EE5B
:1032C000410A7047B1EE422AB4EE420AF1EE10FA1A
:1032D000B8BF30EE010A704790ED001AB4EE601AE4
:1032E000F1EE10FAC8BFC0ED000A90ED001AB4EE7E
:1032F000401AF1EE10FAB8BF80ED000A70470000E6
:103300004CF20400C2F201007047000080B540F2A8
:103310001870C2F2000001F00DFC80BD80B54CF6C3
:10332000D840C2F2010001F005FC80BD80B540F23A
:10333000B860C2F2000001F0FDFB80BD80B54CF624
:103340007840C2F2010001F0F5FB80BD80B540F28B
:103350007870C2F2000001F0EDFB80BDD0F800C033
:103360006FF00F024AF6AB2352FA8CF2CAF6AA2388
:103370000146A2FB0330000905A31B5C40F2FF30AD
:103380002CEA00005F2A88BF0430C1E916037047A9
:1033900000061016000610168269816AB2F5005FF9
:1033A00006D06AB9022912D0012914D0D1B90EE091
:1033B000032917D8DFE801F0020B020F0120704744
:1033C00003293CBF012070471CBF00207047C06A22
:1033D000C0F300607047C06AA0F1C070B0FA80F01E
:1033E000400970470020704780B5D0F800C0D0F881
:1033F00008E0DCF80000BEF1400F20F48020CCF89B
:1034000000000846CCF8043004BF10460A46CCF849
:103410000800CCF80C2080BD10B5E8B14CF669640A
:10342000C2F20104207810B1FD2040B210BD07F0B7
:1034300043FC4DF61431C2F20101086060B143F261
:103440006142C0F6000202200321FEF7B1FE012016
:103450002070002040B210BDFE2040B210BD000020
:1034600080B54DF61430C2F201000068012107F06A
:1034700085FB80BD70470000002843D0B0B50446EE
:10348000451C02202070204600F05EF8E869296A99
:103490006A6AAB6A2860B4F92D00AA60EB606960C3
:1034A00003F01CFDB4F92F106074084603F016FDFC
:1034B000B4F93110A074084603F010FDB4F93310CC
:1034C000E074084603F00AFDB4F93510207508468B
:1034D00003F004FDB4F937106075084603F0FEFCF4
:1034E000B4F93910A075084603F0F8FCB4F93B10A4
:1034F000E075084603F0F2FC20760020BDE8B040FD
:1035000040B27047FE2040B270470000B0B10321C6
:103510000170002180F83D10C0F80110C0F80510BE
:10352000C0F80910C0F80D10C0F81110C0F815103F
:10353000C0F81910C0F81D1048B27047FE2148B2FB
:1035400070470000000000002DE9F0472DED088BCA
:10355000002800F01A8140F22821C2F200014B78C5
:103560008F78012267F30A2300EE103AB8EEC00A02
:1035700000F11D0480F83D2010EE102A2260CA7868
:10358000FB0862F34A1300EE103AB8EEC00A10EEE0
:10359000103AE3600B794F799B0043EA921207F0EF
:1035A000010342EA832200EE102AB8EEC00A10EEB0
:1035B000102A62608A797B0862F3CA1301EE103A1E
:1035C000B8EEC11A11EE103AA3600F7ACB794E7A99
:1035D00012097F0063F30A1247EAD31306F00307C8
:1035E0008D7A43EA4723A0F82D30B308CF7A65F3EC
:1035F0008A13A0F83730FB000F7B4E7B43EA55134C
:10360000A0F8353066F30A278B7BA0F83370F708F3
:10361000CE7B63F34A17A0F83170B7000E7C47EAFF
:10362000931306F0010743EA8723497C9FED5E8AE6
:103630009FED5E9AA0F82F307308BFEE00AAB7EE98
:1036400000BA61F3CA13F0EE480AB0EE491AF0EE80
:103650004A1AB0EE4B2AA0F83920A0F83B30A0F867
:10366000392007F025F8216810EE100A00EE101A34
:10367000F0EE480AB0EE491AF0EE4A1AB0EE4B2AC4
:10368000606007F015F8A16810EE100A00EE101A3D
:10369000F0EE480AB0EE491AF0EE4A1AB0EE4B2AA4
:1036A000206007F005F8E16810EE100A00EE101A2D
:1036B000F0EE480AB0EE491AF0EE4A1AB0EE4B2A84
:1036C000A06006F0F5FF206810EE108AC4F80C80A8
:1036D0000BF066FC9FED300B074659EC10AB5246E1
:1036E0004B460E460BF0A3FC58B99FED2D0B384608
:1036F00053EC102B31460BF08CFC002804BF00204B
:10370000206060680BF04CFC52464B4606460F4664
:103710000BF08DFC58B99FED220B304653EC102B6B
:1037200039460BF076FC002804BF00206060A068DA
:103730000BF036FC52464B4606460F460BF077FC24
:1037400058B99FED170B304653EC102B39460BF050
:1037500060FC002804BF0020A06040460BF020FC65
:1037600052464B4606460F4600250BF060FC68B9F2
:103770009FED0B0B304653EC102B39460BF049FCF8
:10378000002804BF0025E56000E0FE2568B2BDEC1E
:10379000088BBDE8F08700BF7B14AE47E17A84BF99
:1037A0007B14AE47E17A843F0080B04300E0D3440D
:1037B00080B5012001F048FB80BD000080B50820E5
:1037C00001F042FB80BD000080B5102001F03CFB01
:1037D00080BD000080B5202001F036FB80BD0000D8
:1037E00072B600BFFEE7000070B52DED0E8B0446EB
:1037F00000284FF0FF0000F0B6810D46002900F0D0
:10380000B281FEF77FFCD4E90023801A99410BF0C6
:103810001CFC9FEDD70A01EE100A81EE000A84ED30
:10382000020AFEF76FFC2A78C4E90001204611461F
:1038300000F05CFB204606F02BFF94ED02DA95EDDC
:10384000010A95ED02EA04F5367004F5287120EEC0
:103850000DAA06F03BFF94ED141AB0EE408A9FEDDE
:10386000C59A94ED740A38EE011A7AEE010AB0EEA8
:10387000491AFFF713FD94ED141AB0EE40BA94ED17
:10388000750A38EE011A7AEE010AB0EE491AFFF70E
:1038900005FD607C02280BD0012800F0AC800028D8
:1038A00040F048810020C4E99300C4F8540241E18B
:1038B0009FEDB09A04F5F2752846B0EE4A0AF0EE94
:1038C000490AFFF7CDFC94ED790A9FEDAB1AB4EEEF
:1038D000410AF1EE10FA05DD9FEDA82A30EE020A4A
:1038E00085ED000A95ED003A9FEDA52AB1EE484A14
:1038F000B4EE423AF1EE10FABCBF33EE093A85ED70
:10390000003A9FED9E3AB4EE428A33EE485AF1EE09
:1039100010FAB8BFB0EE454AB4EE424A94ED796A67
:1039200034EE095AF1EE10FAB8BFB0EE454A34EE63
:10393000064AB4EE414A34EE033AF1EE10FAC8BF3B
:10394000B0EE434AB4EE424A34EE091AF1EE10FAF0
:10395000B8BFB0EE414AE06894ED151A41782DEEFB
:103960000E0A30EE010A84ED144A84ED150A39B1CD
:10397000D0ED460A90ED470A04F15400FFF7ACFC85
:10398000D4ED021A94ED130AD4EDB20A94EDB31AF1
:1039900004F1680004F028FB9FED7AAA84ED930AF5
:1039A000D4ED021AD4ED0D0A94ED140A04F1E000EE
:1039B000B0EE4A1A04F018FBD4ED021AD4ED0A0A4C
:1039C00004F58E70B0EE4A1AB0EE408A04F00CFB9B
:1039D00084ED940AD4ED021AD4ED0C0A94ED150A84
:1039E00004F5AC70B0EE4A1A04F0FEFAD4ED021AF7
:1039F000D4ED090A73E020462946B0EE40CA04F12E
:103A0000500600F0C1F8E068007838B13046B0EEFA
:103A10004C0AF0EE4B0AFFF75FFC1BE096ED000A44
:103A20009FED551AB4EE410AF1EE10FA05DD9FED57
:103A3000531A30EE010A86ED000A96ED000A9FED5A
:103A4000501AB4EE410AF1EE10FABCBF30EE090A8A
:103A500086ED000AE068417839B1D0ED460A90ED74
:103A6000470A04F15400FFF737FCD4ED021A94ED35
:103A7000130AD4EDB60A94EDB71A04F1680004F005
:103A8000B3FA9FED40AA84ED930AD4ED021AD4ED67
:103A90000D0A94ED140A04F1E000B0EE4A1A04F0A5
:103AA000A3FAD4ED021AD4ED0A0A04F58E70B0EE32
:103AB0004A1AB0EE408A04F097FA84ED940AD4EDE5
:103AC000021AD4ED0C0A94ED150A04F5AC70B0EEB0
:103AD0004A1A04F089FAD4ED021AD4EDA60AB0EE1F
:103AE000409A04F5CA70B0EE4A1A04F07DFAE06814
:103AF00084ED950A90F8041169B194EDA72A90ED30
:103B0000421A94ED943A38EE422A21EE021A33EE2C
:103B1000011A84ED941A90F8051159B194EDA51A83
:103B200090ED432A39EE411A22EE011A30EE010AD5
:103B300084ED950A94ED930A04F5F67003F0E0F92C
:103B400084ED930A94ED940A04F5037003F0D8F918
:103B500084ED940A94ED950A04F50B7003F0D0F906
:103B6000002084ED950A40B2BDEC0E8B70BD00BF05
:103B700000247449DB0FC940DB0F4940DB0FC9C08B
:103B8000DB0F49C00000000000284FF0FF0218BF03
:103B9000002901D150B270474A78022A19D0AAB937
:103BA00091ED010A91ED021A90ED022A90ED143A7E
:103BB00090ED154A20EE020A22EE011A33EE000AB9
:103BC00034EE011A80ED140A80ED151A002250B26D
:103BD0007047CA68026509690022416550B27047A2
:103BE000002808BF7047C16891F8FB20022A05D061
:103BF000012A08D05AB990EDA90A06E090EDAA0A68
:103C0000B1EE400A01E090EDA80A80ED0C0A91F8AF
:103C1000FC20022A05D0012A06D04AB900F52972F3
:103C200004E000F52A7201E000F528721268426390
:103C300091F8F820022A05D0012A06D04AB900F5E9
:103C4000257204E000F5277201E000F52672126883
:103C5000426291F8F910022905D0012906D049B92C
:103C600000F5257104E000F5277101E000F52671EB
:103C70000968816200F52B7C9CE80E103C3080E8DE
:103C80000E10704710B52DED028B002800F09480C7
:103C90000446C1600020607404F1680001F158021C
:103CA0000121B0EE408A04F057FAE16804F1A40063
:103CB00001F138020121B0EE480A04F04DFAE16842
:103CC00004F1E00001F198020121B0EE480A04F08D
:103CD00043FAE16804F58E7001F178020121B0EE3B
:103CE000480A04F039FAE16804F5AC7001F1D80231
:103CF0000121B0EE480A04F02FFAE16804F5CA7019
:103D000001F1B8020121B0EE480A04F025FAE0689A
:103D100090ED4B0A90ED4C1AD0ED440A30EE011AAA
:103D200084ED750A04F5F670B0EE480A84ED741A55
:103D300003F024F9E068B0EE480AD0ED440A04F537
:103D4000037003F01BF9E068B0EE480AD0ED440AB6
:103D500004F50B7003F012F9FDF7A0FDE06881781F
:103D6000012902D10E3003F0B9FCE068817831B945
:103D7000063003F08FFAE068063003F09DF9E06842
:103D80000179012902D12E3003F0A8FCE068C17846
:103D9000012902D1263003F0A1FCE068017931B994
:103DA0001E3003F077FAE0681E3003F085F9E06812
:103DB000C17819B1002009E0FF2007E0163003F0B8
:103DC00069FAE068163003F077F9002040B2BDECE4
:103DD000028B10BD10B50446C0688178012908D156
:103DE0000E3003F0A3FBE06894ED930A0E3003F06D
:103DF000D1FCE0688178E1B9D0F8401194ED930AE4
:103E0000C4F86012D0F84811C4F86812D0F8441110
:103E1000C4F86412D0F83C11C4F85C1290ED5D1A3D
:103E200004F5167120EE010A063084ED960A03F0BF
:103E30009DF9E0680179012908D12E3003F076FB65
:103E4000E06894ED940A2E3003F0A4FCE068C17899
:103E5000012908D1263003F069FBE06894ED950A4A
:103E6000263003F097FCE068C178E1B9D0F868111A
:103E700094ED950AC4F88812D0F87011C4F8901225
:103E8000D0F86C11C4F88C12D0F86411C4F8841204
:103E900090ED5F1A04F5207120EE010A163084EDD2
:103EA000A00A03F063F9E0680179002918BF10BD8A
:103EB000D0F8541194ED940AC4F87412D0F85C113F
:103EC000C4F87C12D0F85811C4F87812D0F8501108
:103ED000C4F8701290ED5E1A04F51B7120EE010A11
:103EE0001E3084ED9B0A03F041F910BDB0B52DEDF5
:103EF000028BC8B30446407C0D46884234D004F19E
:103F0000680004F071F904F1A40004F06DF904F103
:103F1000E00004F069F904F58E7004F065F904F529
:103F2000AC7004F061F904F5CA7004F05DF99FED1E
:103F3000108A04F5F670B0EE480A03F071F804F543
:103F40000370B0EE480A03F06BF804F50B70B0EEA6
:103F5000480A03F065F804F15000FCF765FDD4E968
:103F6000A8016574C4E91401BDEC028BB0BD00BFAB
:103F70000000000010B5002800F085800446C068ED
:103F80008178012911D10E3003F054FCE0680E3025
:103F900003F06AFB48B100F108030ECB406904F559
:103FA000327C8CE80E00C4F8D402E068817889B9CC
:103FB000063003F04DFAE068063003F0ABF848B184
:103FC00000F11C030ECB806A04F5327C8CE80E00F5
:103FD000C4F8D402E0680179012911D12E3003F030
:103FE00029FCE0682E3003F03FFB48B100F10803E4
:103FF0000ECB406904F5367C8CE80E00C4F8E40270
:10400000E068C178012911D1263003F013FCE06883
:10401000263003F029FB48B100F108030ECB4069BC
:1040200004F53A7C8CE80E00C4F8F402E0680179EB
:1040300089B91E3003F00CFAE0681E3003F06AF80C
:1040400048B100F11C030ECB806A04F5367C8CE885
:104050000E00C4F8E402E068C17889B9163003F0B4
:10406000F7F9E068163003F055F848B100F11C0389
:104070000ECB806A04F53A7C8CE80E00C4F8F4029A
:10408000002040B210BDFF2040B210BD10B380B57B
:104090008B68D1E900C2C0F89C32C0E9A5C24B6967
:1040A000D1E903C2C0F8A832C0E9A8C201F1280CC6
:1040B0009CE80C1000F52F7E8EE80C10D1E906C3A9
:1040C000D1E90821C0E9ABC3C0E9AD21FFF788FD04
:1040D000BDE880404FF0FF307047000090F820208E
:1040E000013A012A04D8006800F11402002004E01B
:1040F00000F1240201204FF480211368194311605C
:104100007047000010B590F820E0D0F800C0AEF184
:10411000010EBEF1010FDCF808E00ED81EF0E05FE2
:1041200011D0CEF3016E012000FA0EF018608B68FA
:104130007BB1486843EAC0030DE000F1240101208F
:104140004FF4802223E000F1240101204FF40012FB
:104150001DE008684305D1E9030403430CEB0E108E
:10416000C0F88031C0F88441097D012905D100F5EE
:10417000C2710B6843F480730B605168C0F88C11F6
:10418000126800F5C071C0F88821002001220B6878
:104190001A430A6010BD0000B0B590F82020013A23
:1041A000012A2FD846F20060C4F20000026842F0F3
:1041B00001020260026822F47C520260D1F814E02D
:1041C000CC694A6A0368012C43EA022202600EF0BD
:1041D0001F024FF0010303FA02F2C3696FEA020CF7
:1041E00023EA0203C36113D02CBBC36803EA0C03A8
:1041F000C360CB688C8844EA034300EBCE0423649D
:104200000B4611E0416A41F4802141620120B0BDBA
:10421000C3681343C3600B688C8844EA034300EB14
:10422000CE04236401F10C038C681B8843EA044329
:1042300000EBCE04636443688D6943EA0204D1F85D
:1042400010E0096A002D08BF03EA0C0444604369CA
:10425000BEF1000F43EA020408BF03EA0C0401297F
:10426000446102D1C1691143C161016821F00101BA
:1042700001600020B0BD000080B5FDF7E5FF032818
:1042800008BF80BD4CF25841C2F20101342210FB3C
:104290000210006B002818BF804780BD90F82020D6
:1042A000013A012A84BF00207047006810220029CB
:1042B00008BF0C22805800F00300704710B590F83A
:1042C0002040013C012C0AD8046871B12469A4077C
:1042D0000ED100F1240101204FF4001276E000F12C
:1042E000240101204FF4802270E0E468A40771D01B
:1042F000046804EB011CDCF8B0410CF5D87E14F026
:1043000004049460DCF8B04119BFE4085460640D03
:104310001460DEF800400CF5DA7E04F00204D4608C
:10432000DCF8B44124075ABFDEF8004004F00F0463
:1043300008241461DEF800400029C4F307249461C6
:10434000DEF800404FEA14445461DCF8B8211A70DA
:10435000026802EB0112D2F8B8214FEA12225A7019
:10436000026802EB0112D2F8B8214FEA12429A70A9
:10437000026802EB0112D2F8B8214FEA1262DA7039
:10438000026802EB0112D2F8BC211A71026802EB3A
:104390000112D2F8BC214FEA12225A71026802EBD4
:1043A0000112D2F8BC214FEA12429A71026802EB64
:1043B0000112D2F8BC214FEA1262DA71006814BF10
:1043C00000F1100100F10C01002020220B681A43BB
:1043D0000A6010BD00F1240101204FF40012F5E73E
:1043E00090F820100139012984BF0020704700682F
:1043F000816882688068C1F38061C2F3C062114441
:10440000C0F30070084470472DE9F04F81B00446B6
:1044100000684669D0F804908768D0F80CB0D0F8EE
:1044200010A0D0F81880F10703D1002530071CD464
:1044300023E0F90710D00121BA07816009D4780779
:1044400000F1AA80380700F1B080204600F0A2FAFF
:1044500002E0204600F0B0FA0025F80500F1848063
:10446000F80300F1AA80300707D51BF0100004D034
:10447000206845F400751021C160700708D51BF055
:10448000080005D020680821C160204600F0FAF934
:10449000B00706D52068C068800702D0204600F02B
:1044A00003FA700607D51AF0100004D0206845F40E
:1044B000806510210161B00608D51AF0080005D00A
:1044C000206808210161204600F000FAF00606D5B8
:1044D00020680069800702D0204600F009FAB00386
:1044E00008D519F0100005D0206810214160204641
:1044F00000F010FAF00308D519F0080005D0206884
:1045000008214160204600F0B1FA300440F18F806C
:104510005FEA497040F1888006F4807008EA102054
:1045200028435FEA8871014648BF41F00201B205A5
:1045300058BF01465FEA48700D4648BF45F0040584
:10454000700558BF0D4630056ED518F070006BD061
:1045500010380009052862D8DFE800F003535659E7
:104560005C5F45F008055AE020684FF48071BA0599
:1045700081600AD4780512D4380519D4204600F099
:104580002DFAF8037FF56FAF17E0204600F038FAF8
:10459000F8037FF568AF10E04FF400655DE705F5BF
:1045A0000055F8037FF55FAF07E04FF4805554E7FF
:1045B00005F58045F8037FF556AF20684FF480314C
:1045C000BA0381600AD478030FD4380313D4204689
:1045D00000F028FA30073FF548AF4EE7204600F0DC
:1045E00033FA30073FF541AF47E705F5004530079F
:1045F0003FF53BAF41E705F5803530073FF535AF77
:104600003BE745F010050AE045F0200507E045F0DE
:10461000400504E045F0800501E045F48075206820
:10462000816921F0700181612068042141602DB110
:10463000606A284360622046FFF71EFE01B0BDE8B5
:10464000F08F0000B0B5C8B1044690F8200010B952
:10465000204600F071F82068016841F00101016016
:1046600000F0DAFC054600BF20684168C90707D1A1
:1046700000F0D2FC401B0B28F6D312E00120B0BDA5
:10468000016821F00201016000F0C6FC054600BF90
:104690002068416889070DD500F0BEFC401B0B283F
:1046A000F6D3606A052140F400306062012084F88E
:1046B0002010B0BD217E0268012922F0800208BFCF
:1046C00080320260617E0268012922F0400208BF48
:1046D00040320260A17E0268012922F0200208BF58
:1046E00020320260E17E0268012922F0100218BF28
:1046F00010320260217F0268012922F0080208BFFF
:1047000008320260617F0268012922F0040208BFBA
:1047100004320260D4E901C2D4E9033561691A4365
:104720002A431143ACF101021143C1610020012170
:10473000606284F82010B0BD70B586B0006846F69F
:104740000002C4F2000200219042CDE90411CDE93B
:104750000211019137D046F20041C4F200018842B3
:1047600040F08D8040F25411C2F200010A6843F615
:104770004000C4F20200531C0B6052B900210091AA
:10478000016841F000710160016801F00071009161
:1047900000990021009150F8101C152441F00801E7
:1047A00040F8101C50F8100C142500F00800009080
:1047B00000980320019040F20040C4F2020000F58E
:1047C0000060132638E043F64000C4F20200009176
:1047D000016841F080610160016801F08061009131
:1047E000009940F25411C2F200010A68531C0B6098
:1047F00052B900210091016841F000710160016827
:1048000001F00071009100990021009150F8101CF6
:10481000412441F0020140F8101C50F8100C4025D2
:1048200000F00200009000984FF48250019040F296
:1048300000403F26C4F202000221029100210391B0
:10484000032104910921059101A900F00BFB3046D9
:104850000521002200F09CFD304600F095FD284621
:104860000521002200F094FD284600F08DFD204631
:104870000521002200F08CFD204600F085FD06B0E9
:1048800070BD000080B5FDF7DFFC032808BF80BDC8
:104890004CF25841C2F20101342210FB0210C069EF
:1048A000002818BF804780BD80B5FDF7CDFC0328E8
:1048B00008BF80BD4CF25841C2F20101342210FB06
:1048C00002108069002818BF804780BD80B5FDF7C1
:1048D000BBFC032808BF80BD4CF25841C2F2010165
:1048E000342210FB0210406A002818BF804780BDA8
:1048F00080B5FDF7A9FC032808BF80BD4CF25841E4
:10490000C2F20101342210FB0210006A002818BF15
:10491000804780BD80B5FDF797FC032808BF80BDA8
:104920004CF25841C2F20101342210FB0210806A9D
:10493000002818BF804780BDB0B5044690F820001D
:1049400001281DD1022084F820002068016821F090
:104950000101016000F060FB054600BF206840686F
:10496000C00713D000F058FB401B0B28F6D3606A39
:1049700040F400306062052084F820000120B0BDC2
:10498000606A40F4002060620120B0BD00206062D7
:10499000B0BD000080B5FDF757FC032808BF80BDFF
:1049A0004CF25841C2F20101342210FB0210C068DF
:1049B000002818BF804780BD80B5FDF745FC03285F
:1049C00008BF80BD342148434CF25841C2F2010176
:1049D0000858002818BF804780BD000080B5FDF74B
:1049E00033FC032808BF80BD4CF25841C2F20101DC
:1049F000342210FB02100069002818BF804780BDD8
:104A000080B5FDF721FC032808BF80BD4CF258415A
:104A1000C2F20101342210FB02104068002818BFC6
:104A2000804780BD80B5FDF70FFC032808BF80BD1F
:104A30004CF25841C2F20101342210FB02104069CD
:104A4000002818BF804780BD80B5FDF7FDFB032817
:104A500008BF80BD4CF25841C2F20101342210FB64
:104A600002108068002818BF804780BD80B5FDF720
:104A7000EBFB032808BF80BD4CF25841C2F2010194
:104A8000342210FB0210C06A002818BF804780BD86
:104A900070B5866D044600F0BFFA94F8351002290F
:104AA00025D105462068216C026822F016020260BA
:104AB000426922F08002426109B9A16C19B1016812
:104AC00021F008010160016821F00101016000BFCF
:104AD00020680068C0070ED000F09EFA401B062830
:104AE000F6D320206065032084F835000CE0802098
:104AF0006065012008E0E06D3F2101FA00F0B06040
:104B0000012084F835000020002184F8341070BDA5
:104B100090F83510022909D1052180F83510006878
:104B2000016821F00101016000207047802141658A
:104B300001207047F0B581B00446002000904CF28F
:104B40000000C2F201000268D4E9166048F2B51311
:104B500037680821C1F64E3381403942A2FB032554
:104B60000CD0226813685B0708D5136823F0040390
:104B70001360B160616D41F0010161650121814007
:104B8000394208D022685269120604D5B160616DBD
:104B900041F00201616504218140394208D0226858
:104BA0001268920704D5B160616D41F0040161653E
:104BB00010218140394215D020680268120711D5B2
:104BC000B16002680168520306D4C90506D40168C1
:104BD00021F00801016001E0080342D4216C09B111
:104BE00020468847E16D202000FA01F23A4244D085
:104BF00020680368DB0640D5B26094F8353002685F
:104C0000052B1ED122F016020260426922F08002BA
:104C10004261226C0AB9A26C1AB1026822F0080241
:104C200002603F208840B060012084F83500216D8B
:104C30000020002984F8340040D02046884701B085
:104C4000F0BD0168520310D4C90512D4016821F0E7
:104C500010010160012084F83500002084F8340040
:104C600007E0A16C0029BBD1BCE7080301D4616C4B
:104C700000E0E16B09B120468847606DF0B1606DDE
:104C8000C00717D0052084F835002068A90A0268FB
:104C900022F00102026000BF009A01328A420092B3
:104CA00002D80268D207F7D1012084F8350000202D
:104CB00084F83400E16C09B12046884701B0F0BDAA
:104CC0002DE9F041044600F0A7F9C4B105460220E1
:104CD00084F835000020216884F83400086820F04A
:104CE0000100086026683068C0070BD000F094F916
:104CF000401B0528F6D903212022032042E0012091
:104D0000BDE8F081306848F23F01CFF21001251D67
:104D100000EA010C2ECDD4E9050E41EA0C01114345
:104D200019432943D4E90778084340EA0E01606A31
:104D30003943042841EA080103D1D4E90B23114384
:104D4000194331607169042821F0070141EA000527
:104D50000CD1D4E90A1045EA010538B12046FEF726
:104D60001BFB18B10121402201200BE02046756198
:104D7000FEF7F4FAE16D3F2202FA01F181600022B0
:104D800001210020626584F83510BDE8F081000043
:104D9000B0B5044690F83400012828D0012084F8EA
:104DA0003400A56D94F8350001281DD1022084F847
:104DB0003500002060652046FEF716FBE26D3F23BC
:104DC000206803FA02F2216CAA60026842F016021F
:104DD000026019B1016841F008010160016841F009
:104DE000010101600020B0BD002084F834000220E1
:104DF000B0BD0000B0B5044600F00EF9054640F223
:104E00002800C2F200000078611C18BF044400BFF3
:104E100000F002F9401BA042FAD3B0BD70B540F2D9
:104E2000141604460025C2F2000603E00135102DD9
:104E300008BF70BD24FA05F0C007F7D056F825006A
:104E4000002818BF8047F1E780B543F61441C4F24B
:104E500001010A68024208BF80BD0860FFF7DEFF5B
:104E600080BD00002DE9F04F83B000F13E4202F119
:104E7000FF724FEAB22241F600470192C4F20207E4
:104E800008224FF0010E00254FF0000A4FF00008F5
:104E9000B84208BF072200920AE000BF08F10108EB
:104EA0000AF1040AB8F1100F05F1020500F0A48020
:104EB0000C680EFA08FB14EA0B09EFD04C6804F0FA
:104EC000030CACF1010EBEF1010F11D8032287686B
:104ED00002FA05F6CA68B743AA403A4382604268BC
:104EE000C4F3001722EA0B0207FA08F73A434260BC
:104EF000BCF1030F1CD0C26803238E6803FA05F7C8
:104F0000BA4306FA05F73A43BCF1020FC2600FD16B
:104F10006FF0030202EA580202440AF01C060F2353
:104F2000176A03FA06F40B69A743B3403B431362C5
:104F3000026803234F68AB409A4307F00303AB407A
:104F40001A4317F4403F4FF0010E0260A6D0002232
:104F500043F644030292C4F202031A6843F6004483
:104F600042F480421A601A68C4F2010402F48042DA
:104F70000292029A28F003024FF6084B2244CFF621
:104F8000FF7B52F80B300AF00C070F26BE4023EAD5
:104F9000060C019B009E072B38BF1E4606FA07F73A
:104FA00047EA0C0342F80B30A2684B6842EA090753
:104FB00043F60C4CDE0258BF22EA0907A760C4F290
:104FC000010CDCF800209E0242EA090758BF22EAE1
:104FD0000907CCF8007062689E0342EA090758BFCF
:104FE00022EA090767602268DB0342EA090358BF27
:104FF00022EA0903236051E703B0BDE8F08F000007
:105000000069084018BF012070470000002A08BF4F
:1050100009048161704700004AF28830C2F2010041
:1050200000687047F0B581B0B0B3044690F83D0019
:1050300028B9002084F83C00204600F0BFF8242066
:1050400084F83D002068016821F0010101600168D9
:1050500041F400410160016821F40041016000F069
:1050600061FA48F28041C0F21E0140F60012656804
:1050700088424FF00001C0F23D0248F2A16C4FF0AF
:10508000000338BF01219042C0F2010C38BF012358
:10509000654538BF0B4613B1012001B0F0BD4DF698
:1050A0008361C4F21B31A0FB011221684FEA924ECA
:1050B0004B684FF4967623F03F0343EA92434B60EC
:1050C00044F6D3530F6A0EFB06F6C1F26203A6FB49
:1050D000033627F03F03B709654538BF970C7A1CA4
:1050E0001A430A62CA6948F2A0674CF6FF73C0F21D
:1050F0000107BD4222EA030C0AD801386A00B0FB5E
:10510000F2F001306FF31F30042898BF04202BE029
:10511000A368A0F1010E9BB119206843BEFBF0F01B
:105120000422013062F31F30000512D09BB1192018
:105130006843BEFBF0F00422013062F31F3011E03F
:1051400005EB4500BEFBF0F001306FF31F300005AA
:10515000ECD1012008E005EB4500BEFBF0F001308A
:105160006FF31F3040F4004040EA0C00C86108684B
:10517000D4E9072320F0C000104318430860886872
:1051800048F2FF3204F10C0790438CCF18431043D0
:10519000A6698860C86820F0FF0038433043C860C3
:1051A000086840F00100086000202021206484F895
:1051B0003D10206384F83E0001B0F0BDB0B586B06C
:1051C000006845F60001C4F2000100248842CDE9E0
:1051D0000444CDE90244019431D045F20041C4F2C7
:1051E0000001884254D1002443F630050094C4F2F3
:1051F0000205286801A940F002002860286800F034
:105200000200009000984FF4407001901220CDE908
:105210000204032004900420059040F20040C4F2F0
:105220000200FFF71FFE0094286940F40010286177
:10523000286900F400100090009806B0B0BD43F655
:1052400030050094C4F202052868122140F02000C5
:105250002860286800F0200000900098032001904A
:1052600004900420059040F20040C4F20200CDE911
:10527000021400F5805001A9FFF7F4FD009428699D
:1052800040F480002861286900F4800000900098B4
:1052900006B0B0BD40F228004AF28831C2F20000E8
:1052A000C2F2010100780A681044086070470000EB
:1052B00080B543F60040C4F20200016841F4007179
:1052C0000160016841F480610160016841F480710E
:1052D0000160032000F06CF80F2000F005F800F0EA
:1052E0002BF8002080BD0000B0B540F22802C2F2C9
:1052F00000024CF200011278C2F201014FF47A73FD
:105300000968B3FBF2F20446B1FBF2F1084601F082
:105310005DF80F2C4FF001050CD858B94FF0FF3055
:1053200021460022002500F033F84CF2F430C2F29E
:10533000010004602846B0BD80B582B0002043F66D
:1053400040010190C4F202014A6842F480424A607E
:105350004A6802F480420192019A00900868002293
:1053600040F08050086008680F2100F080500090E5
:1053700000986FF0010000F00BF802B080BD000053
:1053800080B504F0C1FF80BD80B504F0D1FF80BDC1
:1053900070B514460D46064604F0DAFF294622464B
:1053A00002F00CFE0146304604F0DAFF70BD00004A
:1053B00080B504F0EFFF80BD2DE9F041002800F03A
:1053C0008B8043F60808C4F202080446D8F8F803B4
:1053D0000D4600F00700884207D288F8F853D8F845
:1053E000F80300F00700A84276D12068810717D59E
:1053F000410705D5D8F8001041F4E051C8F8001075
:10540000010705D5D8F8001041F46041C8F8001034
:10541000D8F80010A26821F0F0011143C8F800107C
:10542000C0073FD1D8F8F80300F00700A84207D919
:1054300088F8F853D8F8F80300F00700A8424BD1D9
:105440002068410707D5D8F80010E26821F4E05140
:105450001143C8F80010000708D5D8F800002169EA
:1054600020F4604040EAC100C8F8000000F07EF877
:10547000D8F800104FF22022C1F30311C0F6000249
:10548000515C4CF2000220FA01F14CF2F430C2F20D
:1054900001000068C2F201021160FFF725FF002041
:1054A000BDE8F0816068811E022907D258F8081C07
:1054B00089015CBF0120BDE8F08110E0012807D11F
:1054C00058F8081C89035CBF0120BDE8F08106E0A4
:1054D00058F8081C890702D40120BDE8F081D8F8EB
:1054E000001021F003010843C8F80000FFF794FD05
:1054F000064641F2883700BFD8F80000616800F026
:105500000C00B0EB810F8DD0FFF786FD801BB842F9
:10551000F2D90320BDE8F0814CF20000C2F2010094
:105520000068704780B5FFF7F7FF43F60801C4F243
:10553000020109684FF23022C1F38221C0F6000255
:10554000515CC84080BD000080B5FFF7E5FF43F621
:105550000801C4F2020109684FF23022C1F342315E
:10556000C0F60002515CC84080BD000010B543F693
:105570000404C4F20204606800F00C0008280AD099
:10558000042819BF42F20040C0F2F40041F6003096
:10559000C0F2B70010BD206821682368490241F6B7
:1055A0000031C0F2B70100F03F02C3F388105CBFC6
:1055B00042F20041C0F2F401A1FB00010023FAF71E
:1055C000A5FE21680222C1F3014102EB4101B0FBBB
:1055D000F1F010BD2DE9F04182B0002800F0A2806A
:1055E0000446007843F60006C007C4F2020643D022
:1055F000B06800F00C00042805D1306880033BD56A
:105600006068C8BB8EE0B06800F00C00082802D1CA
:1056100070684002F1D46568B5F5A02F0AD0B5F5E1
:10562000803F0BD0306820F480303060306820F448
:10563000802006E0306840F480203060306840F41C
:1056400080303060FFF7E8FC002D054611D000BF28
:105650003068800310D4FFF7DFFC401B6428F7D9C3
:1056600022E100BFFFF7D8FC401B64284FF0030085
:1056700055D830688003F5D4207880071AD5B068F3
:1056800010F00C0F09D0B06800F00C00082840F0B2
:105690008A807068400200F186803068800702D5F9
:1056A000E06801283ED13068216920F0F80040EA26
:1056B000C10030602078000738D4207840074CD4EF
:1056C000A5695DB3B06800F00C00082840F09E802A
:1056D000012D27D07068E16900F480028A4221D14F
:1056E000216A00F03F028A421CD147F6C071626A0B
:1056F0000140B1EB821F15D1A26A0023CFF6FF73E0
:1057000003EBC23200F440316FF30F02914209D132
:10571000E16A00F07060B0EB016F03D1002002B0CD
:10572000BDE8F081012002B0BDE8F0816069002889
:1057300040F20000C4F2472057D00121C0F8801E7B
:10574000FFF76AFC054600BF706F8007B5D4FFF70E
:1057500063FC401B0228F7D9A6E0306C10F080589B
:105760000AD100200190306C40F080503064306CE1
:1057700000F080500190019847F20007C4F2000742
:105780003868C00524D4386840F480703860FFF76A
:1057900043FC05463868C0051AD4FFF73DFC401BA2
:1057A0000228F7D980E0E068002851D00020C4F238
:1057B000472001210160FFF72FFC05463068800774
:1057C0003FF571AFFFF728FC401B0228F6D96BE0CC
:1057D000A568052D50D0012D52D0306F20F001006A
:1057E0003067306F20F004004DE00021C0F8801ECB
:1057F000FFF712FC054600BF706F80077FF55DAFB5
:10580000FFF70AFC401B0228F6D94DE00027C4F23E
:10581000472700203866FFF7FFFB022D05460BD116
:105820003068800158D5FFF7F7FB401B02284FF086
:105830000300F5D973E700BF306880017FF56EAFD4
:10584000FFF7EAFB401B02284FF00300F4D966E79C
:105850000020C4F2472000210160FFF7DDFB054670
:10586000306880077FF526AFFFF7D6FB401B022884
:105870004FF00300F4D952E7306F40F00400306776
:10588000306F40F001003067FFF7C6FB002D054682
:1058900041F2883714D000BF306F800713D4FFF770
:1058A000BBFB401BB842F7D9032002B0BDE8F08132
:1058B000FFF7B2FB401BB8424FF003003FF62FAF9B
:1058C000306F8007F4D4B8F1000F7FF4F9AE306C7C
:1058D00020F080503064F3E604F11C052FCD08431E
:1058E0000021CFF6FF7140EA821001EBC3316FF364
:1058F0000F0140EA05600843706001203866FFF739
:105900008BFB0446306880013FF508AFFFF784FB4E
:10591000001B02284FF00300F4D900E780B502F025
:105920004DFE022808BF80BD4CF2C441C2F2010105
:1059300001EB40108069002818BF804780BD00003F
:1059400070B538B10446406A30B10020206104F1DE
:10595000140007E0012070BD6068B0F5827F03D0BD
:1059600004F11C00002101600026A66294F8510099
:1059700020B9204684F8506000F03CF8022084F8FA
:10598000510094E80F0001F48271056802F40442AA
:1059900025F040050560114403F4006223691144B9
:1059A00003F002026369114403F00102A369E5698F
:1059B000114403F40072114405F03802256A1144C1
:1059C00005F08002A56A114305F4005211430160FD
:1059D000626A042101EA134102F01002114441609D
:1059E000C16921F40061C1610120666584F851003C
:1059F000304670BD2DE9F04F87B0044643F20007F2
:105A00000068C4F201070026B8420696CDE9046694
:105A10000396029602D007B0BDE8F08F43F630003F
:105A20000196C4F20200416902AD41F48051416126
:105A3000416946F2404801F4805101910199019673
:105A400001684FF0020941F00201016001684FF066
:105A5000030A01F0020101910199019601684FF0DA
:105A6000050B41F0010101600068294600F00100CA
:105A7000019001981820029007F55440C4F20208E2
:105A8000CDE90396CDF814A0CDF818B0FFF7EAF9E8
:105A90008020CDE9020904A880E8400C07F55040B9
:105AA0002946FFF7DFF940F2B865C2F200054FF46E
:105AB00040304FF0C0674FF48069C5E908062846BA
:105AC000C5E90087C5E90266C5E90496C5E9066629
:105AD000FFF7F6F8002818BFFDF782FEE564AC6317
:105AE0004CF6784508F11800C2F201054021C5E9DD
:105AF000000705F10800002280E806024FF400309C
:105B0000C5E908022846C5E90522EA61FFF7D8F889
:105B1000002818BFFDF764FEA564AC6307B0BDE8BC
:105B2000F08F00002DE9F04182B0044690F851005A
:105B3000012815D10E4600294FF0010060D017460C
:105B4000002A5DD060681D46B0F5827F02D1A06852
:105B5000002858D0FFF760FA94F85010012903D1BB
:105B6000022002B0BDE8F0818046012084F8500098
:105B7000042084F8510000206065A663A787E787AA
:105B80002063A086E086A1682064B1F5004F6064C0
:105B900008D12068016821F040010160016821F40A
:105BA0008041016020680168490603D4016841F022
:105BB00040010160E168E08F91B3002855D06E1C70
:105BC0000BE000BFC068A16B21F8020BA163E08F5E
:105BD0000138E087E08F002847D020688168C90736
:105BE000F0D1FFF719FA002EF4D0A0EB0800A8427C
:105BF000F0D3012084F85100002084F850000320E5
:105C000002B0BDE8F081042084F8510020463146FE
:105C100032463B46009500F09FF902B0BDE8F081A6
:105C200018B36E1C0BE000BF007BA16B0870A06B6B
:105C30000130A063E08F0138E087E08FA8B12068D1
:105C40008168C907F0D1FFF7E7F9002EF5D0A0EB86
:105C50000800A842F1D3012084F85100002084F804
:105C60005000032002B0BDE8F0812046294642469C
:105C700002F016FC00281CBF20206065012084F87B
:105C80005100002084F85000606D002818BF0120EA
:105C900002B0BDE8F081000010B5044690F8510054
:105CA00001281CBF022010BD13460A4600294FF0F0
:105CB000010018BF002B00D110BDA06858B9616861
:105CC000B1F5827F07D1042084F8510020461146A7
:105CD00000F03EFA10BD94F85010012904BF0220D4
:105CE00010BD012184F85010042184F851100021C6
:105CF000B0F5004F6165A263A387E387C4E9101183
:105D0000A186E18608D12068036823F04003036080
:105D1000036823F480430360E06C48F2493E48F294
:105D20006D33C0F6000EC0F60003C0E90F3E48F226
:105D30002533C0F60003D4F800C0C0E91331E38F67
:105D40000CF10C01FFF724F840B1606D40F0100039
:105D50006065002084F85000012010BD21680868AB
:105D6000400603D4086840F040000860002084F832
:105D700050004A6842F020024A604A6842F001023C
:105D80004A6010BD80B502F019FC022808BF80BD32
:105D90004CF2C441C2F2010101EB401040680028FE
:105DA00018BF804780BD000080B502F007FC0228C4
:105DB00008BF80BD4CF2C441C2F2010101EB4010AA
:105DC0000069002818BF804780BD00002DE9F04120
:105DD00082B01D4616460F460446FFF71DF994F89B
:105DE000511001290DD18046002F4FF0010018BF3E
:105DF000002E02D102B0BDE8F08194F850000128D5
:105E000003D1022002B0BDE8F081012084F85000E7
:105E1000032084F85100002060652763A686E6868B
:105E2000A063A087E087A168C4E91000B1F5004F26
:105E300008D12068016821F040010160016841F447
:105E40008041016020680168490603D4016841F07F
:105E5000400101606168731EE268B1FA81F1B3FA32
:105E600083F349095B09B2F5006F41EA030124D1CC
:105E700039B1216B0988C160B81C2063E08E0138FC
:105E8000E086E08E002846D06E1C09E0216B31F8D8
:105E9000022BC2602163E08E0138E086E08ED0B331
:105EA000206881688907F1D4FFF7B6F8002EF5D095
:105EB000A0EB0800A842F1D323E039B1397801738F
:105EC000206B01302063E08E0138E086E08E10B355
:105ED0006E1C0AE0216B09780173206B013020638E
:105EE000E08E0138E086E08EA8B1206881688907DD
:105EF000F0D4FFF791F8002EF5D0A0EB0800A842EF
:105F0000F1D3012084F85100002084F850000320D0
:105F100002B0BDE8F08120462946424602F008FB67
:105F200000281CBF20206065A06838B900200190BF
:105F30002068C1680191806801900198012084F86F
:105F40005100002084F85000606D002818BF012027
:105F500002B0BDE8F08100002DE9F04381B01E469B
:105F600015460F460446FFF757F894F8511081463E
:105F7000012909D06068B0F5827F14D104294FF05F
:105F8000020007D1A16829B9002F4FF0010018BF06
:105F9000002D02D101B0BDE8F083002EFAD094F8B4
:105FA0005000012803D1022001B0BDE8F083012098
:105FB00084F8500094F85100002104281CBF0520EB
:105FC00084F851006165A563E687A6872763E686A6
:105FD0002068A686216461640168490603D40168CB
:105FE00041F0400101606168731EE268B1FA81F11D
:105FF000B3FA83F3DDF8208049095B09B2F5006F3D
:1060000041EA030139D139B1216B0988C160B81C5B
:106010002063E08E0138E086012608F1010500BF0B
:10602000E08E10B9E08F00286CD020688168890765
:106030000CD5E18E012E09D141B1216B002631F83A
:10604000022BC2602163E18E0139E1868168C907B4
:106050000AD0E18F41B1C068A16B012621F8020B83
:10606000A163E08F0138E087FEF7D6FF002DD7D07F
:10607000A0EB09004045D3D33AE039B13978017338
:10608000206B01302063E08E0138E086012608F1A4
:10609000010500BFE08E08B9E08F98B320688168E1
:1060A00089070DD5E18E012E0AD149B1216B002659
:1060B00009780173206B01302063E08E0138E0869F
:1060C00020688168C9070BD0E18F49B1C068A16B16
:1060D00001260870A06B0130A063E08F0138E087D3
:1060E000FEF79AFF002DD5D0A0EB09004045D1D393
:1060F000012084F85100002084F85000032001B0F2
:10610000BDE8F083204641464A4602F011FA40B10C
:1061100020206065002084F85000012001B0BDE817
:10612000F083A06838B9002000902068C168009111
:10613000806800900098012084F85100002084F8C5
:106140005000606D002818BF012001B0BDE8F08349
:1061500070B5044690F85100012806D100294FF08F
:10616000010018BF002A0CD170BD6568B5F5827FAB
:106170000ED104284FF00200F6D1A568002DEDD015
:10618000F2E7002B08BF70BD94F85000012801D140
:10619000022070BD012084F8500094F851000026C0
:1061A00004281CBF052084F8510066652163A3867E
:1061B000E386A263A387E387C4E9106694F85100DD
:1061C00048F2493148F26133C0F60001C0F60003DD
:1061D000042808BF0B4648F26D3048F24541C0F62E
:1061E0000000C0F6000108BF0146E06C2568C0E968
:1061F0000F1348F22531C0F60001C0E91316E38FF2
:1062000005F10C01FEF7C4FD38B1606D40F01000DF
:106210006065012084F8506070BD2268216BA06C1D
:10622000536843F001035360C0E90F66C0E9136689
:10623000E38E0C32FEF7ACFD40B1606D40F0100013
:106240006065002084F85000012070BD2168086856
:10625000400603D4086840F040000860002084F83D
:1062600050004A6842F020024A604A6842F0020246
:106270004A6070BD10B5044690F8510001280AD15B
:1062800000294FF0010018BF002A00D110BD94F87A
:106290005000012801D1022010BD012084F85000D7
:1062A0000320002384F8510063652163A286E286FF
:1062B000A363C4E91033A387E387A068B0F5004F58
:1062C00008D12068026822F040020260026842F4AD
:1062D00080420260A06C48F2553C48F2D532C0F6CC
:1062E000000CC0F60002C0E90F2C48F22532C0F6BF
:1062F0000002D4F800E0C0E91323E38E0EF10C0293
:10630000FEF746FD40B1606D40F010006065002072
:1063100084F85000012010BD21680868400603D4AD
:10632000086840F040000860002084F850004A6887
:1063300042F020024A604A6842F002024A6010BD00
:1063400080B502F03BF9022808BF80BD4CF2C44181
:106350004001C2F201010858002818BF804780BDE3
:1063600080B502F02BF9022808BF80BD4CF2C44171
:10637000C2F2010101EB4010C068002818BF80473D
:1063800080BD000080B502F019F9022808BF80BD69
:106390004CF2C441C2F2010101EB401080680028B8
:1063A00018BF804780BD000080B502F007F90228C1
:1063B00008BF80BD4CF2C441C2F2010101EB4010A4
:1063C0004069002818BF804780BD000080B502F0FA
:1063D000C1FF80BD7047000070470000002804BF67
:1063E0000120704710B5044690F83D0028B9002000
:1063F00084F83C00204600F01FF8022084F83D009D
:106400002068211D03F02CF8012084F8460084F850
:106410003E0084F83F0084F8400084F8410084F88E
:10642000420084F8430084F8440084F8450084F86E
:106430003D00002010BD000080B582B0006844F22D
:106440000041C4F20101884201D002B080BD0020A9
:10645000019043F64400C4F202000168002241F4B6
:10646000003101600068052100F4003001900198BE
:106470001920FEF78DFF1920FEF786FF02B080BDC0
:1064800070470000B0B504460068C168026902EABE
:106490000105A9071DD4680731D4280747D4E806A9
:1064A0005CD4E80773D128067BD4680606D520683B
:1064B0006FF040010161204600F0C0F9A80658BF06
:1064C000B0BD20686FF0200101612046FFF784FF16
:1064D000B0BD6FF002010161012121778069800761
:1064E00003D02046FFF7CCFF05E0204600F092F8ED
:1064F000204600F00DF9002020776807CDD52068F0
:106500006FF00401016102212177806910F4407F5E
:1065100003D02046FFF7B4FF05E0204600F07AF8EC
:10652000204600F0F5F8002020772807B7D520682E
:106530006FF00801016104212177C069800703D051
:106540002046FFF79DFF05E0204600F063F8204657
:1065500000F0DEF800202077E806A2D520686FF072
:106560001001016108212177C06910F4407F03D038
:106570002046FFF785FF05E0204600F04BF8204657
:1065800000F0C6F800202077E8073FF48CAF2068C1
:106590006FF001010161204600F04EF928067FF5F9
:1065A00084AF20686FF0800101612046FFF712FF81
:1065B00068067FF583AF7AE780B586B044F2004184
:1065C0000068C4F20101002288420592CDE903224D
:1065D0000292019201D006B080BD43F630000092D5
:1065E000C4F20200036843F020030360006800F077
:1065F000200000900098402001900220CDE9020286
:106600000320059001F5504001A90492FEF72AFCF1
:1066100006B080BD70470000B0B5044690F83C005D
:10662000012804BF0220B0BD0D464FEAB20101208F
:10663000032984F83C0037D8DFE801F0020A12226F
:106640002068294602F0B4FF206850F8181F0EE0B9
:106650002068294602F0DEFF206850F8181F16E077
:106660002068294603F00CF8206850F81C1F41F000
:1066700008010160016821F00401016029690FE04F
:106680002068294603F030F8206850F81C1F41F4B8
:1066900000610160016821F48061016029690902DB
:1066A0000268114301600020002184F83C10B0BD55
:1066B000002804BF0120704710B5044690F83D0043
:1066C00028B9002084F83C00204600F01FF8022082
:1066D00084F83D002068211D02F0C2FE012084F8EC
:1066E000460084F83E0084F83F0084F8400084F8B7
:1066F000410084F8420084F8430084F8440084F8A0
:10670000450084F83D00002010BD000070470000E7
:106710007047000010B5044641B1082909D004298A
:1067200014BF04F1410004F13F0004E004F13E0015
:1067300001E004F14000007801281CBF012010BDD9
:10674000022041B1082909D0042914BF84F841006E
:1067500084F83F0004E084F83E0001E084F8400043
:106760002068012202F012FF206841F2FF71C4F29A
:10677000000188420FDC40F2FF71C4F20001884240
:1067800017DCB0F1804F49D040F20041C4F2000163
:10679000884243D049E040F2FF32C4F20102904205
:1067A00014DC41F60003C4F20003984236D0002303
:1067B00014E040F60001C4F2000188422ED040F6F9
:1067C0000041C4F20001884228D02EE044F20003C8
:1067D000C4F20103984221D040F20043C4F2010305
:1067E000984222D1436C884243F400434364C2DDA3
:1067F000904207DC41F60001C4F2000188420DD04E
:10680000002107E044F20001C4F20101884205D0F2
:1068100040F20041C4F20101884206D1816801F0D2
:106820000701062904BF002010BD016841F00101E5
:106830000160002010BD000070470000704700009C
:106840007047000080B503F0B1FB052808BF80BD8C
:1068500040F25C1100EBC000C2F2000101EB8000CD
:106860000069002818BF804780BD0000B0B582B025
:10687000036804461868D9685A6900F02F05202D6E
:1068800001F0200505D125B1204603F0B9FB02B087
:10689000B0BD5FEA007C1EBF02F0010E01F49072F1
:1068A00012EB0E024AD1226B0840C1063DD5012AE7
:1068B0003BD1002001901868019058680190019820
:1068C0005869400642D4A08DE18DE28D002A1CBF9C
:1068D000401A5FEA004101D102B0B0BD216851E821
:1068E000031F226821F4907142E80313002BF5D1B5
:1068F000216851E8051F226821F0010142E80513D3
:10690000002BF5D1202184F842100021216300BF23
:10691000216851E8031F226821F0100142E80313A7
:10692000002BF5D10221616354E0010654D44006E6
:10693000D2D5204603F020FB02B0B0BDC20718BF7D
:1069400011F480725DD1420761D467E0E06B0168A9
:1069500049688AB2002A44D0A38D9A4241D2E18587
:10696000C069B0F5807F30D0206850E8030F2168FF
:1069700020F4807041E80302002AF5D1206850E835
:10698000050F216820F0010041E80502002AF5D139
:10699000206850E8050F216820F0400041E805021A
:1069A000002AF5D1202084F842000020206300BF97
:1069B000206850E8030F216820F0100041E803022E
:1069C000002AF5D1E06BFEF763F802206063A08D2A
:1069D000E18D401A81B20FE0204603F039FC02B08D
:1069E000B0BDA18D91427FF477AFC069B0F5807FD3
:1069F0007FF472AF022060632046FFF721FF02B0F0
:106A0000B0BD626C42F001026264420706D5BEF17D
:106A1000000F03D0626C42F002026264820706D566
:106A2000BEF1000F03D0626C42F004026264BCF15C
:106A3000000F06D55EEA050203D0626C42F0080240
:106A40006264626C002A3FF447AF0840800602D5BA
:106A5000204603F0D5FA20684069616C00F04000E0
:106A600001F00801401827D0204603F05DFA2068A5
:106A7000406940061BD500BF206850E8050F21681B
:106A800020F0400041E80502002AF5D1E06B70B12A
:106A900049F62961C0F600010165FEF739F80028C2
:106AA0003FF41AAFE06B016D884702B0B0BD2046DD
:106AB000FFF7C8FE02B0B0BD2046FFF7C3FE0020BE
:106AC000606402B0B0BD0000002804BF0120704720
:106AD00010B5044690F8410028B9002084F8400021
:106AE000204600F021F8242084F841002068C16885
:106AF00021F40051C160204603F0E6FA20680169E4
:106B000021F490410161416921F02A014161C1688C
:106B100041F40051C16000202021606484F84110DC
:106B200084F84210606310BD2DE9F04387B004463D
:106B3000006840F6FF71C4F2010188424FF0000185
:106B40000691CDE90411CDE9021163DC44F2004164
:106B5000C4F20001884200F0AC8044F60001C4F2A7
:106B60000001884240F04181002643F63000019642
:106B7000C4F20200016941F480210161016901F45C
:106B80008021019101990196016841F004010160A1
:106B9000006802A900F00400019001984FF44060E1
:106BA00002900220CDE903060320059007200690FD
:106BB0000020C4F2020000F50060FEF753F940F235
:106BC000187546F22800C2F20005C4F202004FF028
:106BD00000614FF480624FF4807385E843002846DB
:106BE000C5E90362C5E90566C5E907366E62FEF7C9
:106BF00067F8002818BFFCF7F3FD272005210022C5
:106C0000E563AC63FEF7C4FB2720FEF7BDFB07B0CE
:106C1000BDE8F08341F20041C4F20101884275D021
:106C200041F20001C4F20101884240F0DE800026FA
:106C300043F630000196C4F202004169002441F09D
:106C4000100141614169C4F2020401F01001019197
:106C500001990196016802AD41F0020101600168ED
:106C60004FF0020801F002010191019901960168BB
:106C70004FF0030941F0010101600068072700F0AF
:106C80000100019001988020029004F5806029465F
:106C9000CDE90386CDF814900697FEF7E3F84FF49C
:106CA0000070CDE90208CDE904690697204629461F
:106CB00027E0002043F630010190C4F202010A6986
:106CC00042F400320A610A6902F400320192019A28
:106CD00001900A6842F008020A60096801F00801A0
:106CE00001910199602102910221CDE90310032055
:106CF0000590072006900020C4F2020000F54060D5
:106D000002A9FEF7AFF807B0BDE8F083002643F60E
:106D100030000196C4F20200416946F2280841F0B1
:106D2000200141614169C4F2020801F02001019192
:106D300001990196016841F040010160006802A9D3
:106D400000F04000019001984FF48440029002202E
:106D5000CDE9030603200590082006900020C4F228
:106D6000020000F5C050FEF77DF84CF6D84508F556
:106D70008060C2F201054FF020674FF48069C5E9D9
:106D800000072846C5E90266C5E90496C5E9066616
:106D9000C5E90866FDF794FF002818BFFCF720FD41
:106DA000E563AC6340F2787508F58F60C2F20005C8
:106DB0004021C5E9000705F1080080E842022846A5
:106DC000C5E90566C5E907666E62FDF779FF00282B
:106DD00018BFFCF705FD472005210022A563AC6321
:106DE000FEF7D6FA4720FEF7CFFA07B0BDE8F083EA
:106DF00080B590F84230202B1CBF022080BD0029B6
:106E00004FF0010318BF002A01D1184680BD0023AE
:106E1000036303F0C7F90346184680BD80B503F04D
:106E2000C5F8052808BF80BD40F25C1100EBC0002A
:106E3000C2F2000101EB8000C068002818BF804743
:106E400080BD000080B503F0B1F8052808BF80BD03
:106E500040F25C1100EBC000C2F2000101EB8000C7
:106E60008068002818BF804780BD000080B503F00F
:106E70009DF8052808BF80BD40F25C1100EBC00002
:106E8000C2F2000101EB80004068002818BF804773
:106E900080BD0000FEE7000045F6DF1110EE100A8D
:106EA000C5F63771B6EE001AA1EB600020EE011AAC
:106EB00000EE100A21EE002A22EE002AB7EE083A70
:106EC00033EE422A22EE000A21EE001A20EE011AC9
:106ED00033EE411A20EE010A7047000040F26111C2
:106EE000884204BF01207047B0F5806F04BF0320C3
:106EF0007047A0F29F60B0FA80F0400940007047F0
:106F000010B52DED088B88B3B0EE408A90ED010AE4
:106F100090ED069A90ED021A90ED07AA29EE000A6C
:106F200038EE400A2AEE011A30EE41BA04461BEE52
:106F3000100A03F0E1F9002808BFB0EE4B8A94ED87
:106F4000030A94ED041A94ED052A20EE080A29EEAE
:106F5000011A30EE010A2AEE021A30EE010A84ED1F
:106F6000068A84ED079ABDEC088B10BD9FED020ADE
:106F7000BDEC088B10BD00BF00000000002808BF5A
:106F8000704710B5F5EE400A0446C0ED000A002037
:106F9000F1EE10FAA061E0612EDD80EE200A9FED97
:106FA0001E1A81EE000A06F0A3FF9FED1C1AB7EE31
:106FB000002A20EE011A31EE023A20EE000ABFEE5E
:106FC000005A30EE033A30EE055A32EE411A80EEA6
:106FD000034A35EE055A30EE010A85EE035A80EE7B
:106FE000030A34EE041A84ED034A84ED041A84ED96
:106FF000054A84ED015A07E04FF07E519FED050AE6
:10700000C4E903106061606084ED020ABDE81040CD
:10701000704700BF00000000DB0F4940F304B53F9C
:1070200010B52DED048B10B3B0EE408A90ED030A3D
:1070300090ED041A90ED052A30EE010A30EE020AB6
:1070400088EE009A044619EE100A03F045F900286C
:107050002046B0EE480A08BFB0EE489A84ED069A82
:1070600084ED079AFFF74CFFBDEC048B10BD9FED3C
:10707000020ABDEC048B10BD00000000B0B5012871
:1070800002D9FF2040B2B0BD40F22025C2F2000577
:10709000044655F8200060B98820FAF777FF0028E9
:1070A00045F82400EDD08821F9F7ABFA55F8240013
:1070B0000470002040B2B0BD80B584B0D8B100F0FB
:1070C00029F8014600284FF0FC0015D08A888DF879
:1070D0000C00009208228DF804204FF0FF32CDF80A
:1070E0000520029208786946FAF7E4FD002818BFE7
:1070F0004FF0FF3000E0FE2040B204B080BD000041
:1071000001288FBF002040F22021C2F2000151F877
:10711000200070472DE9F04128B3057880462846C5
:10712000FFF7EEFFF8B1014690F88400D8B10A1DD0
:10713000002309E00126002E08BFBDE8F08191F888
:1071400084600133B3420ED252F82340002CF1D0B8
:107150002678AE42EED16688B8F80270BE42E9D118
:1071600000262046E7E70020BDE8F08110B50C4678
:10717000014600284FF0FE0018BF002C01D140B29C
:1071800010BD0846FFF7C6FF20B1214600F0D4F835
:1071900040B210BDFC2040B210BD0000B0B52DEDD6
:1071A000028B00286BD00D46002968D00446B5F844
:1071B00001009FED340A0004DFED330A00BA10210C
:1071C00004F08CFB84ED070AE8782979000140EA95
:1071D0001110BBEE0E0AF3EE0E0A0C2104F07EFB3A
:1071E00084ED080A2879697900F00F00B0EE408A32
:1071F00041EA0020BAEE080AF2EE080A0C2104F077
:107200006DFB84ED090AA87994ED071A02EE100AC5
:10721000B5EE401AB8EE422AF1EE10FA84ED0A2AD1
:107220000BDA9FED1A2A00BF31EE021AB5EE401AB2
:10723000F1EE10FAF8DB84ED071A94ED071A9FEDD2
:10724000132AB4EE421AF1EE10FA0ADB9FED103A5F
:1072500031EE031AB4EE421AF1EE10FAF8DA84EDC8
:10726000071AE07958B132EE411AB1EE482AB1EE70
:10727000400A84ED071A84ED082A84ED090ABDEC62
:10728000028BB0BDDA0F49C1DA0F4941DB0FC940AB
:10729000DB0FC9C070B538B104460078FFF7EEFEC9
:1072A00028B1FF2040B270BDFE2040B270BD2078F2
:1072B000FFF726FF0028F4D090F8842005469AB105
:1072C000281D002105E000BF95F88420013191427E
:1072D0000AD250F82120002AF6D0528863889A42B8
:1072E000F2D1FD2040B270BD1F2ADAD83020FAF763
:1072F0004DFE0028D5D030210646F9F782F92068E6
:107300006168C6E900010020E27930722078618866
:1073100032760322FAF788FB18B13046FAF7AAFD55
:10732000BFE795F8840005EB8001013085F8840003
:10733000002040B24E6070BD2DE9F04381B02DEDCC
:10734000048B84B0044600284FF0FE0071D00D4637
:1073500000296ED095ED001A95ED012A95ED023ABF
:10736000E079B1EE430AB1EE428AB1EE419A0028CB
:1073700002BFB0EE430AB0EE428AB0EE419ADFEDB2
:10738000300A9FED301A102003F046F98046FBEEDC
:107390000E0AB3EE0E1AB0EE480A0C2003F03CF9C8
:1073A0009FED298A95ED030A9FED281A0746F0EE16
:1073B000480A0C2003F030F995ED040A8146B1EE3D
:1073C000041AF0EE480A0C2003F026F90646FAEEFD
:1073D000080AB2EE081AB0EE490A0C2003F01CF9B4
:1073E0003A094FEA1923A5888DF8072022784FEA39
:1073F000182143EA0713070A47EA061736090095DA
:1074000008258DF805108DF80C00694610468DF89A
:1074100004508DF806808DF808308DF809908DF8AD
:107420000A608DF80B70FAF745FC002818BF4FF082
:10743000FF3040B204B0BDEC048B01B0BDE8F08376
:10744000DA0F49C1DA0F4941000000000000FA4399
:10745000F0B587B0A0B3077805463846FFF750FE71
:10746000A8B390F8841069B3011D002205E000BFA5
:1074700090F8843001329A4224D251F82240002CF4
:10748000F6D063886E88B342F2D1F4B169886D4654
:1074900038462A460023FAF7C1F9D0B1FAF732FE8E
:1074A000D4E90423801A48F2A162C0F20102994192
:1074B000801A71F1000024BF00202072FF2014E028
:1074C000FE2012E00024002CE0D1FC200DE0FC2086
:1074D0000BE001202072FAF715FEC4E9040105F162
:1074E0000D012046FFF75AFE002040B207B0F0BD64
:1074F000B0B5012802D9FF2040B2B0BD4CF2FC4526
:10750000C2F20105044655F8200060B94820FAF798
:107510003DFD002845F82400EDD04821F9F771F829
:1075200055F824000470002040B2B0BDB0B584B05E
:1075300048B304780546204600F064F828B369880B
:10754000A1F201210A295BD8012202FA01F10A07FE
:107550001DD111F0F00F30D040F2FF110091082141
:107560008DF804100A3000216A4600BF00EB410389
:107570005B7802EB41056B7110F811300131042981
:10758000AB71F3D131E0FE2037E0FC2035E04FF461
:107590000071009108218DF80410023000216A4624
:1075A00000EB41035B7802EB41056B7110F8113081
:1075B00001310429AB71F3D117E040F2FF210091B2
:1075C00008218DF80410123000216A4600EB4103B7
:1075D0005B7802EB41056B7110F811300131032922
:1075E000AB71F3D10020ADF80B0069462046FAF7E5
:1075F00061FB002818BF4FF0FF3040B204B0B0BDAF
:10760000FF20FAE701288FBF00204CF2FC41C2F2B4
:10761000010151F82000704748B102280BD0012821
:1076200014BF4FF6FF704FF4804000B2704742F233
:10763000107000B2704747F2305000B2704700003F
:10764000022905D2A0F2012189B2072909D805E053
:1076500007D1A0F2052189B2062902D8013840B22B
:107660007047FF2040B27047F0B581B008B30746BD
:107670000078FFF7C7FFE0B1014690F84400C0B1C1
:1076800001F11802002306E0012585B191F844506C
:107690000133AB420DD252F82340002CF4D0658860
:1076A0007E88B542F0D100252046002DEED101B0F4
:1076B000F0BD002001B0F0BD022884BFB7EE000A83
:1076C000704740B202A101EB800090ED000A7047C4
:1076D000000010422CA099410000803F70B538B1E5
:1076E00004460078FFF704FF28B1FF2040B270BDC8
:1076F000FE2040B270BD2078FFF784FF0028F4D050
:1077000090F8442005469AB105F11800002104E0E4
:1077100095F84420013191420AD250F82120002AE4
:10772000F6D0528863889A42F2D1FD2040B270BDF3
:107730000A2ADAD85020FAF729FC0028D5D00646C4
:1077400020686168C6E9000106F118002821F8F7F1
:1077500058FF62792078618886F828200322FAF79A
:1077600063F918B13046FAF785FBBEE795F8440097
:1077700005EB8001013085F84400002040B28E61A5
:1077800070BD000080B59FED020A00F003F880BDD7
:107790000000000070B52DED048B00283ED005469A
:1077A0000078B0EE408AFFF72DFFC8B3B7EE000AAD
:1077B000B4EE408AF1EE10FAC8BFB0EE408ABFEED8
:1077C000000AB4EE408A0446F1EE10FAB8BFB0EEFB
:1077D000408A6879B1EE489A0028284608BFB0EE82
:1077E000489AFFF741FFE8B12E7968883146FFF7E4
:1077F00027FF002818D405463046FFF70DFF00EE9E
:10780000100AB8EEC00A29EE000ABDEEC00A10EE5A
:10781000100A04EB45014880002006E0FE2004E049
:10782000FC2002E0FC2000E0FF2040B2BDEC048B15
:1078300070BD00002DE9F04F87B0002852D00446FB
:107840000078FFF7DFFE00284ED0054690F8440090
:1078500000284BD005F11806E8464FF0010A40F227
:10786000E93B4FF0000908E00121002941D095F8DB
:10787000441009F1010989453AD256F82970002FC0
:10788000F2D07A8861888A42EED12078424600237D
:10789000F9F7C4FF70B1FAF735FCD7E90823801A6D
:1078A0009941B0EB0B0071F1000016D3002038763F
:1078B000FC2013E087F818A0FAF724FCC7E90801B8
:1078C0003846414600F0CAFA07F108030FCB07F12A
:1078D0002C0C8CE80F00002000E0FF200021002984
:1078E000C5D106E0FE2004E0FC2002E0FC2000E020
:1078F000FC2040B207B0BDE8F08F000010B54CF698
:10790000284046F20041C2F20100C4F20001032205
:1079100000234FF0807480E80E0000F10C014FF45A
:10792000102C4FF4001E81E8085084618383FCF71B
:1079300089FE002818BFFBF753FF10BD10B54CF6A9
:10794000504046F60001C2F20100C4F200010322D9
:1079500000234FF0807480E80E0000F10C014FF41A
:10796000102C4FF4001E81E8085084618383FCF7DB
:1079700069FE002818BFFBF733FF10BD80B582B049
:10798000002043F630010190C4F202010A6842F47B
:1079900000120A600A6802F400120192019A009033
:1079A0000868002240F4800008600868052100F49F
:1079B0008000009000980C20FDF7EAFC0C20FDF7F9
:1079C000E3FC392005210022FDF7E2FC3920FDF718
:1079D000DBFC3A2005210022FDF7DAFC3A20FDF716
:1079E000D3FC3B2005210022FDF7D2FC3B20FDF714
:1079F000CBFC452005210022FDF7CAFC4520FDF700
:107A0000C3FC02B080BD000080B549F249304FF29E
:107A1000F832C0F60000C0F60002002103F050F971
:107A20004CF68031C2F20101086049F2B9704FF2A0
:107A30007C32C0F60000C0F60002002103F040F9DD
:107A400080BD00002DE9F04F87B04FF0000A43F6EB
:107A50003000CDF818A0CDE904AACDE902AACDF8EE
:107A600004A0C4F20200016840F2004841F00201A3
:107A700001600168C4F2020801F00201019101995C
:107A8000CDF804A0016808F5A05441F04001016060
:107A90000168002201F0400101910199CDF804A094
:107AA0000168402641F001010160016801F0010117
:107AB00001910199CDF804A0016841F0080101602D
:107AC000016801F0080101910199CDF804A0016855
:107AD00041F004010160016801F004010191019984
:107AE000CDF804A0016841F020010160016801F0B7
:107AF000200101910199CDF804A0016841F08001B5
:107B000001600068402100F080000190019820464B
:107B1000FDF77CFA08F58069484602210022FDF74E
:107B200075FAA8F580673846102101220125FDF776
:107B30006DFA404602210022FDF768FA4046012115
:107B40000122FDF763FACDE9026502AE2046314617
:107B5000CDE90455FDF786F9082002904FF4041B87
:107B600020463146CDE903B5FDF77CF902244846AD
:107B70003146CDE90245CDE9045AFDF773F938469F
:107B80003146CDE9025B0495FDF76CF91020CDE993
:107B9000020538463146CDE90455FDF763F930203A
:107BA000CDE9020B484631460495FDF75BF94046A6
:107BB0003146CDE90245CDE9045AFDF753F9404677
:107BC0003146CDE90255CDE90455FDF74BF90620C4
:107BD00005210022FDF7DCFB0620FDF7D5FB09207F
:107BE00005210022FDF7D4FB0920FDF7CDFB0A207B
:107BF00005210022FDF7CCFB0A20FDF7C5FB17206D
:107C000005210022FDF7C4FB1720FDF7BDFB07B0DF
:107C1000BDE8F08F80B540F2D87045F20041C2F265
:107C20000000C4F2000148F2A06200234FF4804C2F
:107C3000C0F2010280E80E00C0E9033CC0E9053350
:107C4000C0E90733FDF7EEF9002818BFFBF7C8FDC0
:107C500080BD000080B54CF6385045F60001C2F2F8
:107C60000100C4F2000148F2A06200234FF4804CEE
:107C7000C0F2010280E80E00C0E9033CC0E9053310
:107C8000C0E90733FDF7CEF9002818BFFBF7A8FDC0
:107C900080BD0000B0B540F62C0043F20001C2F2F6
:107CA0000000C4F201014FF48272002380E80E004C
:107CB00000F10C014FF0020C4FF0010E4FF4007474
:107CC000182581E808500A21C0E90645C0E90833B3
:107CD000C0E90A31FDF734FE002818BFFBF780FD2C
:107CE000B0BD000080B588B04CF68C5044F2004224
:107CF0000021C2F20100C4F2010241F2883307916F
:107D0000CDE90511CDE90311CDE90111C0E900214B
:107D1000C0E9021301618161FEF760FB002818BF12
:107D2000FBF75EFD4CF68C50C2F20100FEF7C0FC82
:107D3000002818BFFBF754FD602001900020CDE91A
:107D4000020005904CF68C50C2F2010001A90022FD
:107D5000FEF762FC002818BFFBF742FD4CF68C5082
:107D6000C2F20100FEF728FC08B080BD80B54CF6D9
:107D7000D45041F20001C2F20100C4F2010100231B
:107D80004FF00C0C4FF4E13280E80E00C0E90333F1
:107D9000C0E905C3C361FEF797FE002818BFFBF7D3
:107DA0001FFD80BD80B540F6840044F20041C2F260
:107DB0000000C4F2000100234FF00C0C4FF4E1323C
:107DC00080E80E00C0E90333C0E905C3C361FEF7D4
:107DD0007BFE002818BFFBF703FD80BD10B54CF6F5
:107DE0001C6044F6000C48F2A062C2F20100C4F22A
:107DF000000CC0F201024FF4805300214FF4806E5A
:107E00000424C0E900C2C0E90231C0E904E4C0E9C9
:107E10000611FEF759FE002818BFFBF7E1FC10BD64
:107E200080B540F6CC0041F20041C2F20000C4F23D
:107E3000010100234FF00C0C4FF4E13280E80E00FA
:107E4000C0E90333C0E905C3C361FEF73DFE002866
:107E500018BFFBF7C5FC80BDFEE700002DE9F04729
:107E60008846B1F80D10044608BA4FEA1049B8F830
:107E700011002679B8F80F1005BA304691FAB1FA18
:107E8000FFF7CAFB07463046FFF716FC01EE109AD3
:107E90009FED453AB8EE412A9FED441A22EE032A9F
:107EA00022EE014A02EE10AA15FB27F0B8EEC23A04
:107EB00002EE100AA0799FED3E5AB8EEC22A22EED9
:107EC000052A48B1B4F84000A9EB0000B0F5805F86
:107ED0000CDD4FF0FF300DE00020A4F84090C4E925
:107EE000110084ED024A84ED033A1CE010F5805F36
:107EF00003DA0120616C0844606494ED115A83EE4A
:107F0000003AB8EEC55A25EE015A34EE054A84EE21
:107F1000004AA4F8409020EE022A84ED033A84ED52
:107F2000124A84ED024A94ED020A84ED042AB5EE69
:107F3000400AF1EE10FA08DA30EE010AB5EE400A16
:107F4000F1EE10FAF8DB84ED020A94ED020AB4EEC9
:107F5000410AF1EE10FA0ADB9FED162A30EE020A12
:107F6000B4EE410AF1EE10FAF8DA84ED020A94F860
:107F7000280078B131EE400A84ED020A94ED030A3C
:107F800094ED041AB1EE400A84ED030AB1EE410A01
:107F900084ED040A98F8130000EE100AB8EE400AC7
:107FA00084ED050ABDE8F08700000039DB0FC94009
:107FB00000008038DB0FC9C0FEE7000000F00700BA
:107FC00080F00703042B28BF04234FF0FF3C033845
:107FD0000CFA03F338BF0020994381400CFA00F0FB
:107FE00022EA000008437047B0B52DED0A8B044625
:107FF00010EE100AB0EE618AB0EE419AB0EE60AABF
:10800000B0EE40BA02F070F9002800F09C801AEE41
:10801000100A02F069F9002800F0958019EE100AA4
:1080200002F062F9002800F08E8018EE100A02F0CB
:108030005BF9002800F087806068B0EE4B0A90ED95
:10804000071AF0EE4A0AFBF729F96068B0EE40BA69
:1080500090ED001A04F11C0020EE01CA21EE0A0A7C
:10806000FEF74EFF207888B1012811D194ED051A52
:1080700094ED022A30EE411AB4EE428AF1EE10FA83
:10808000C8BFB0EE482A81EE029A01E09FED309A17
:1080900019EE100A84ED04BA84ED050A02F024F901
:1080A00065689FED2B0A002808BFB0EE409A95ED59
:1080B000010A95ED032A2CEE000A29EE022A95ED1D
:1080C000021A30EE42AA94ED030A9FED229A2CEE9A
:1080D000082A32EE008AB4EE491AF1EE10FA28EEC0
:1080E00001BA1ADD18EE100A02F0FEF8A8B13AEE55
:1080F0000B0A95ED051AB0EEC00AB4EE410AF1EE96
:1081000010FA0ADC95ED040AB0EEC81AB4EE401A73
:10811000F1EE10FAD8BF84ED038A3AEE0B8A18EE1E
:10812000100A02F0E1F870B1D5ED050AF4EE490A43
:10813000F1EE10FA05DDB0EE480AF9F7BBF8B0EE43
:10814000408A84ED068A94ED060ABDEC0A8BB0BD28
:1081500000000000BD37863570B52DED048B90B35F
:10816000044650681646B0EE408A0D4602F0BCF850
:1081700058B3B06802F0B8F848B3F06802F0B4F849
:1081800038B3306902F0B0F828B3706902F0ACF887
:1081900018B3B7EE000A80EE089A666019EE100A6E
:1081A00002F0A2F8D8B1D6ED060A04F11C00B0EE38
:1081B000480A84ED029AFEF7E1FE2046257000F0A1
:1081C00013F800200CE0FF200AE0FF2008E0FF2069
:1081D00006E0FF2004E0FF2002E0FF2000E0FF2097
:1081E00040B2BDEC048B70BD10B568B100F11C014C
:1081F00000249FED070AC0E90344C0E9054408468E
:10820000FEF70EFF60B210BDFF2460B210BD00BFCC
:108210000000000000280EBFFF210021C16048B20D
:108220007047000000000000000000000000000097
:10823000EFF30980BFF36F8F154B1A681EF0100F14
:1082400008BF20ED108A20E9F04F10602DE90900E9
:108250004FF0500080F31188BFF34F8FBFF36F8F43
:1082600003F0AAFE4FF0000080F31188BDE809007A
:1082700019680868B0E8F04F1EF0100F08BFB0ECA6
:10828000108A80F30988BFF36F8F704700BF00BF6B
:10829000A809002080B502F00FFD40F6E811C2F2F7
:1082A00000010860A8B148F2D922C0F600020220FD
:1082B0000321F9F77DFF40F22821C2F200010020DE
:1082C000C1E90000C1E90200C1E90400087640B23A
:1082D00080BDFE2040B280BD80B540F6E810C2F2FD
:1082E00000000068012102F049FC80BD80B5022039
:1082F000F9F730FF40F22821C2F200011922FEF7FF
:1083000077FD002818BF4FF0FF3080BD80B50246D2
:108310000120012102F072FC0138B0FA80F040091E
:1083200080BD000080B5806B01684A6822F00302BE
:108330004A60416D41F010014165012180F8511002
:10834000FDF7ECFA80BD000080B5806BFDF72CFDD9
:1083500080BD000080B5806BFEF702F880BD000094
:1083600080B5806BFEF720F880BD0000B0B5846B4F
:108370000546FCF751FE29680968C90526D402465E
:108380002068A168436823F02003436031B9616825
:10839000B1F5827F02D16FF0030101E06FF00101BE
:1083A0004368194041602046642100F079F80028B4
:1083B0001CBF202060650020E087012084F8510068
:1083C000606D18B12046FDF7A9FAB0BD2046FDF753
:1083D000D9FCB0BDB0B582B0846B0546FCF71CFE7D
:1083E00029680968C90528D402462068416821F037
:1083F00020014160416821F0020141602046642172
:1084000000F096F818B1606D40F020006065A0683B
:1084100038B9002001902068C168019180680190FE
:1084200001980020E086012084F85100606D20B1A1
:108430002046FDF773FA02B0B0BD2046FDF780FF7D
:1084400002B0B0BDB0B5846B0546FCF7E5FD296808
:108450000968C9051FD402462068416821F020013F
:1084600041602046642100F063F818B1606D40F06F
:10847000200060652068416821F003014160002010
:10848000E086E087012084F85100606D18B1204635
:10849000FDF744FAB0BD2046FDF774FFB0BD000003
:1084A000B0B582B0044640680B46B0F5827F20D15B
:1084B000A168B1F5004F02D0B1F5806F04D12168F9
:1084C0000D6825F040050D60B0F5827F11D1A068E0
:1084D000B0F5806F1DD100922046012100220025B9
:1084E00000F076F890B1606D032540F020006065E3
:1084F0000CE00092204601210022002500F068F8DF
:1085000020B1606D032540F020006065284602B070
:10851000B0BD0092204680210022002500F058F8CE
:108520000028F3D0606D032540F020006065EDE782
:1085300070B582B00D461646022101222B46044634
:10854000009600F045F838B1606D032540F020003A
:108550006065284602B070BD4CF20000C2F2010016
:10856000006849F68171C1F25E61A0FB0101480D0E
:108570004FF47A71484301906068B0F5827F0FD163
:108580002046802100222B460096002500F020F88E
:108590000028DED0606D032540F020006065D8E73C
:1085A000019840B101980138019020688068000668
:1085B000F6D40025CDE70025CBE70000006843F2A4
:1085C0000001C4F20101401A18BF012040007047A9
:1085D0002DE9F04782B00A9C984615460E46814622
:1085E000FCF71AFD201A00EB0804FCF715FD4CF20D
:1085F0000001C2F201010968C1F3CB31614301916D
:10860000D9F8001089683140891BB1FA81F1490914
:10861000A94203D1002002B0BDE8F087824608F1EC
:1086200001070CE0019801380190D9F8000080683A
:108630003040801BB0FA80F04009A842EAD0002FF9
:10864000F3D0FCF7E9FCA0EB0A00A04204D20198A9
:108650000028E7D10024E8E7D9E900014268B1F534
:10866000827F22F0E00242600BD1D9F80810B1F508
:10867000004F02D0B1F5806F03D1016821F04001B5
:108680000160D9F82810B1F5005F07D1016821F425
:1086900000510160016841F400510160012089F836
:1086A0005100002089F85000032002B0BDE8F08797
:1086B000074B19680868B0E8F04F80F30988BFF3EA
:1086C0006F8F4FF0000080F31188704700BF00BF2C
:1086D000A809002080B501F055FE80BD90ED000A8C
:1086E00091ED001AB7EE002A30EE011AB4EE421AEC
:1086F000F1EE10FAD8BF704782EE011A20EE010A9F
:1087000080ED000A91ED000A21EE000A81ED000AD9
:1087100070470000002804BFBFEE000A704782695E
:10872000137823B1012B2AD19FED181A01E09FED98
:10873000151A02EB810292ED020A90ED672A00EB16
:10874000011191ED093A20EE020A30EE430A20EEC3
:10875000002A21EE013A82EE032AB0EEC03AB7EECB
:10876000000AB4EE413AF1EE10FA30EE422A9FEDE3
:10877000060AB8BFB0EE420A80ED460A70479FED88
:10878000020A704700004842000000000000C84391
:10879000B0B52DED048B10B30446B0F8200100B342
:1087A00094ED001A94ED472A9FED208AD4ED490AF2
:1087B00094ED680A31EE429AB0EE481A0D46FAF787
:1087C0006DFDA169B7EE001A91ED062A81EE022A2D
:1087D000B4EE429AF1EE10FA05DA002021E0FF2013
:1087E0001FE0FF201DE0B4EE410AF1EE10FA4FF059
:1087F000000016DCAA78A2B12068F0EE480AC4F89E
:108800001C0191ED050A04F5D070B8EE400A88EE1F
:10881000000AFAF725FDB4F820010138A4F8200178
:10882000002040B2BDEC048BB0BD00BFDB0FC940DF
:1088300048B181690978012908D061B942F2000183
:10884000C4F2CB5105E0FF2040B270470021C4F2D2
:108850007A51C0F89C11002040B27047B0B52DEDA0
:10886000028B054600284FF0FF0027D00C4629B3A5
:10887000F9F748FC06F0E9FB9FED128A00EE100ABA
:1088800080EE080A85ED000AF9F73CFCD5E90223E1
:10889000801A994106F0D9FB00EE100A80EE080A12
:1088A00085ED040AF9F72EFCC5E902012846FFF719
:1088B000BFFF2846214600F0ABF8002040B2BDECD7
:1088C000028BB0BD002474492DE9F04F81B02DED2D
:1088D000028B834600284FF0FF0000F0928088460C
:1088E000002900F08E80B5EE400AB0EE408AF1EE2D
:1088F00010FA40F3868098F80440CBF81880F8F717
:10890000CDFFB4B308F1700908F1900A08F12C0505
:108910000BF5D2760BF2EC472846FEF7DFFE304629
:108920000121B0EE480A4A46FFF716FC06F5B4707E
:108930000121B0EE480A5246FFF70EFCDBF81800A2
:10894000B0EE480AD0ED4C0A3846FEF717FBDBF8CC
:108950001800B0EE480AD0ED4D0A07F1C000FEF74E
:108960000DFB013C05F10A0506F13C0607F1200765
:10897000D2D108F16800FEF7B1FEDBF8180090F8DC
:108980006C0078B101283BD10BF2744008F1F00281
:108990000121B0EE480AFFF7DFFB0BF5966008F502
:1089A00088720CE00BF2744008F1B0020121B0EEC5
:1089B000480AFFF7D1FB0BF5966008F1D0020121C0
:1089C000B0EE480AFFF7C8FBDBF81800B0EE480A23
:1089D000D0ED4E0A0BF26C60FEF7D0FADBF818000F
:1089E000B0EE480AD0ED4F0A0BF28C60FEF7C6FAE3
:1089F0000020CBE94700CBE94900CBF82C0100E08F
:108A0000FC2040B2BDEC028B01B0BDE8F08F00004D
:108A1000B0B500B30446806990F82020F2B194F814
:108A2000DC20032A67D8DFE802F00259233A94EDEC
:108A3000240A9FED421A80EE010A90ED091AB4EE65
:108A4000410AF1EE10FA68DD2268012084F8DC00AA
:108A5000C4F8D82061E0FF2568B2B0BD00252046EB
:108A600084F8DC5084F8D45000F0F4F868B2B0BD5B
:108A700090ED050A9FED2F1AB8EE400A81EE000A2C
:108A800094ED491A00202268A4F82001032084F8FC
:108A9000DC00C4F8D82031EE000A84ED680A2046D4
:108AA00000F0D8F894ED000A94ED361A9FED222AD2
:108AB00030EE410AB4EE420AF1EE10FA30DB94EDEA
:108AC000240A9FED1E1A002580EE010AB3EE041A57
:108AD000B4EE410AF1EE10FAC8DA0DE094ED240A82
:108AE0009FED161A80EE010A90ED091AB4EE410AC4
:108AF000F1EE10FA04DA002568B284F8DC50B0BD5B
:108B000094ED000A94ED361A90ED0A2A30EE410AEF
:108B1000B4EE420AF1EE10FA05DA204600F09AF8B7
:108B2000002568B2B0BD012084F8D400022084F88A
:108B3000DC00F5E7DB0FC9C09A99993E00007A4442
:108B4000002843D0F0B581B02DED028B044680693A
:108B50000779EFB19FED1F8A04F5D27504F2EC4658
:108B60002846FFF741FB05F5B470FFF73DFB3046A3
:108B7000B0EE480AFEF754FA06F1C000B0EE480A1B
:108B8000FEF74EFA013F05F13C0506F12006E7D15C
:108B900004F27440FFF728FB04F59660FFF724FB0E
:108BA0009FED0C8A04F26C60B0EE480AFEF738FACA
:108BB00004F28C60B0EE480AFEF732FA0020BDECF9
:108BC000028B01B0BDE8F04040B27047FF2040B2D8
:108BD000704700BF00000000F0B170B50446806926
:108BE000067966B104F5D2752846FFF713FB05F543
:108BF000B470FFF70FFB013E05F13C05F4D104F220
:108C00007440FFF707FB04F59660FFF703FB0020B5
:108C1000BDE8704040B27047FF2040B2704700008E
:108C2000A0B18169097951B100F59672002300BFA6
:108C300042F8043F0139936113639364F8D1002132
:108C4000C0E96411C0F8981148B27047FF2148B2DA
:108C5000704700002DE9F04F81B02DED088B84B0F6
:108C6000824600284FF0FF0000F048820E4600299F
:108C700000F04482DAF818009AF81C10047940F6E3
:108C800051170029C2F2000700F0D0809AF8D000F6
:108C9000002800F0EA80022800F06481012840F0FA
:108CA0001582002C019673D09FEDACBA9FEDAC8A73
:108CB000A0002A24002740F2AC564FF000084FF0E5
:108CC00000090290DAF818009AED671A0119897AFA
:108CD0000139C9B200EB810090ED020A5FFA89F117
:108CE00020EE010A504680EE0B9AFFF713FD0AEBC7
:108CF00008050AEB070BD5ED3E0ADAED041AB0EED3
:108D000040AA0BF5D270B0EE490AB0EE481AFFF750
:108D10006BF9DAF8180085ED4C0A2044807AD5ED1D
:108D20003E0A0AEB800090ED430ADAED041A05F5DD
:108D300098710BF54370B0EE481A0391FFF754F9A0
:108D400003982AEE000A05F5A47185ED520AFFF793
:108D5000C5FC95ED4C0A95ED521A0AEB060030EE73
:108D6000010A85ED580AFEF7CBF8DAF8180085ED10
:108D70005E0A20440230FEF70DFD029808F1040857
:108D800009F101090A343C37404506F1200699D122
:108D900040F25810C2F200009FEDE98A90ED000AFF
:108DA000DAED041ADAED490A0AF27440B0EE481A14
:108DB000FFF71AF9DAED041ADAED4B0A0AF59660B4
:108DC000B0EE481A8AED640AFFF70EF90AF28C60D9
:108DD0008AED650AFEF794F8DAF818008AED660A5B
:108DE0006830FEF7D7FC019E7078002800F08D8176
:108DF00040F65117C2F200073878002840F0698128
:108E0000B078002800F065819AF81C000221032840
:108E10008AF8D01000F08781022800F089810128AB
:108E200040F050810120AAF8200152E16CB104EB1E
:108E300084004400002500BFDAF8180028442C30D4
:108E4000FEF7A0FC0A35AC42F6D1DAF8180068301B
:108E5000FEF798FC9AED490A40F25810C2F2000061
:108E60008AED680A80ED000A33E10196BCB304EB99
:108E700084009FEDB38A4FEA400800274FF4D2796F
:108E80006FF0030B40F2AC540AEB09063046FFF7D3
:108E9000C1F90AEB0B05D5ED3F0ADAED041A3046AD
:108EA000B0EE480AB0EE481AFFF79EF80AEB04004D
:108EB00085ED4D0A85ED590AFEF722F8DAF818001B
:108EC00085ED5F0A38442C30FEF764FC0A3709F15F
:108ED0003C090BF1040BB84504F12004D4D140F255
:108EE0005810C2F200009FED968A90ED000ADAED6C
:108EF000041ADAED490A0AF27440B0EE481AFFF794
:108F000073F8DAED041ADAED4B0A0AF59660B0EE62
:108F1000481A8AED640AFFF767F80AF28C608AED56
:108F2000650AFDF7EDFFDAF818008AED660A683089
:108F3000FEF730FC019E40F651177078C2F2000730
:108F4000002800F0C6805046FFF7FAFD5046FFF7B4
:108F500043FE5046FFF764FE0120B8E000C0DA454A
:108F600000000000504631460196FFF711FC002C2E
:108F700070D09FED72BA9FED728AA0002A244FF044
:108F8000000840F2AC59002700260290DAF81800D9
:108F90009AED671A0119897A0139C9B200EB81008B
:108FA00090ED020AF1B220EE010A504680EE0B9AD3
:108FB000FFF7B0FB0AEB07050AEB080BD5ED3E0AFD
:108FC000DAED041AB0EE40AA0BF5D270B0EE490A01
:108FD000B0EE481AFFF708F8DAF8180085ED4C0AE9
:108FE0002044807AD5ED3E0A0AEB800090ED430ADA
:108FF000DAED041A05F598710BF54370B0EE481AD6
:109000000391FEF7F1FF03982AEE000A05F5A4711B
:1090100085ED520AFFF762FB95ED4C0A95ED521A69
:109020000AEB090030EE010A85ED580AFDF768FFEA
:10903000DAF8180085ED5E0A20440230FEF7AAFB3C
:109040000298043701360A3408F13C08B84209F1A5
:1090500020099BD19FED3A8ADAED041ADAED490A2C
:109060009AED680A0AF27440B0EE481AFEF7BCFFA7
:10907000DAED041ADAED4B0A0AF59660B0EE481AFA
:109080008AED640AFEF7B0FF0AF28C608AED650A89
:10909000FDF736FFDAF818008AED660A6830FEF749
:1090A00079FB019E40F65117B078C2F2000780B9F3
:1090B00001208AF8D000DAF8240140F25811C2F2F7
:1090C000000108600020AAF8200102E000208AF8D0
:1090D000D000DAF818002C30FEF728FADAF8180079
:1090E0004168052902D35430FEF720FADAF8180057
:1090F0006830FEF71BFAB0783870002040B204B038
:10910000BDEC088B01B0BDE8F08F5046FFF718FDAD
:109110005046FFF785FD002040F651178AF8D00031
:10912000C2F20007D5E741F60A20AAF82001D0E7ED
:10913000DAF81800C069AAF82001CAE700C0DA45C9
:109140000000000000280EBFFF200177002040B281
:1091500070470000002800F0EB802DE9F0472DED6E
:10916000068B8246806990F80480B8F1000F57D0D2
:109170009FED718A4FEA88093427002540F2EC46BA
:109180002424B7EE009ABFEE00AA2EE00AEB0400FA
:1091900090ED000A0AEB0600FDF7B2FE80EE081A19
:1091A0000AEB050080ED380A043520361034B4EEA1
:1091B000491AF1EE10FAC8BFB0EE491ADAF81810E1
:1091C000B4EE4A1AF1EE10FAB8BFB0EE4A1AC95D11
:1091D00080ED3E1A0AEB810090ED430A0A3730EE2B
:1091E000010AA94580ED430A1AD0DAF8180038447C
:1091F0000838FEF71FFBDAF8180038440838FEF785
:1092000033FA0028C2D000F12C0C0AEB85019CE84F
:109210000C10806B01F1200E8EE80C10C862B5E7CF
:109220009AED450A01EE108AB8EEC11A80EE010AE5
:10923000DAF81800B6EE001A683020EE010A8AED5E
:10924000450AFEF7F7FADAF818006830FEF70CFA6C
:1092500001460AF180005022F7F799F9DAF8180070
:109260009AED321A90ED040A20EE010AB5EE400A9A
:10927000F1EE10FA8AED490A0BDA9FED301A00BFC1
:1092800030EE010AB5EE400AF1EE10FAF8DB8AED95
:10929000490A9AED490A9FED291AB4EE410AF1EE06
:1092A00010FA0ADB9FED262A30EE020AB4EE410ADC
:1092B000F1EE10FAF8DA8AED490A9AF8A8000028C7
:1092C0001CBF31EE400A8AED490A9AED230A0AF2E0
:1092D0006C60FDF715FE9AED231A9FED1A2AB7EE82
:1092E000003A81EE021A8AED4A0A9AED090A9AEDCD
:1092F0000D2A0AF2AC6030EE420AB4EE431AF1EEE7
:1093000010FAC8BFB0EE431ABFEE003AB4EE431AEB
:10931000F1EE10FAB8BFB0EE431A8AED4B1A80EDA9
:10932000000A0020BDEC068BBDE8F04740B2704754
:10933000FF2040B2704700BF00C0DA45DB0FC940D4
:10934000DB0FC9C00080BB4580B501F0B5FC01F062
:1093500011FD80BDB0B501380024B4EB106F1CBF07
:109360000120B0BD4EF21005CEF2000568604FF04E
:10937000FF300F2100F0F4FF0720AC60286020468A
:10938000B0BD000080B5FBF785FF03F03BFD012871
:1093900018BF02F00DFF80BD70B592B006AC20463C
:1093A0003021F7F72EF9002543F640000595CDE969
:1093B0000355CDE901550095C4F20200016802266B
:1093C00041F080510160006800F0805000900098EA
:1093D00047F200000095C4F20000016841F48041AA
:1093E0000160006800F48040009000980120069021
:1093F0004FF4803007904FF480000D9006200E90BF
:10940000A820CDE90F060420119020460C96FCF709
:10941000E1F888B90F20CDE901064FF4A05004907F
:109420004FF48050059001A805210395FBF7C4FF78
:10943000002804BF12B070BDFAF7D2F94EF688507A
:10944000CEF20000016841F4700101607047000035
:1094500080B54CF68C50C2F20100FDF713F880BDC8
:10946000B0B540F6FF3E0568C4F2000E40F2004C75
:109470007045C4F2010C0FDCB0F1804F19D040F2FE
:109480000043C4F20003984213D040F60003C4F234
:10949000000398420DD011E040F60043C4F20003EF
:1094A000984206D0604504D00023C4F201039842DC
:1094B00004D14B6825F0700243EA020541F6FF73C0
:1094C000C4F2000398420DDC70451FDCB0F1804F00
:1094D00041D040F20043C4F2000398423BD040F632
:1094E000000321E043F6FF73C4F20103984220DC3D
:1094F00042F20003C4F2000398422CD00023C4F2CD
:109500000103984227D0604525D029E040F600436A
:10951000C4F2000398421ED041F60003C4F20003D7
:10952000984218D041F60043C4F20003984212D08A
:1095300016E044F20003C4F2010398420BD044F653
:109540000003C4F20103984205D044F20043C4F280
:109550000103984204D1CB6825F4407243EA020526
:109560000A688C684B69C46240F480648262644516
:1095700004BF09690163026825F0800142F004021A
:1095800019430260012242610160B0BD80B501F063
:109590001F014FF0010CD0F820E00CFA01F32EEA85
:1095A00003030362036A02FA01F11943016280BDF9
:1095B000B0B5026A036A40F2004523F0010303627A
:1095C000D0F804E0D0F818C08C6822F0020240F411
:1095D0008063C4F20105AB4242EA040205D1CC68C3
:1095E00022F00C0224F0040422430C68AB4207D1A1
:1095F000D1E905532EF4407E45EA0E0545EA030EF7
:109600002CF073032343C0F804E08361496841638D
:109610000262B0BD70B5026A036A40F2004423F0F2
:1096200010030362D0F804E0D0F818C08D6822F06F
:10963000200240F48063C4F20104A34242EA05120E
:1096400007D1CD686FF0400622F0C00206EA05158A
:109650002A430D68A34207D1D1E905642EF4406383
:1096600043EA860343EA840E2CF4E64343EA0523E7
:10967000C0F804E0836149688163026270BD000044
:1096800070B5026A036A40F2004423F480730362F7
:10969000D0F804E0D0F81CC08D6822F4007240F4C9
:1096A0008063C4F20104A34242EA052207D1CD68D7
:1096B00040F2FF462D0222F44062B5432A430D6872
:1096C000A34207D1D1E905642EF4405343EA0613BF
:1096D00043EA041E2CF073032B43C0F804E0C3617B
:1096E0004968C163026270BD70B5D0F820C0026ADB
:1096F00040F2004622F4805202624268C3690C685C
:10970000D1F808E040F48065C4F20106B54204D106
:109710004D6922F4804242EA851223F4E64343EA8B
:1097200004234260C3612CF40056496846EA0E32B5
:109730000164026270BD000001F032F805F0E1F84A
:109740009FED1B0B53EC102B04F018FF05F0ACF849
:109750000446002000F0DCFF01F018F80546FEF793
:1097600099FD40F20C364DF638272544C2F200062A
:10977000C2F2010710E000BF3046F9F7C7FEF86DEE
:1097800001F054F9F86D31460022002301F006F98A
:10979000284600F0CDFF2544FEF7A8FD1420FEF773
:1097A000B5FD0028E8D03046F9F766FEE7E700BFD0
:1097B0000000000000407F4010B501F009F849F6B4
:1097C00009104FF2A422C0F60000C0F600020021EA
:1097D00001F076FA4DF63824C2F20104206049F611
:1097E00091404FF25832C0F60000C0F6000200214E
:1097F00001F066FA606049F6C1204FF2EC22C0F633
:109800000000C0F60002002101F05AFAA06049F6FB
:1098100049504FF2A032C0F60000C0F6000200210D
:1098200001F04EFAE06049F649104FF2C822C0F646
:109830000000C0F60002002101F042FA206149F662
:1098400029404FF23432C0F60000C0F60002002179
:1098500001F036FA606149F641304FF21032C0F63D
:109860000000C0F60002002101F02AFAA06149F6CA
:10987000E9504FF2C432C0F60000C0F600020021E9
:1098800001F01EFAE06149F239704FF28022C0F611
:109890000000C0F60002002101F012FA206202204E
:1098A0000A21002201F02AF86062022034210022FD
:1098B00001F024F8206302201421002201F01EF898
:1098C000606302202021002201F018F820640220A9
:1098D0004FF4C461002201F011F8E0630220582126
:1098E000002201F00BF8A06502204D21002201F0BA
:1098F00005F8E06500F09CFF01F0DEF901F03AFAAE
:1099000010BD00000000000000F04AFF04F0F9FF65
:109910009FED0B0B53EC102B04F030FE04F0C4FF52
:109920000446002000F0F4FE00F030FF051900BFEF
:10993000284600F0FDFE2544FAE700BF00BF00BF47
:109940000000000000407F4084B000F029FF04F0D8
:10995000D8FF9FED570B53EC102B04F00FFE04F0D3
:10996000A3FF0546002000F0D3FE00F00FFF40F2F9
:10997000F01AC2F2000A40F204010446C2F20001E9
:109980005046F7F7EDFC5046F7F7C4FC4CF6E030D4
:109990004CF66C61C2F20100C2F20101F6F782FFDF
:1099A0005046F7F7B7FCB7EE001A81EE000A40F612
:1099B00014104FF2CC42C2F20000C0F600020021A7
:1099C000FEF7CAFB0020F8F713FB0AF1100040F283
:1099D0005C389FED398A9FED399A40F2846904EB37
:1099E000050B02900AF11C00C2F20008C2F2000945
:1099F00003950190F7F702FEF7F778FCF7F782FC82
:109A0000F7F798FCF7F7A4FC00F0E2FE5046F7F7F2
:109A100049FD5046F7F790FD4CF6E034C2F20104E0
:109A2000DDE901214CF66C632046C2F20103F7F731
:109A300001F840462146F6F7C7FE00F0F9FEDAEDE0
:109A40000A0A40F61410C2F20000B0EE480AB0EE66
:109A5000491AF0EE491AFEF7C7FA0020F8F79AFA09
:109A60000AF1100C9CE8181098E80700DAF8246056
:109A7000C9E90A344DF63824C2F20104DAE907755F
:109A8000C9E90260206BC9E90075C9E90412C9F887
:109A900030C000F0CBFF206B49460022002300F0CD
:109AA0007DFF584600F044FE03988344A2E700BFC0
:109AB0000000000000407F40000020420000000045
:109AC00088B000F06DFE04F01CFF9FED190B53EC05
:109AD000102B04F053FD04F0E7FE0446002000279D
:109AE00000F016FE00F052FE0646F9F709FC4CF2B3
:109AF0000855C2F201059FED100A00F530712846A5
:109B000000F058FC2644E84628464146CDE9067751
:109B1000CDE90477CDE90277CDE90077F8F74EFF7C
:109B20002846F9F775F8304600F002FE2644EBE7C8
:109B30000000000000407F400000FA4300000000E9
:109B400082B000F02DFE04F0DCFE9FED350B53ECEF
:109B5000102B04F013FD04F0A7FE0446002000F0D3
:109B6000D7FD00F013FE0646F9F7CAFB40F2442980
:109B7000C2F2000900F564714846F8F7CFFD019480
:109B800026444DF638254CF6783440F208384CF629
:109B90007C3AC2F2010509F1880BC2F2010409F115
:109BA000AC07C2F2000809F1C109C2F2010A00BF04
:109BB000E86D4CF62831C2F201010022002300F0CA
:109BC00059FE40F24420C2F20000F8F77DFE686BB7
:109BD000C4F800B0C8F80070CAF8009000F026FF82
:109BE000686BD8F800100022002300F0D7FEA86AA6
:109BF00000F01CFFA86ADAF800100022002300F031
:109C0000CDFE286C00F012FF286C21680022002392
:109C100000F0C4FE304600F08BFD01980644C7E713
:109C20000000000000407F4000F0BAFD04F069FE33
:109C30009FED150B53EC102B04F0A0FC04F034FE48
:109C40000446002000F064FD00F0A0FD4CF68835CD
:109C5000C2F2010506462846F9F7DEFB4DF6382725
:109C60002644C2F2010700BFB86D00F0DFFEB86DF8
:109C700029460022002300F091FE304600F058FDF6
:109C80002644F1E700BF00BF0000000000407F4015
:109C900000F086FD04F035FE9FED270B53EC102BF2
:109CA00004F06CFC04F000FE8146002000F030FD62
:109CB00000F06CFD0646F9F723FB40F27835C2F25E
:109CC00000059FED1F0A01462846F9F7DBFF4DF618
:109CD00038244CF6F43840F270674E44C2F2010466
:109CE000C2F20108C2F200074FF0010A16E000BFFD
:109CF000606B39460022002300F0BCFD2846FAF7CD
:109D000039F92846394687F800A0F9F76DFD28464D
:109D1000FAF760F8304600F00BFD4E44206B4146E8
:109D20000022002300F0A6FD0028E1D1284641468C
:109D3000FAF7ACF9DCE700BF0000000000407F400C
:109D40000000FA430000000000F02AFD04F0D9FDF5
:109D50009FED210B53EC102B04F010FC04F0A4FD3C
:109D60000446002000F0D4FC00F010FD0646F9F790
:109D7000C7FA4DF28835C2F201059FED190A00F5C8
:109D8000C0712846FEF7A0FD28460221FFF7DAF948
:109D90004DF6382940F6C01840F6BC172644C2F2EA
:109DA0000109C2F20008C2F2000700BFD9F828007A
:109DB00041460022002300F05DFD2846FFF7CAF966
:109DC00028463946FEF74AFD304600F0B1FC2644ED
:109DD000ECE700BF00BF00BF0000000000407F4074
:109DE0000000FA430000000000F0DAFC04F089FDF6
:109DF0009FED0B0B53EC102B04F0C0FB04F054FD53
:109E00000446002000F084FC00F0C0FC051900BFEF
:109E1000284600F08DFC2544FAE700BF00BF00BFD4
:109E20000000000000407F4080B5806B0021C185AC
:109E3000FCF708FD80BD000010B5846B2068406908
:109E400094F84110212907D110F0800004D000209F
:109E5000E084204600F09CF82068406994F84210A5
:109E6000222907D110F0400004D00020E0852046D0
:109E700000F05AF8606C40F0100060642046FCF777
:109E8000E1FC10BD80B50168806B0968C9052FD45D
:109E90000021C185016851E8031F026821F4807127
:109EA00042E80313002BF5D1016851E8051F026851
:109EB00021F0010142E80513002BF5D1016851E8BA
:109EC000051F026821F0400142E80513002BF5D17F
:109ED000202180F84210016B012909D1016851E865
:109EE000031F026821F0100142E80313002BF5D193
:109EF00000214163016B012903D1818DFCF7A0FC96
:109F000080BDFCF78BFF80BD80B5806B0121416374
:109F1000016B012904D1818D4908FCF791FC80BDBA
:109F2000FCF790FF80BD0000016851E8031F026844
:109F300021F4907142E80313002BF5D1016851E838
:109F4000051F026821F0010142E80513002BF5D13D
:109F5000016B01290AD100BF016851E8031F0268A3
:109F600021F0100142E80313002BF5D1202180F8E5
:109F7000421000210163704780B50168CA6822F071
:109F80004002CA60202180F84110FCF76FFF80BDBD
:109F9000016851E8031F026821F0C00142E8031381
:109FA000002BF5D1202180F841107047006840F661
:109FB000FF71C4F20101884210DC44F20041C4F296
:109FC0000001884204BF0120704744F60001C4F23A
:109FD0000001884204BF022070470FE041F20001F7
:109FE000C4F20101884204BF0020704741F20041E1
:109FF000C4F20101884204BF032070470520704766
:10A0000080B582B090F8421022291ED18268B2F544
:10A01000805F02D1016900294AD0816AB2F5805F70
:10A0200007D00AB9026922B10268526802F07F02C1
:10A0300001E0026852680A700121826A114481625B
:10A04000C18D01390A04C18501D002B080BD01680B
:10A05000CA6822F02002CA60CA6822F48072CA600C
:10A060004A6922F001024A61202180F84210002151
:10A070004163026B012A23D1016300BF016851E8EB
:10A08000031F026821F0100142E80313002BF5D1F1
:10A0900001680A68D20606D5002201920A68019278
:10A0A000496801910199818DFCF7CAFB02B080BD1E
:10A0B0000168826A49686FF35F2111800221BCE761
:10A0C000FCF7ACFE02B080BD10B504460068D4E9D0
:10A0D00002C22369016921F440511143016162699F
:10A0E00043EA0C01E3691143C268194349F20C6366
:10A0F0009A431143C1604169A26921F4407141F260
:10A100000043114340F48062C4F201039A4241616A
:10A1100002D1FBF719FA01E0FBF704FAE169636881
:10A120001922B1F5004FA0FB02011CD15A00DB0F30
:10A13000F6F7ECF848F21F51C5F2EB11A0FB012332
:10A140005A096FF0630302FB0300322303EBC000E4
:10A15000A0FB01014FF4F87000EA111000EB0210AF
:10A16000C1F342111AE09A009B0FF6F7CFF848F2BC
:10A170001F51C5F2EB11A0FB01235A096FF06303D5
:10A1800002FB0300322303EB0010A0FB0101F020CF
:10A1900000EA511000EB0210C1F34311226808439A
:10A1A000906010BDF0B581B013460027044681626F
:10A1B00083854764222084F84200E06B49F6856578
:10A1C00049F609760A462168C0F60005C0F6000681
:10A1D000C0E90F5649F63966C0F600060431C0E9F9
:10A1E0001367FAF7D5FD38B110206064202084F899
:10A1F0004200012001B0F0BD009720680168009185
:10A20000406800900098206950B100BF206850E875
:10A21000030F216840F4807041E80302002AF5D161
:10A22000206850E8050F216840F0010041E8050270
:10A23000002AF5D1206850E8050F216840F0400061
:10A2400041E80502002AF5D1002001B0F0BD000070
:10A2500090F84110212923D18168B1F5805F01D1A7
:10A26000016931B1016A02684B1C036209785160CF
:10A2700007E0016A036831F8022B6FF35F225A602E
:10A280000162C18C01390A04C18418BF704700689B
:10A29000C16821F08001C160C16841F04001C16026
:10A2A0007047000010B54CF61C64C2F20104204651
:10A2B000FCF7DCFA2046F7F75DFF10BD10B540F65D
:10A2C000CC04C2F200042046FCF7D0FA2046F7F78F
:10A2D00051FF10BDFEE7000000F0FF40B0F1FF406D
:10A2E00018BF01207047000000F0FF40B0F1FF40B0
:10A2F00018BF01207047000020F00040A0F1FF408F
:10A30000B0FA80F040097047002848BF704700F05D
:10A310001F01012202FA01F14EF280124009CEF231
:10A32000000242F82010BFF34F8FBFF36F8F7047CA
:10A33000002848BF704700F01F01012202FA01F116
:10A340004EF200124009CEF2000242F8201070478F
:10A350004EF60C50CEF200000068C0F302207047A9
:10A360004EF6145300F00F02CEF2000309011A4416
:10A3700000F16043B0F1FF3FC8BF03F564421170C4
:10A38000704700004EF61F50CEF200000021017011
:10A39000704700004EF60C51CEF200010A684FF6ED
:10A3A000FF031A4060F30A2242F0806040F0FD7023
:10A3B0000860704770B52DED048B044600284FF0FF
:10A3C000FF0018BF002900F0C680B5EE400AB0EECD
:10A3D000408AF1EE10FA40F3BE800320C4F8601406
:10A3E0002072D1F8C80004F5C3621060D1F8CC0027
:10A3F0005060F7F753FA8025D4F860042844FDF73D
:10A400006DF90835A02DF7D1A02500BFD4F8600460
:10A410002844FDF763F90835C02DF7D14FF2E83035
:10A42000C0F6000090E80E00C06804F58A6C04F5E0
:10A43000387500268CE80E00C4F85C04D4F860146B
:10A44000A81901F140020021B0EE480AFDF784FE90
:10A450003C36F02EF2D16FF0EF0500BF6619D4F84C
:10A46000602406F538700121B0EE480AFDF774FE4D
:10A47000D4F8601406F5F87001F120020121B0EE65
:10A48000480AFDF769FE3C35E8D1D4F8601404F5BC
:10A49000747001F160020121B0EE480AFDF75CFE24
:10A4A000B3EE049A04F28440B0EE480AF0EE490A92
:10A4B000FCF764FD04F2A440B0EE480AF0EE490A4D
:10A4C000FCF75CFD04F2C440B0EE480AF0EE490A25
:10A4D000FCF754FD04F2E440B0EE480AF0EE490AFD
:10A4E000FCF74CFD04F20450B0EE480AF0EE490AC5
:10A4F000FCF744FD04F22450B0EE480AF0EE490A9D
:10A50000FCF73CFD04F24450B0EE480AF0EE490A74
:10A51000FCF734FD04F26450B0EE480AF0EE490A4C
:10A52000FCF72CFD04F28450B0EE480AF0EE490A24
:10A53000FCF724FD04F2A450B0EE480AF0EE490AFC
:10A54000FCF71CFD04F2C450B0EE480AF0EE490AD4
:10A55000FCF714FD002040B2BDEC048B70BD000080
:10A560007047000040F6DB7110EE100AC3F6C971A7
:10A5700061F31E0000EE100A70470000F0B581B0D4
:10A58000F0B1044640F6A810C2F200000068A042F4
:10A590001FD001F02FFA4CF61870C2F20100656965
:10A5A000076840F6B410C2F20000066801F046FAEF
:10A5B000BD424FF0020018BFB5420DD101B0F0BD51
:10A5C0004FF0500080F31188BFF36F8FBFF34F8FB0
:10A5D000FEE7002001B0F0BD4EF22460C2F201009F
:10A5E00085420CD04EF238610120C2F20101002DEB
:10A5F00008BF04208D4208BF042001B0F0BDA06A4E
:10A6000010B1022001B0F0BD94F85C1003200129C4
:10A6100008BF022001B0F0BD4FF0FF3101FA00F099
:10A62000C04302EE100A30EE600AB8EEC22A31EEE4
:10A63000601A20EE020A80EE010ABDEEC00A10EE9A
:10A64000100A704700207047FAF732FEFEF7A4FEAA
:10A65000FDF7F8F9FDF792F9FDF750F9FDF76EF9FE
:10A66000FDF7D8FAFDF7F6FAFDF714FBFDF77EFBD0
:10A67000FDF798FBFDF7B2FBFDF734FBFDF7D0FBD0
:10A6800000F092F8FDF7C0F900F0B8F8FEE700001E
:10A690000146C068B6EE002A90ED4C1A90ED4B0AC8
:10A6A00021EE021A30EE010A002081ED130A7047F4
:10A6B00030EE600A32EE612A20EE020A31EE601AB4
:10A6C00080EE010A30EE210A70470000401A811026
:10A6D00000EE101A9FED0B1AB8EEC00A30EE011A08
:10A6E0009FED0A2A0C28C8BFB0EE410A9FED061A5A
:10A6F000B4EE420A30EE011AF1EE10FAB8BFB0EE35
:10A70000410A7047DB0FC9C0DB0FC940DB0F49C0EE
:10A71000EFF3058100291CBF6FF00500704700288A
:10A7200004BF0020704780B501F068FA002080BDAA
:10A7300010B582B0EFF3058119B16FF0050002B0DA
:10A7400010BD044602F072FB211A0129019005DBBD
:10A7500001A801F07DFA002002B010BD6FF00300E7
:10A7600002B010BD80B502F04DFB022808BF80BDCD
:10A7700008B9032080BD4CF2C040C2F2010000685D
:10A780000138B0FA80F0400980BD000080B5EFF3D9
:10A79000058010B102F050FB80BD02F047FB80BD88
:10A7A0004FF47A7070470000EFF3058000281CBF5B
:10A7B0006FF0050070474CF2C040C2F20100016822
:10A7C000002911BF4FF0FF300121016000207047C8
:10A7D00080B5EFF3058000281CBF6FF0050080BD39
:10A7E00002F010FB28B1022805D101F0DDFB0020AA
:10A7F00080BD012080BD4FF0FF3080BD10B5EFF36C
:10A80000058000281CBF6FF0050010BD4CF2C0444D
:10A81000C2F20104206801281CBF4FF0FF3010BDB8
:10A82000FDF758FF0220206001F06AFB002010BDF8
:10A8300010B5EFF3058018B16FF00504204610BD88
:10A8400002F0E0FA02280ED080B902F0CDFC012817
:10A850004FF001040CD002F0D5FA002808BF4FF0E9
:10A86000FF34204610BD0024204610BD4FF0FF34B9
:10A87000204610BD10B582B01C46B0FA80F3B1FA84
:10A8800081F25B095209EFF3058CBCF1000F42EA3B
:10A89000030219D0002C18BF0124224315D1002235
:10A8A000019201AA01F088FF01281AD10198A8B1EC
:10A8B0004EF60450CEF200004FF080510160BFF31D
:10A8C0004F8FBFF36F8F09E01AB16FF0030002B032
:10A8D00010BD224601F0AEFE012806D1002002B0D4
:10A8E00010BD6FF0020002B010BD6FF00100002C2F
:10A8F00008BF6FF0020002B010BD0000B0B582B01A
:10A90000144600294FF00005EFF3058218BF002818
:10A9100002D1284602B0B0BD002AFAD19CB1A56888
:10A92000D5B1E268502A16D32269A2B1D4F814C076
:10A9300001FB00F2002394454FF0000228BF0122E2
:10A9400010D24DB10EE0012300226AB9E3B100221A
:10A9500001F064FC0EE01DB9E2680AB92269C2B1D7
:10A9600000220023002AF1D0A36822690025009567
:10A9700001F078FC054655B1002C14BF2168002178
:10A98000284601F005F9C4E70025002DF4D1002583
:10A99000BFE76269B2FA82F25309D5E7B0B582B077
:10A9A0001C46B0FA80F3B1FA81F5EFF305825B093A
:10A9B0006D09002A43EA050207D0002C18BF0124C4
:10A9C000224306D06FF003052CE0CAB16FF00305F7
:10A9D00028E00022019201AA002301F0A1FD012834
:10A9E0001CD10198E8B14EF60450CEF200004FF0B1
:10A9F00080510160BFF34F8FBFF36F8F002511E0CF
:10AA000022460023002501F0B9FC01280AD06FF08E
:10AA10000105002C08BF6FF0020503E06FF002058E
:10AA200000E00025284602B0B0BD000010B5EFF3ED
:10AA3000058119B16FF00504204610BD00280FBF35
:10AA40006FF003040021002401F058FC204610BDE3
:10AA500010B50C46EFF3058100291CBF6FF005000F
:10AA600010BD014620F0010050B111F001010AD1E2
:10AA7000214601F0F7FE012804BF002010BD09E0C7
:10AA80006FF0030010BD214601F0D0FF012804BF84
:10AA9000002010BD6FF00100002C08BF6FF0020015
:10AAA00010BD000070B5EFF30581B9B90028044668
:10AAB00014BF60680020010710D494B1A36843B1AB
:10AAC000E26800214F2A4FF0000288BF01220AD815
:10AAD0004BB9E168B1FA81F1490903E00025284644
:10AAE00070BD0121002200F001063AB1A168002EDC
:10AAF0000CBF0120042001F07FFB06E0C9B1002E4D
:10AB00000CBF0120042001F06BFB054635B1002C81
:10AB100014BF21680021284601F03AF8B5FA85F003
:10AB2000400986F00101084308BF45F001052846A9
:10AB300070BD0025002DEAD1F0E7000080B5EFF3ED
:10AB4000058100291CBF6FF0050080BD014620F083
:10AB5000010040B111F0010108D1002100220023C1
:10AB600001F00CFC04E06FF0030080BD01F040FD3B
:10AB7000013818BF6FF0020080BD0000B0B584B08E
:10AB800048B3B1F1FF3F26DD04464FF0FF3003909C
:10AB9000EFF3058018B300250DF1080C20460122C3
:10ABA00000230295CDF800C002F090F803AB2046D8
:10ABB00000210022009502F089F80298D0B14EF6EB
:10ABC0000450CEF200004FF080510160BFF34F8F70
:10ABD000BFF36F8F0EE06FF0030003900AE0204692
:10ABE0000122002301F0F4FF03AB204600210022E4
:10ABF00001F0EEFF039804B0B0BD00002DE9F04F66
:10AC000083B00C46EFF3058129B16FF00507384694
:10AC100003B0BDE8F08F0546002849D44FF0000B83
:10AC20009246A00758BFAB4602F000F900906FF0C3
:10AC3000010804F0010054460027BAF1000F08BFD4
:10AC40006FF00208019002E04746002EDFD000209E
:10AC5000594602AA234602F0A3F906460128F3D179
:10AC6000029807EA050140EA01090198002809EA6B
:10AC7000050007D100286FF0020718BF4F4607D024
:10AC8000C5E700BFA8426FF0020708BF4F46BED01D
:10AC9000BAF1000FBBD002F0C9F800994F46401A34
:10ACA000241A4FF0000038BF0446002ECFD1AEE783
:10ACB0006FF00307ABE7000080B502F09DF880BDA0
:10ACC00070B584B08E46002100280391EFF3058112
:10ACD00046D0002944D1FAB19369002B08BF18234C
:10ACE000382B16D81179C90713D1556994681168A2
:10ACF0004FEA950C002D08BF4FF0800CFCB1D668D0
:10AD0000602E1BD3D5B11569C5B10024012555B9F5
:10AD10001BE0002004B070BD0124002118234FF077
:10AD2000800C00258DB1946812690294CDE900323F
:10AD30006246734601F010FF039011E00CB9D4682D
:10AD40009CB100250024002DEDD14CB103AC009343
:10AD50001FFA8CF27346019401F0CAFE012802D159
:10AD6000039804B070BD0020E6E71469B4FA84F4D7
:10AD70006409D6E710B5EFF3058100291CBF6FF019
:10AD8000050010BD044660B12046FFF7F7FB04281C
:10AD900004BF6FF0020010BD204600F0ADFF0020A0
:10ADA00010BD6FF0030010BDF0B581B00D464AF63E
:10ADB000400140F6A816C2F20101C2F200060F6877
:10ADC00031680446081D00F09FFD601C0AD14DB19A
:10ADD0003068011D4EF22460C2F2010000F0F2FD65
:10ADE00001B0F0BD3068E41944600AD340F6B410F5
:10ADF000C2F2000000683168043100F0C5FD01B006
:10AE0000F0BD4CF61870C2F20100006831680431E0
:10AE100000F0BAFD4EF2D050C2F2010001688C423F
:10AE200038BF046001B0F0BD70B5044600F0E2FD2B
:10AE30004EF23030C2F20100016840F6A81501312F
:10AE40000160C2F2000529684AF63C06C2F201061A
:10AE500041B1306860B92868E16AC06A884298BF29
:10AE60002C6005E02C600068012801D100F0E0F9B9
:10AE70004EF23830C2F201000168013101606164B4
:10AE80004EF23C31C2F20101E06A0A68904288BF8A
:10AE900008604CF6207100EB8000C2F2010101EB6A
:10AEA0008000211D00F08EFD00F0C8FD306880B1EB
:10AEB0002868E16AC06A884228BF70BD4EF6045017
:10AEC000CEF200004FF080510160BFF34F8FBFF30F
:10AED0006F8F70BD70B582B000F08CFD4AF64406ED
:10AEE000C2F20106306850BB4EF2A054C2F2010417
:10AEF000204600F039FD4AF2F075C2F201052846FD
:10AF000000F032FD40F6AC10C2F2000004604CF6D6
:10AF10001C70C2F201004CF6786240F654130560D2
:10AF20000025C2F20102C2F200030A20102100959E
:10AF300001F098F9306010B103A100F029FE00F093
:10AF40007DFD02B070BD00BF546D72510000000065
:10AF5000F0B581B04AF28C35C2F201052868E0B143
:10AF60004EF238664EF23037C2F20106C2F20107E5
:10AF700000F040FDF068C468201D00F0C5FC386892
:10AF80000138386028680138286000F057FD2046F5
:10AF900000F058F828680028EAD101B0F0BD0000A0
:10AFA00080B5026C002A08BF80BDD0E902C31344FB
:10AFB000C360634524BF0368C360C368084619467D
:10AFC000F5F7A0FA80BD000070B5866B036C0446EF
:10AFD000E3B115461AB3E0681A46F5F793FAE1684B
:10AFE000206C2268091A9142E16003D2A1684042B4
:10AFF0000844E060A81EB0FA80F040093146002EF7
:10B0000018BF01210840361A002516E020680025E7
:10B0100098B9A06802F00CF8A56005460DE06068DC
:10B020001A46F5F76FFA216CD4E9010200250844AD
:10B030006060904224BF20686060711C2846A16354
:10B0400070BD000010B5044690F85D00022808BFEE
:10B0500010BD012803D030B9206B00F007FD204659
:10B0600000F004FD10BD4FF0500080F31188BFF3D5
:10B070006F8FBFF34F8F00BFFEE70000416A0029CA
:10B080000FBF0020006B0068C0F13800704700005F
:10B0900040F6AC11C2F2000109680A68B2FA82F304
:10B0A0005B090360002A0EBF0020C8680068704773
:10B0B00040F6EC10C2F20000C21D22F0070210F0B0
:10B0C000070CA0EB020318BF10464EF21C62C2F23E
:10B0D00001020021C2E9000149F69912C0F2010201
:10B0E000BCF1000F18BF1A440244083A40F6B013EE
:10B0F00022F00702C2F200031A60C2E90011111A1D
:10B100001A68C0E900214AF61C00C2F20100016081
:10B110004EF2CC50C2F2010001604EF2B450C2F2C5
:10B1200001000121017070474CF620744EF6045561
:10B13000C2F20104CEF200054FF08056FFF708FF7F
:10B1400020680228FAD32E60BFF34F8FBFF36F8FB2
:10B15000F4E70000002808BF704780B500210160B7
:10B16000C0E9021100210022002301F007F9BDE827
:10B1700080407047B0B5049D002914BF2A602D603F
:10B18000C5E90F01284601211C4601F0B7F885F8F2
:10B190004C40B0BD2DE9F0470A9C8246206B164614
:10B1A0000F46DDE908599100A5229846F5F721FAE6
:10B1B000206B00EB8600A0F1040020F007067FB1B1
:10B1C00004F13400002100BF7A5C42547A5C1AB169
:10B1D0000F2901F10101F7D3002084F8430002E0B8
:10B1E000002084F834000027201D372D28BF372584
:10B1F000E562C4E9135700F0C3FB04F1180000F046
:10B20000BFFBC5F13800A06130465146424624617B
:10B2100064626765A76584F85C7000F04BFBB9F168
:10B22000000F206018BFC9F80040BDE8F08700009B
:10B23000B0B54CF620750024C2F20105281900F0C3
:10B2400093FB1434B4F58C6FF8D14EF2B854C2F2BB
:10B250000104204600F088FB4AF60405C2F201050D
:10B26000284600F081FB4AF62800C2F2010000F0F7
:10B270007BFB4EF23860C2F2010000F075FB4EF22B
:10B280002460C2F2010000F06FFB4CF61870C2F2AD
:10B290000100046040F6B410C2F200000560B0BDC9
:10B2A00080B54EF21C62C2F2010200BF1146126864
:10B2B0008242FBD3D1F804C001EB0C03834203D1DB
:10B2C0004068604448600846D0F804C000EB0C03B6
:10B2D000934201D013460BE040F6B013C2F20003D4
:10B2E0001B689A4204D0D2E9003E0EEB0C02426089
:10B2F0008142036018BF086080BD000080B58C46A5
:10B30000014641F804CF9445006108D99A4201D220
:10B310009C4511D240F6AC10C2F2000007E08069F3
:10B32000D21A824208D24CF61C70C2F201000068A8
:10B3300000F02AFB002080BD012080BD10B504462E
:10B3400000F058FBA06BB0FA80F0440900F076FBE7
:10B35000204610BD10B5044600F04CFBA06BE16B1D
:10B36000401AB0FA80F0440900F068FB204610BD96
:10B3700008480068006880F308884FF0000080F3F8
:10B38000148862B661B6BFF34F8FBFF36F8F00DFD3
:10B3900000BF00BF08ED00E070B582B040F6AC120F
:10B3A000C2F2000212680546D2680E46D468201D1B
:10B3B00000F0AAFA94F82800410704D400F0FE0037
:10B3C00084F8280010E0A0693246411920462B4637
:10B3D000FFF794FF40B10026204600212A460023B3
:10B3E000009601F0C5FF20B1216A2046884702B0CF
:10B3F00070BD4FF0500080F31188BFF36F8FBFF323
:10B400004F8F00BFFEE700002DE9F04186B04AF6FD
:10B410004407C2F20107386802A900224FF0000871
:10B4200001F008F900286AD001AC02AD0BE000F091
:10B43000FE0086F8280000BF38682946002201F087
:10B44000F9F800285BD00298B0F1FF3F03DCDDE99A
:10B4500003200599904702980028EDD4049E706956
:10B4600010B1301D00F050FA204600F0B3F80299F8
:10B470000929E1D80246DFE801F0080808052A3961
:10B480000808052A96F82800D1E796F82800039BBB
:10B49000B16940F0010086F8280019443046FFF7F2
:10B4A0002DFF0028C8D0316A3046884796F828001A
:10B4B0004007C1D50398B16900230A18304600211E
:10B4C000CDF8008001F054FF0028B5D123E096F8B4
:10B4D000280040F00101039886F82810B06188B177
:10B4E000811830461346FFF709FFA5E796F82800B4
:10B4F00081073FF59CAF304600F0B8FA9CE706B0F4
:10B50000BDE8F0814FF0500080F31188BFF36F8FDA
:10B51000BFF34F8FFEE74FF0500080F31188BFF369
:10B520006F8FBFF34F8F00BFFEE7000070B582B092
:10B530000E46044600F038FD01A800F04BF80199D2
:10B5400019B101F051FE02B070BD05464EB9A542D9
:10B5500007D301F049FE20462946FFF71DFF02B040
:10B5600070BD4EB14CF61C70C2F20100006800685C
:10B57000B0FA80F0420900E000224AF64400C2F22C
:10B5800001000068611B00F017FB01F02DFE002890
:10B59000D9D14EF60450CEF200004FF08051016038
:10B5A000BFF34F8FBFF36F8F02B070BD4CF61870B2
:10B5B000C2F201000168096821B10068C068C06872
:10B5C000406801E04FF0FF304EF2D051C2F201016D
:10B5D0000860704770B5044601F028FC40F6A416D8
:10B5E000C2F2000631680546884203D200F008F82E
:10B5F000012000E0002020602846356070BD00007A
:10B600002DE9F04182B040F6AC17C2F2000738686D
:10B61000016891B34FF0000809E000BF606038682E
:10B620002946246100F0B0F93868016829B3C06880
:10B63000C4680668251D284600F066F9216A204680
:10B64000884794F828004007EED5A0693044B042FE
:10B65000E4D82046002132460023CDF8008001F0D6
:10B6600087FE0028E0D14FF0500080F31188BFF32F
:10B670006F8FBFF34F8F00BFFEE74CF61C71C2F215
:10B6800001010A6808603A6002B0BDE8F08100007C
:10B6900081B00020009040F22C00C2F2000000684F
:10B6A0004FF0500181F31188BFF36F8FBFF34F8FBD
:10B6B000013001D0FEE700BF00980028FCD001B0A7
:10B6C0007047000082B001AC2046FFF7E1FC019911
:10B6D000FFF72CFFFFF798FEF6E70000F0B581B00A
:10B6E000044600F087F994F94560012E0FDB04F160
:10B6F000240500BF286850B1284601F02DFD002820
:10B7000018BF00F069FB70B2013E0128F2DCFF2691
:10B7100084F8456000F092F900F06CF994F94470F7
:10B72000012F0EDB04F11005286850B1284601F006
:10B7300013FD002818BF00F04FFB78B2013F01282D
:10B74000F2DC84F8446000F079F901B0F0BD00004B
:10B750002DE9F04381B0044600F026FC40F6B01617
:10B76000C2F200063068002808BFFFF7A1FC4EF2C5
:10B77000B458C2F2010898F80000002818BF4FF032
:10B78000004020420DD0002401F02EFD60071ED0A5
:10B790004FF0500080F31188BFF36F8FBFF34F8FCE
:10B7A000FEE7C4B114F0070004F108011EBF081A37
:10B7B00000F108015FEA41700ED04FF0500080F3B5
:10B7C0001188BFF36F8FBFF34F8F00BFFEE7204696
:10B7D00001B0BDE8F08300214EF2CC59C2F201095C
:10B7E000D9F800004A1E8242CDD24EF21C60C2F24D
:10B7F000010005682F4657F8042F8A4211D22B68A2
:10B800005BB100BF1F4657F8042F28461D468A42E9
:10B8100007D22B68002BF5D103E04EF21C60C2F278
:10B82000010033689D42AED004682B68521A112A79
:10B83000036010D36818430709D04FF0500080F31D
:10B840001188BFF36F8FBFF34F8F00BFFEE74260D9
:10B850003960FFF725FD4AF61C003968D9F8002049
:10B86000C2F201000368511A9942C9F8001038BFAA
:10B87000016098F80000396800284FF0000018BFF8
:10B8800041F0004128604EF2D450C2F2010002683B
:10B8900008343960511C016076E7000040F6A810BA
:10B8A000C2F20000016819B101680A6D01320A652F
:10B8B0000068704703464BF29160C0F600004FF0FD
:10B8C000807C21F0010103E903106FF0020043F8CE
:10B8D000240CA3F1440043F8202C704702EE100A18
:10B8E0004FF0FF30884030EEC01AB8EEC22AC04395
:10B8F00021EE021A02EE100AB8EEC22A81EE021AF6
:10B9000031EE000A70470000D0E9013201699A6007
:10B91000D1F804C082688445536008BF4A600022A1
:10B920000261086801380860086870474EF24053A9
:10B93000C2F2010303604EF24030C2F2010008601F
:10B9400080201060704700004AF29073C2F2010339
:10B9500003604AF29030C2F2010008604FF4807038
:10B9600010607047704700004FF0FF31024642F808
:10B97000081F00214260C0E90322016070470000F7
:10B98000002101617047000080B5D1F800C01CF1B2
:10B99000010207D000F108039E465B681A68624501
:10B9A000FAD901E0D0F810E0DEF8042008614A601E
:10B9B0009160C1F808E0CEF804100168013101601F
:10B9C00080BD0000D0F800C0436808619A684B60F1
:10B9D0008A609A68996051600CF1010101607047BA
:10B9E000DFF80C00016841F470010160704700BF8E
:10B9F00088ED00E04FF0500080F31188BFF36F8FA7
:10BA0000BFF34F8F40F22C00C2F2000001684A1CC5
:10BA1000026001B170474EF60450CEF2000000689B
:10BA2000000608BF70474FF0500080F31188BFF345
:10BA30006F8FBFF34F8F00BFFEE7000040F22C0076
:10BA4000C2F20000016839B10139016018BF7047C6
:10BA5000002080F3118870474FF0500080F3118868
:10BA6000BFF36F8FBFF34F8FFEE70000B0B5002824
:10BA700008BFB0BD04464EF2B450C2F201000078D7
:10BA800054F8041C002818BF4FF0004008420CD0A6
:10BA9000A4F108052A6892B14FF0500080F3118894
:10BAA000BFF36F8FBFF34F8FFEE74FF0500080F36F
:10BAB0001188BFF36F8FBFF34F8F00BFFEE721EAFE
:10BAC000000044F8040C00F06FFA4EF2CC51C2F2C0
:10BAD000010154F8040C0A68104408602846FFF776
:10BAE000DFFB4AF62400C2F2010001680131016067
:10BAF00001F07AFBB0BD00004EF21000CEF2000063
:10BB00000021016081604CF20001C2F2010109686C
:10BB100044F6D352C1F26202A1FB02124FF0FF3190
:10BB200001EB92114160072101607047EFF305803E
:10BB3000102814D34EF2F031CEF20001405C4AF2EC
:10BB40008531C2F201010978884208D24FF05000D5
:10BB500080F31188BFF36F8FBFF34F8FFEE74EF670
:10BB60000C50CEF200004EF228310068C2F2010102
:10BB7000096800F4E060884298BF70474FF05000B9
:10BB800080F31188BFF36F8FBFF34F8FFEE7000084
:10BB90004EF2DC5C0022C2F2010C00BF5CF83230D5
:10BBA00023B10132082A08BF7047F7E70CEBC20344
:10BBB0004CF832105860704770B515460E46044672
:10BBC000FFF718FF94F84400FF2804BF002084F812
:10BBD000440094F84500FF2804BF002084F8450085
:10BBE000FFF72CFFA06B28B904F1240031462A4648
:10BBF00000F014F92046FFF771FD70BD10B5D8B103
:10BC000004464EF23430C2F20100006848B14FF0F1
:10BC1000500080F31188BFF36F8FBFF34F8F00BFC9
:10BC2000FEE700F0C1F920460021FFF7BDF801F062
:10BC3000DBFA002818BF10BD4EF60450CEF200000B
:10BC40004FF080510160BFF34F8FBFF36F8F10BD76
:10BC5000B0B590B10D46D1B104464EF23430C2F2C7
:10BC600001000068E8B14FF0500080F31188BFF385
:10BC70006F8FBFF34F8F00BFFEE74FF0500080F390
:10BC80001188BFF36F8FBFF34F8F00BFFEE74FF0F8
:10BC9000500080F31188BFF36F8FBFF34F8F00BF49
:10BCA000FEE700F081F94AF64000C2F201000068A8
:10BCB0002268904202EB050102D2914202D309E0D0
:10BCC000914201D3814205D92160081A0021FFF772
:10BCD0006BF800E0216001F087FA002818BFB0BDC2
:10BCE0004EF60450CEF200004FF080510160BFF3D9
:10BCF0004F8FBFF36F8FB0BD70B50446FFF77AFE6C
:10BD000040F6A816002CC2F2000608BF3468251DB4
:10BD10002846FFF7F9FDA06A18B104F11800FFF7F3
:10BD2000F3FD4EF23830C2F20100016801310160CA
:10BD3000306884420CD04EF23030C2F2010001680B
:10BD4000013901602046FFF77DF9FFF72FFC0DE078
:10BD50004EF23860C2F201002946FFF733FE4AF284
:10BD60008C30C2F20100016801310160FFF766FE0C
:10BD70004AF63C00C2F201000068E8B13068844233
:10BD800018BF70BD4EF23430C2F20100006840B1FD
:10BD90004FF0500080F31188BFF36F8FBFF34F8FC8
:10BDA000FEE74EF60450CEF200004FF080510160E5
:10BDB000BFF34F8FBFF36F8F70BD00004AF62001B5
:10BDC000C2F20101096801604AF64001C2F20101B4
:10BDD00009684160704700004AF64800C2F201005D
:10BDE000012101607047000010B568B10C4640F6B3
:10BDF000A811C2F2000109681831FFF7C5FD2046FD
:10BE00000121FEF7D1FF10BD4FF0500080F31188E3
:10BE1000BFF36F8FBFF34F8FFEE70000B0B590B157
:10BE20000D4640F6A811C2F2000109681446183107
:10BE3000FFF7C8FD002C18BF4FF0FF3528462146FC
:10BE4000FEF7B2FFB0BD4FF0500080F31188BFF392
:10BE50006F8FBFF34F8F00BFFEE7000070B528B3B0
:10BE6000026D04461AB3E06C884238BF0846012AC6
:10BE70001CD1E16A814208BF70BD40F6A812C2F22F
:10BE800000021268A2421CD0A269E062002A5CBFD4
:10BE9000C0F13800A0614CF62076606901EB8101A9
:10BEA000C2F2010606EB8101884214D070BD4FF04A
:10BEB000500080F31188BFF36F8FBFF34F8F00BF27
:10BEC000FEE74FF0500080F31188BFF36F8FBFF390
:10BED0004F8F00BFFEE7251D2846FFF715FD4EF2E8
:10BEE0003C31C2F20101E06A0A68904288BF0860F2
:10BEF00000EB800006EB80002946FFF763FD70BD74
:10BF000010B586B0002405A804A903AACDE904440D
:10BF1000FFF70CFDDDE9032005990023CDE90101C0
:10BF20004BF22910C0F600001DA1009400F014FE91
:10BF30004AF61801C2F20101086010B101F0DEF901
:10BF40000446601C22D0012C1ED14FF0500080F31B
:10BF50001188BFF36F8FBFF34F8F4EF2D050C2F2F4
:10BF600001004FF0FF3101604AF63C00C2F20100CF
:10BF7000012101604AF64000C2F201000021016087
:10BF8000FEF7EEFA00F08AF806B010BD4FF0500050
:10BF900080F31188BFF36F8FBFF34F8FFEE700BFB1
:10BFA00049444C45000000004EF23430C2F201001A
:10BFB0000168013101607047B0B54EF23430C2F211
:10BFC0000100006830B14AF64800C2F201000121C8
:10BFD0000160B0BD4AF64800C2F2010000210160D4
:10BFE000FEF730FB4EF22C31C2F201010A6840F636
:10BFF000A8159042C2F2000504D92B68821A5C6D24
:10C0000022445A6508602868006B0168B1F1A53FB9
:10C010000BD14168B1F1A53F07D18168B1F1A53FCE
:10C0200003D1C068B0F1A53F04D028682968343135
:10C03000FFF798FC4EF23C30C2F2010001684CF66A
:10C04000207201EB8103C2F2010252F823404CB985
:10C0500002EB8303143B00BFB1B153F8144901391B
:10C06000002CF9D001EB810302EB830252F8043F6C
:10C070005B68141DA342136001D15B6813601268F2
:10C08000D2682A600160B0BD4FF0500080F3118883
:10C09000BFF36F8FBFF34F8FFEE7000080B582B014
:10C0A0004EF20040CEF200004CF27021C4F20F11AB
:10C0B000D0F800294B1C9A4209D14FF0500080F370
:10C0C0001188BFF36F8FBFF34F8F00BFFEE7D0F82B
:10C0D00000298A4209D14FF0500080F31188BFF344
:10C0E0006F8FBFF34F8F00BFFEE701784AF28532B2
:10C0F0000191FF2101700178C2F201028DF8031055
:10C100009DF8031001F0500111704EF22831C2F277
:10C11000010107220A609DF90320B2F1FF3F0CDC08
:10C120000A6800BF9DF80330013A5B008DF80330C8
:10C130009DF90330002BF5D40A600A68032A2DD13B
:10C140004FF4E06303EA02220A6001990170D0F81B
:10C15000201941F47001C0F82019D0F8201941F0DD
:10C160007041C0F82019FFF7C7FC40F22C00C2F262
:10C17000000000210160FFF733FC4EF63470CEF270
:10C180000000016841F040410160FFF7F1F8FFF75E
:10C1900013FFFFF77DFA002002B080BD4FF0500082
:10C1A00080F31188BFF36F8FBFF34F8FFEE700005E
:10C1B00080B54FF0500080F31188BFF36F8FBFF34D
:10C1C0004F8F00F043FE30B14EF60450CEF2000027
:10C1D0004FF080510160002080F3118880BD000085
:10C1E00010B502460120002100F018F80446FEF7C1
:10C1F000B1FF204610BD000010B582B00B4684464A
:10C20000012000210022CDF800C000F02BF80446E8
:10C21000FEF7A0FF204602B010BD0000F0B581B0CF
:10C22000B0B105464843503014460E46FFF790FA29
:10C23000074650B1002007F1500287F84600284613
:10C24000314623460097FEF795FF384601B0F0BD12
:10C250004FF0500080F31188BFF36F8FBFF34F8F03
:10C26000FEE70000B0B582B068B11D46ABB1F1B9D0
:10C27000EAB14FF0500080F31188BFF36F8FBFF326
:10C280004F8F00BFFEE74FF0500080F31188BFF3DF
:10C290006F8FBFF34F8F00BFFEE74FF0500080F36A
:10C2A0001188BFF36F8FBFF34F8F00BFFEE751B10F
:10C2B0004AB94FF0500080F31188BFF36F8FBFF37E
:10C2C0004F8F00BFFEE750230193019B502B0AD1F3
:10C2D000069B019C012485F846400095FEF74AFF25
:10C2E000284602B0B0BD4FF0500080F31188BFF374
:10C2F0006F8FBFF34F8F00BFFEE7000070B5F8B13E
:10C3000004460E46FFF776FB2068D4E90F1200259D
:10C3100002FB0103013901FB0201A563C4E901032A
:10C32000FF20E16084F8440084F8450004F1100027
:10C330007EB1FFF719FB04F12400FFF715FB18E0AD
:10C340004FF0500080F31188BFF36F8FBFF34F8F12
:10C35000FEE7016869B100F0FFFE50B14EF60450EF
:10C36000CEF200004FF080510160BFF34F8FBFF35A
:10C370006F8FFFF763FB012070BD00002DE9F04FC8
:10C3800083B00292B8B11D460E460446E9B1022DB3
:10C3900003D1E06B012840F09A8000F033FD00BB30
:10C3A0000298F0B14FF0500080F31188BFF36F8F07
:10C3B000BFF34F8FFEE74FF0500080F31188BFF3BB
:10C3C0006F8FBFF34F8F00BFFEE7206C0028DED0D9
:10C3D0004FF0500080F31188BFF36F8FBFF34F8F82
:10C3E000FEE7FFF707FBA06B022D58D0E16B8842F8
:10C3F00055D304F1100801206F464FF0000B0DF1EA
:10C4000008094FF0805A00BF0299002900F07B8094
:10C41000C00702D03846FFF7D1FCFFF70FFBFFF74C
:10C42000C3FDFFF7E7FA94F84400FF2808BF84F83B
:10C4300044B094F84500FF2808BF84F845B0FFF7E2
:10C44000FDFA3846494600F00FFB00285ED1204631
:10C45000FEF780FFA0B102994046FFF7C5FC2046D9
:10C46000FFF73CF900F0C0FE78B94EF60450CEF26A
:10C470000000C0F800A0BFF34F8FBFF36F8F04E040
:10C480002046FFF72BF900F0AFFEFFF7B3FAA06BE1
:10C49000022D04D0E16B88424FF00000B4D2204658
:10C4A00031462A46FEF790FD54F8241FC9B12046B4
:10C4B00000F052FE08B34EF60450CEF200004FF0EA
:10C4C00080510160BFF34F8FBFF36F8F15E04FF0C6
:10C4D000500080F31188BFF36F8FBFF34F8F00BF01
:10C4E000FEE750B14EF60450CEF200004FF08051FE
:10C4F0000160BFF34F8FBFF36F8FFFF79FFA0120EB
:10C5000003B0BDE8F08FFFF799FA04E02046FFF78B
:10C51000E5F800F069FE002003B0BDE8F08F0000F0
:10C520002DE9F04381B0E8B11E46914605460F461D
:10C5300009B3022E02D1E86B012837D1FFF7F6FAD2
:10C54000EFF311884FF0500080F31188BFF36F8F25
:10C55000BFF34F8FA86B022E19D0E96B884216D318
:10C5600000203FE04FF0500080F31188BFF36F8F41
:10C57000BFF34F8FFEE7286C0028DAD04FF0500051
:10C5800080F31188BFF36F8FBFF34F8FFEE795F8ED
:10C590004540A86B284639463246FEF715FDFF2C6C
:10C5A0000DD0601C85F8450001201BE04FF05000C5
:10C5B00080F31188BFF36F8FBFF34F8FFEE755F8FD
:10C5C000240F70B1284600F0C7FD0146B9F1000FF5
:10C5D0004FF0010006D000291CBF0120C9F800005F
:10C5E00000E0012088F3118801B0BDE8F08300006D
:10C5F000B0B5A8B18568044600F0FEFB85421CBFBB
:10C600000020B0BDE0680138E0601CBF0120B0BD73
:10C610002046002100220023FFF7B0FE0120B0BD1C
:10C620004FF0500080F31188BFF36F8FBFF34F8F2F
:10C63000FEE700002DE9F04F85B0049298B10C465A
:10C640000546002900F0A58000F0DCFBA8B904989D
:10C6500098B14FF0500080F31188BFF36F8FBFF394
:10C660004F8F00BFFEE74FF0500080F31188BFF3FB
:10C670006F8FBFF34F8F00BFFEE705F1240005F178
:10C680001009019002AF0DF1100A4FF000080AE006
:10C690002846FFF723F800F0A7FD2846FEF74EFED8
:10C6A000002840F08480FFF7A5F9D5F838B0BBF139
:10C6B000000F1DD028462146FEF772FCABF10100A9
:10C6C000A863286970B1484600F046FD50B14EF6A7
:10C6D0000450CEF200004FF080510160BFF34F8F45
:10C6E000BFF36F8FFFF7AAF900200126A0B95FE022
:10C6F000049850B1B8F1000F02D13846FFF75EFB45
:10C700004FF00108012038B952E0FFF797F90026F1
:10C71000002000284CD000BFFFF790F9FFF744FC41
:10C72000FFF768F995F84400FF2804BF002085F85A
:10C73000440095F84500FF2804BF002085F8450017
:10C74000FFF77CF93846514600F08EF900289FD15A
:10C750002846FEF7F3FDB0B104990198FFF744FBBA
:10C760002846FEF7BBFF00F03FFD00289BD14EF6A8
:10C770000450CEF200004FF080510160BFF34F8FA4
:10C78000BFF36F8F8FE72846FEF7A8FF00F02CFD60
:10C7900089E7286C00283FF457AF4FF0500080F332
:10C7A0001188BFF36F8FBFF34F8F00BFFEE70026E6
:10C7B000304605B0BDE8F08F2DE9F04381B000B3FD
:10C7C000914605460E4631B3FFF7B0F9EFF31188F5
:10C7D0004FF0500080F31188BFF36F8FBFF34F8F7E
:10C7E000AC6B24B395F8447028463146FEF7D8FB6D
:10C7F000601EFF2FA8631CD0781C85F84400012020
:10C800002AE04FF0500080F31188BFF36F8FBFF321
:10C810004F8F00BFFEE7286C0028D5D04FF05000A6
:10C8200080F31188BFF36F8FBFF34F8FFEE70020B7
:10C8300012E055F8100F70B1284600F08DFC01464B
:10C84000B9F1000F4FF0010006D000291CBF0120F4
:10C85000C9F8000000E0012088F3118801B0BDE8AC
:10C86000F08300002DE9F04F85B0049158B10446E3
:10C87000006C90B14FF0500080F31188BFF36F8FC0
:10C88000BFF34F8FFEE74FF0500080F31188BFF3E6
:10C890006F8FBFF34F8F00BFFEE700F0B3FA50B9C0
:10C8A000049840B14FF0500080F31188BFF36F8FB0
:10C8B000BFF34F8FFEE704F1240004F1100501904F
:10C8C0004FF0000802AF0DF1100A4FF000094FF0D1
:10C8D000000B0AE02046FEF701FF00F085FC204631
:10C8E000FEF72CFD002840F07F80FFF783F8A06B57
:10C8F000F0B10138A063206810B9FEF7CFFFA06047
:10C90000286870B1284600F027FC50B14EF604505C
:10C91000CEF200004FF080510160BFF34F8FBFF3A4
:10C920006F8FFFF78BF801260020B8B96FE000BFCA
:10C93000049850B1BBF1000F02D13846FFF73EFA20
:10C940004FF0010B012048B961E0B9F1000F62D14D
:10C95000FFF774F800200026002858D0FFF76EF883
:10C96000FFF722FBFFF746F894F84400FF2808BFC2
:10C9700084F8448094F84500FF2808BF84F8458077
:10C98000FFF75CF83846514600F06EF80028A1D158
:10C990002046FEF7D3FC28B92046FEF79FFE00F0A4
:10C9A00023FCA2E7206838B9FFF724F8A06800F05C
:10C9B00089FB8146FFF742F804990198FFF714FAC2
:10C9C0002046FEF78BFE00F00FFC00287FF48DAFB1
:10C9D0004EF60450CEF200004FF080510160BFF3DC
:10C9E0004F8FBFF36F8F80E7B9F1000F0ED0FFF7C5
:10C9F00001F82046FEF742FBA168024608461146B0
:10CA0000FFF72CFAFFF71AF8002600E00026304660
:10CA100005B0BDE8F08F4FF0500080F31188BFF3F0
:10CA20006F8FBFF34F8F00BFFEE7000070B568B196
:10CA3000866804460D4600F0DFF986420FD0204696
:10CA40002946FFF70FFF58B9002070BD4FF0500086
:10CA500080F31188BFF36F8FBFF34F8FFEE7012084
:10CA6000E1680131E16070BDB0B5D0B10D4611B3E0
:10CA70000446FEF7BFFF4AF64000C2F2010001681B
:10CA80002868421C21D04AF620036268C2F20103E2
:10CA9000D3F800C091421AD323689C4517D00124D3
:10CAA00022E04FF0500080F31188BFF36F8FBFF387
:10CAB0004F8F00BFFEE74FF0500080F31188BFF3A7
:10CAC0006F8FBFF34F8F00BFFEE700240CE0891A81
:10CAD000884206D9401A28602046FFF76FF90024E3
:10CAE00002E0002001242860FEF7A8FF2046B0BD28
:10CAF0002DE9F04383B007469000984615468946D5
:10CB0000FEF726FE78B106466020FEF721FE38B11A
:10CB10000446066354B94FF0FF3003B0BDE8F0831C
:10CB20003046FEF7A3FF0024002CF4D0DDE90A1004
:10CB3000002284F85D20CDE90010384649462A4697
:10CB400043460294FEF726FB2046FEF76DF90120CE
:10CB500003B0BDE8F083000070B586B00B9CCCB18B
:10CB60000C9E06B360250495049D602D25D1049D7F
:10CB7000DDF828C0022586F85D5005AD3463CDE9A7
:10CB800000C50296FEF706FB3046FEF74DF9059804
:10CB900006B070BD4FF0500080F31188BFF36F8F67
:10CBA000BFF34F8FFEE74FF0500080F31188BFF3C3
:10CBB0006F8FBFF34F8F00BFFEE74FF0500080F341
:10CBC0001188BFF36F8FBFF34F8F00BFFEE70000E8
:10CBD000F0B581B0D0B11D46174604460E46FEF7AB
:10CBE00009FF002D1CBFA06D286094F85C00022195
:10CBF000042F84F85C1012D80125DFE807F0230326
:10CC00001C262000A16D3143A1651FE04FF05000AC
:10CC100080F31188BFF36F8FBFF34F8FFEE7A16DD5
:10CC2000013113D04FF0500080F31188BFF36F8FA4
:10CC3000BFF34F8FFEE7A16D0131A16506E0022829
:10CC400003D1002501283CD103E0A6650125012878
:10CC500037D1261D3046FEF757FE4EF23C31C2F268
:10CC60000101E06A0A68904288BF08604CF62071B2
:10CC700000EB8000C2F2010101EB80003146FEF7BB
:10CC8000A1FEA06A48B14FF0500080F31188BFF3B5
:10CC90006F8FBFF34F8F00BFFEE740F6A811C2F2BF
:10CCA0000001E06A0968C96A88420AD94EF6045050
:10CCB000CEF200004FF080510160BFF34F8FBFF301
:10CCC0006F8FFEF7BBFE284601B0F0BD2DE9F041A5
:10CCD00020B31D46174604460E46FEF727FFEFF326
:10CCE00011884FF0500080F31188BFF36F8FBFF3AE
:10CCF0004F8F002D1CBFA06D286094F85C000221AE
:10CD0000042F84F85C1012D80125DFE807F0230314
:10CD10001C262000A16D3143A1651FE04FF050009B
:10CD200080F31188BFF36F8FBFF34F8FFEE7A16DC4
:10CD3000013113D04FF0500080F31188BFF36F8F93
:10CD4000BFF34F8FFEE7A16D0131A16506E0022818
:10CD500003D10025012849D103E0A665012501285A
:10CD600044D1A06A48B14FF0500080F31188BFF35E
:10CD70006F8FBFF34F8F00BFFEE74EF23430C2F229
:10CD80000100006830B14AF6280004F11801C2F22F
:10CD9000010015E0261D3046FEF7B6FD4EF23C318F
:10CDA000C2F20101E06A0A68904288BF08604CF64E
:10CDB000207100EB8000C2F2010101EB80003146DE
:10CDC000FEF700FE40F6A811C2F20001E06A096811
:10CDD000C96A88420AD9069800281CBF012101604F
:10CDE0004AF64800C2F201000121016088F311886F
:10CDF0002846BDE8F081000040F6A810C2F200000D
:10CE0000006870474AF63C00C2F201000068002842
:10CE100004BF012070474EF23430C2F201000068B6
:10CE2000B0FA80F040094000704700004AF6400028
:10CE3000C2F201000068704780B5FEF777FE4AF63F
:10CE40004000C2F20100006880BD00002DE9F04FF3
:10CE500081B04EF23430C2F20100006840B14EF2AF
:10CE6000D850C2F20100016800240131016092E053
:10CE70004AF64000C2F2010001684E1C066021D350
:10CE80004CF61870C2F201000168096849B14FF010
:10CE9000500080F31188BFF36F8FBFF34F8F00BF37
:10CEA000FEE740F6B412C2F20002016813680360A4
:10CEB0004AF620001160C2F20100016801310160F0
:10CEC000FEF774FB4EF2D051C2F20101086840F641
:10CED000A81A4CF620788642C2F2000AC2F2010873
:10CEE00001D2002445E04CF61877C2F201073868F9
:10CEF0000024006898B34EF23C3BC2F2010B19E0EB
:10CF0000D9F82C00DBF80010884288BFCBF800006D
:10CF100000EB800008EB80002946FEF753FDD9F8AE
:10CF20002C00DAF80010C96A3A68884228BF012448
:10CF30001068B8B13868C068D0F80C904D4655F804
:10CF4000040F864210D32846FEF7DEFCD9F82800ED
:10CF50000028D5D009F11800FEF7D6FCD0E74FF035
:10CF6000FF3005E04FF0FF304EF2D051C2F2010128
:10CF70000860DAF80000C06A00EB800058F8200072
:10CF800001284AF64800C2F2010088BF0124006867
:10CF9000002818BF0124204601B0BDE8F08F000032
:10CFA0002DE9F0411E46154688460746FEF722FD4C
:10CFB00040F6A814C2F20004206890F85C00022831
:10CFC00019D02068816D21EA0701816520684FF042
:10CFD000010180F85C1076B130460121FDF7E4FED6
:10CFE0004EF60450CEF200004FF080510160BFF3C6
:10CFF0004F8FBFF36F8FFEF721FDFEF7FBFC15B1DE
:10D000002068806D28602068002590F85C10002062
:10D01000022905D1216801258A6D22EA08028A6564
:10D02000216881F85C00FEF709FD2846BDE8F08123
:10D03000B0B580B1044640F6A810C2F20000006806
:10D04000A0420AD04FF0500080F31188BFF36F8FD9
:10D05000BFF34F8FFEE70020B0BD206D38B301381D
:10D0600020654FF0000018BFB0BDE16AE26C91424C
:10D070001CD0251D2846FEF747FCE06CC0F13801A6
:10D08000A1614EF23C31E062C2F201010A689042B5
:10D0900088BF08604CF6207100EB8000C2F20101ED
:10D0A00001EB80002946FEF78DFC0120B0BD4FF05A
:10D0B000500080F31188BFF36F8FBFF34F8F00BF15
:10D0C000FEE70000F0B581B000B340F6A816C2F24A
:10D0D00000060446C06A3168C96A884219D2A1694B
:10D0E000002904D43168C96AC1F13801A1614CF644
:10D0F0002077616900EB8000C2F2010707EB800036
:10D1000081420FD03068C06AE06221E0002001B0A7
:10D11000F0BDE16C3068C26A0020914238BF012046
:10D1200001B0F0BD251D2846FEF7EEFB30684EF23B
:10D130003C31C06AC2F20101E0620A68904288BFD5
:10D14000086000EB800007EB80002946FEF73AFC00
:10D15000012001B0F0BD0000B0B5C068C5687DB168
:10D1600005F118042046FEF7CFFB4EF23430C2F230
:10D170000100006868B14AF62800C2F201001DE013
:10D180004FF0500080F31188BFF36F8FBFF34F8FC4
:10D19000FEE72C1D2046FEF7B7FB4EF23C31C2F2F3
:10D1A0000101E86A0A68904288BF08604CF6207165
:10D1B00000EB8000C2F2010101EB80002146FEF786
:10D1C00001FC40F6A811C2F20001E86A0968C96AC8
:10D1D000884291BF00204AF64801C2F201010120B5
:10D1E00088BF0860B0BD00002DE9F04F81B04EF25D
:10D1F0003434C2F20104206868B1FEF7FBFB2068FA
:10D2000001382060206880B10024FEF717FC20461A
:10D2100001B0BDE8F08F4FF0500080F31188BFF3EC
:10D220006F8FBFF34F8F00BFFEE74EF23030C2F278
:10D230000100006800285DD04AF62806C2F2010607
:10D2400030684AF64808C2F2010890B34EF23C3703
:10D250004CF6207940F6A81BC2F20107C2F2010980
:10D26000C2F2000B4FF0010AF068C56805F1180022
:10D27000FEF74AFB2C1D2046FEF746FBE86A39689C
:10D28000884288BF386000EB800009EB80002146AF
:10D29000FEF798FBE86ADBF80010C96A884228BFED
:10D2A000C8F800A030680028DED1002D18BFFEF7B6
:10D2B0007DF94EF2D854C2F20104256855B1012619
:10D2C000FFF7C4FD002818BFC8F80060013DF7D182
:10D2D00000202060D8F8000070B14EF60450CEF265
:10D2E00000004FF080510160BFF34F8F0124BFF366
:10D2F0006F8F8AE7002488E7002486E780B586B030
:10D30000FDF7E8FD4AF64400C2F20100006808B3E8
:10D310000020CDE9040005A804A903AAFEF714FB28
:10D32000DDE903200221DDF814C0CDE900104BF245
:10D33000C560C0F600000CA10023CDF808C0FFF7BF
:10D340000BFC4EF24C61C2F20101086010B10120E9
:10D3500006B080BD4FF0500080F31188BFF36F8F8F
:10D36000BFF34F8FFEE700BF546D7220537663000A
:10D3700010B584B0A8B14AF64404C2F20104844650
:10D380002068C0B10529CDE90012CDF808C015DC30
:10D39000FFF738FD01462068022916D1069A694632
:10D3A00015E04FF0500080F31188BFF36F8FBFF38B
:10D3B0004F8F00BFFEE7002004B010BD69461A463B
:10D3C0000023FFF7ADF804B010BD6946002200232A
:10D3D000FEF7D4FF04B010BD03B4019841000098DB
:10D3E00050EAC12018BF04204A0D18BF40F00100C8
:10D3F00040F2FF72B2EB515F08BF40F0020001281B
:10D4000008BF052002B070474100080218BF042081
:10D410000A0E18BF40F001004FF07F4232EA0101CE
:10D4200008BF40F00200012808BF05207047000037
:10D4300010B54FF00E402DED028BB0EE408A18EE85
:10D44000104A00EB4400B0F1506F4AD84FF0FC4056
:10D45000B0EB440F22D2B0EEC80AF7EE000A30EE6D
:10D46000C00AF6EE000A60EE208A18EE900A00F07C
:10D4700073FF01EE100A14F0004F1DBFDFED2D0AFF
:10D480009FED2D0AB1EE411ADFED2C0A08BF9FED8A
:10D490002C0AF8EE001A21EE218A05E0DFED290AB8
:10D4A00068EE088AB0EE600A9FED271ADFED271AB2
:10D4B00030EE080A48EE811A9FED251A08EEA11AEF
:10D4C000DFED241A48EE811A9FED231A08EEA11A07
:10D4D00068EE281ABDEC028B01EE810A30EE200ABC
:10D4E00010BD4FF0E440B0EB440F0CD918EE100A19
:10D4F000FFF78AFF042808BF00F068FEB0EE480A74
:10D50000BDEC028B10BD4FF07F40B0EB440F07D253
:10D51000B0EE480ABDEC028BBDE8104000F048BEFA
:10D520000120F3F79DF8BDEC028BBDE8104000F040
:10D5300045BE00000000C9BF22AAFDB90000C93FD6
:10D5400022AAFD390000000024FE1C3DC78AD83CF9
:10D550001E67383D1B93993DAFAA2A3E000000008C
:10D5600070B59B482DED020B2DED068B079D25F028
:10D570000044A04218DC9748844202DC0AD1069895
:10D5800040B19DED060BBDEC068B02B0BDE87040CE
:10D5900000F0E8BD002DCCBF9FED8F0B9FED900BF1
:10D5A000BDEC068B02B070BD8F48A04215DD8F48E0
:10D5B000A042D8BF4FF0FF3458DD9DED060B51EC73
:10D5C000100BFFF709FF042808BF00F0E1FD9DEDF7
:10D5D000060BBDEC068B02B070BD9DED060B51EC49
:10D5E000100B00F0ADFECDE9060181489FED828B66
:10D5F000A0423CDD8248A0421FDD00249FED82ABAB
:10D600009DED060B53EC1A2B51EC100B00F002FFB2
:10D610009DED060B41EC190B53EC1A2B51EC100B42
:10D6200001F0FAF953EC182B01F0CCFB53EC192B59
:10D6300000F0A4FFCDE9060149E09DED060B0124B1
:10D6400053EC182B51EC100B00F0E4FE9DED060B93
:10D6500041EC190B53EC182B51EC100B01F0B2FB01
:10D6600053EC192B00F08AFFCDE906012FE0684842
:10D67000A0421FDD02249FED689B9DED060B53EC3D
:10D68000192B51EC100B01F0C7F953EC182B00F0DB
:10D69000C1FE9DED060B41EC180B53EC192B51EC20
:10D6A000100B01F08FFB53EC182B00F067FFCDE956
:10D6B00006010CE09DED060B032453EC102B9FEDAF
:10D6C000580B51EC100B00F059FFCDE906019DED10
:10D6D000060B53EC102B51EC100B01F09DF941ECB3
:10D6E000180B53EC182B01F097F941EC190B4E482D
:10D6F0000621B0EE490AF0EE690A784400F0B6FC63
:10D7000053EC182B51EC100B01F086F941EC180B7F
:10D710004648B0EE490AF0EE690A0521784400F067
:10D72000A5FC53EC192B51EC100B01F075F941ECF1
:10D73000100B51EC180B53EC102B002C0EDA00F0F0
:10D7400069FE9DED061B53EC112B01F065F99DED73
:10D75000061B53EC112B01F05DFA35E000F05AFE88
:10D760009DED061B53EC112B01F056F941EC100B0B
:10D770002F48784400EBC40090ED001B51EC100BD7
:10D7800053EC112B01F01EFB9DED061B53EC112BEE
:10D7900001F018FB41EC100B2648784400EBC40064
:10D7A00090ED001B51EC100B53EC112B01F032FAF1
:10D7B00041EC100B002DA2BFBDEC068B02B070BD7A
:10D7C00051EC100B00F0E7FD41EC100B01E70000FD
:10D7D000000010440000F07F182D4454FB21F93F55
:10D7E000182D4454FB21F9BF0000DC3F0000203E0F
:10D7F0000000F33F00000000000000000000F03FC8
:10D800000000E63F000000000000000000000040B3
:10D810000080034000000000000000000000F83F0E
:10D82000000000000000F0BFCA1A0000801A0000CB
:10D830000A1A0000C219000070B56F4E2DED040BDE
:10D840002DED048B82B0DDF824C0DDE907235C42B6
:10D850002CF000411C4341EAD474069D22F00040A4
:10D86000B44205D86C422C4340EAD474B4420BD97C
:10D870009DED081B9DED060B02B0BDEC048B04B0C2
:10D88000BDE8704000F078BCACF14054A4F17F6476
:10D890001C430BD0022404EAAC7444EAD27405435E
:10D8A0009FED578B9FED582B07D015E09DED060B94
:10D8B00051EC100B00F03CFD42E0002C11BF012C9C
:10D8C0009DED060B02B0BDEC048B04BF04B070BD2F
:10D8D000022C38D0032C3BD00B439FED4D1B9FED0A
:10D8E0004E0B0AD0B14218D1B04209D121F080418B
:10D8F00020F08040099107900FE0002A15DA10E02F
:10D90000474B7B44002C08BF93ED000B0DD0012C3E
:10D9100010D0022C17D0032C1AD0B0421DD1002AEF
:10D9200003DAB0EE410AF0EE610A02B0BDEC048BFE
:10D9300004B070BD93ED000B51EC100B00F02BFD0B
:10D9400041EC100BF1E7B0EE480AF0EE680AECE7A4
:10D95000B0EE420AF0EE620AE7E7401A00159FEDCA
:10D96000329B3C28C8BF8DED000B17DCBCF1000FCB
:10D97000BCBF10F13C0F8DED009B0FDB9DED080B44
:10D9800053EC102B9DED060B51EC100B00F0F6FD47
:10D9900000F0D6FC00F0CCFCCDE90001B4B1012CC4
:10D9A00010D0022C9FED220B53EC102B9DED000BA1
:10D9B00051EC100B19D001F005FA53EC182B01F0C3
:10D9C00001FABDE7019880F0004001909DED000B49
:10D9D00053EC192B51EC100B00F02AFF04BF02206E
:10D9E000F2F73EFE9DED000B9FE701F0EBF953ECE3
:10D9F000182B01F00FF9A3E70000F07F00000000F2
:10DA0000182D4454FB210940182D4454FB2109C012
:10DA1000182D4454FB21F9BF182D4454FB21F93F24
:10DA2000F2180000000000000000000000000000EC
:10DA3000075C143326A6A13C70B54FF068422DED6B
:10DA4000048BF0EE408A18EE900AB0EE608A18EE71
:10DA5000101A02EB4003B3F1654F3CBF02EB4102E9
:10DA6000B2F1654F7DD200BFC0F3C753C1F3C752B7
:10DA70009A1A1B2A09DD10F0004F14BF9FED830A8C
:10DA80009FED830ABDEC048B70BD12F11A0F36DADC
:10DA900011F0004F09D010F0004F0CBF9FED7D0A30
:10DAA0009FED7D0ABDEC048B70BD88EE889A19EE5F
:10DAB000100AFFF7A9FC042808BF00F087FB18EE46
:10DAC000900AFFF7A1FC054618EE100AFFF79CFC30
:10DAD000044619EE100AFFF797FC042D18BF052D18
:10DAE00008D1042C18BF052C04D1002804BF022043
:10DAF000F2F7B6FDB0EE490ABDEC048B70BD4200F2
:10DB0000B2EB410F3AD910F0004F19BFDFED630AB5
:10DB10009FED630ADFED630A9FED630AB0EE481ADA
:10DB20000A46B1EE688A80F00041F0EE418A104664
:10DB30000A1A5200B2F1807F34D2484010F0004FF0
:10DB4000DFED5A1A9FED5A2A1DBFBEEE001A70EE85
:10DB5000E10A30EE420AB6EE001A08BF70EEA10AE2
:10DB600000E040E008BF30EE020AB0EE682A01EEA5
:10DB7000482A08EE818AC2EE081A15E011F0004F1B
:10DB800004BF9FED4C0AF0EE400AD1D010F0004FD8
:10DB900019BFDFED490A9FED490ADFED490A9FED04
:10DBA000490AC5E7C8EE881A21EEA11A9FED462A58
:10DBB000DFED462A41EE022A9FED452A01EE222A98
:10DBC000DFED442A41EE022A9FED432ABDEC048B8F
:10DBD00001EE222A21EE811A01EE020A30EE210A1C
:10DBE00030EE200A70BD4FF07F42B2EB400F28BFED
:10DBF000B2EB410F09D2F0EE480AB0EE680ABDEC74
:10DC0000048BBDE8704000F0D6BA40EA01035B0027
:10DC100008BF41F0FF410BD0B2EB400F08BFB2EBA1
:10DC2000410F08D120F0804008EE900A21F0804199
:10DC300008EE101A18E7B2EB400F12BF5FEA41037B
:10DC400040F0FF4001F000413FF40EAFB2EB410F56
:10DC500012BF5FEA400200F0004041F0FF413FF494
:10DC600003AF4A0092EA40033FF5FEAE002AACBF84
:10DC70009FED1A0A9FED1A0A68EE808A28EE008A44
:10DC800018EE900A18EE101AEEE60000DB0FC9BF7E
:10DC9000DB0FC93FDB0F4940DB0F49C00000C9BFA4
:10DCA00022AAFDB90000C93F22AAFD390060ED3E5D
:10DCB000C30ACE3700000000000049C022AA7DBA86
:10DCC0000000494022AA7D3A2DAD65BD8FB8D53DF3
:10DCD0000FB511BE61C84C3EA8AAAABE0000804F75
:10DCE0000000802F00B510EE101A2DED028B81B0D0
:10DCF000524A6846B2EB410F2ED94FF0E640B0EBE6
:10DD0000410F94BF00204FF0FF3000900098B0EE1C
:10DD1000408A00286ADB10F0010F4BD068EE080A39
:10DD20009FED471A9FED470A00EE810A9FED461AC4
:10DD300010F0020F00EE801AB7EE000A00EE810A22
:10DD400002BF01B0BDEC028B00BD00BF01B0B1EE5F
:10DD5000400ABDEC028B00BD3C4B21F000429342D7
:10DD600041D911F0004FDFED3A0A20EE201ADFED25
:10DD7000390A19BF31EE601A71EE200A31EE201A0D
:10DD800071EE600ABDEEE01A11EE100A9FED321A34
:10DD900000F0030000EEC10A9FED301A009000EE83
:10DDA000C10A9FED2F1A00EEC10A9FED2E1A00EE58
:10DDB000C10AABE728EE080A9FED2B1ADFED2B0A0C
:10DDC00010F0020F40EE010A9FED291A00EE201A12
:10DDD00061EE000AB0EE480A08EE200AB6D101B0A2
:10DDE000BDEC028B00BD00F0F9F98FE718EE100AC8
:10DDF0004000B0F17F4F0DD218EE100AFFF704FB80
:10DE0000042808BF00F0E2F9B0EE480A01B0BDEC0A
:10DE1000028B00BD09D10120F2F722FC01B0BDEC5C
:10DE2000028B5DF804EB00F0C9B901B0B0EE480A0E
:10DE3000BDEC028B5DF804EB00F0BAB9B61F927E20
:10DE4000B93AB2BACA9F2A3DDDFFFFBE490E494624
:10DE500083F9223F0000004B0000C93F00A0FD39BC
:10DE60000020A2331A61342C336D4CB9DA82083C9D
:10DE7000A0AA2ABE00B52DED048BB0EE409AF0EEBC
:10DE8000609A83B051EC190B00F0D0FE41EC180BF6
:10DE900018EE100A18EE901A8DED008B002818BFAE
:10DEA0000120084320F00040C0F17F6000F1E04015
:10DEB000C00F14D019EE101A19EE900A8DED009BC8
:10DEC000002918BF0121084320F00040C0F17F6005
:10DED00000F1E040C00F04BF0120F2F7C1FBB0EE3B
:10DEE000480A03B0F0EE680ABDEC048B00BD0000E8
:10DEF00000B510EE101A2DED028B81B04D4A684628
:10DF0000B2EB410F3CD94FF0E640B0EB410F94BF6C
:10DF100000204FF0FF3000900098B0EE408A0028BB
:10DF20005FDB28EE080ADFED440A9FED441A00EE9D
:10DF3000201ADFED430A40EE010A9FED421A00EE7F
:10DF4000201ADFED410A10F0010F40EE010A9FEDAB
:10DF50003F1A00EE201A61EE000AB0EE480A08EE01
:10DF6000200A02BF01B0BDEC028B00BDBFEE001A5B
:10DF700001B0C1EE000ABDEC028BB0EE600A00BD3C
:10DF8000334B21F00042934228D911F0004FDFEDCE
:10DF9000310A20EE201ADFED300A19BF31EE601A87
:10DFA00071EE200A31EE201A71EE600ABDEEE01A21
:10DFB00011EE100A9FED291A00F0030000EEC10ACD
:10DFC0009FED271A009000EEC10A9FED261A00EE81
:10DFD000C10A9FED251A00EEC10A9DE700F0FEF888
:10DFE0009AE718EE100A4000B0F17F4F0DD218EEFC
:10DFF000100AFFF709FA042808BF00F0E7F8B0EEAE
:10E00000480A01B0BDEC028B00BD09D10120F2F736
:10E0100027FB01B0BDEC028B5DF804EB00F0CEB83D
:10E0200001B0B0EE480ABDEC028B5DF804EB00F0E5
:10E03000BFB80000B61F927EBCE9223C0B6D063BC8
:10E040008A76CE3CACB5593D35A1083E29AAAA3EF8
:10E05000490E494683F9223F0000004B0000C93FAA
:10E0600000A0FD390020A2331A61342C70B504469B
:10E070002DED028B4D1E00EBC500B0EE408AF0EE98
:10E08000608A90ED000B35F0060017D053EC182B8A
:10E0900051EC100B00F0C0FC41EC100B6D1E04EBBA
:10E0A000C50090ED001B51EC100B53EC112B00F050
:10E0B000B1F941EC100B35F00600E7D1022D36D056
:10E0C000042D1CD0062D1CBFBDEC028B70BD53EC83
:10E0D000182B51EC100B00F09FFC94ED0A1B53EC35
:10E0E000112B00F097F953EC182B00F095FC94EDF0
:10E0F000081B53EC112B00F08DF941EC100B53EC85
:10E10000182B51EC100B00F087FC94ED061B53EC20
:10E11000112B00F07FF953EC182B00F07DFC94EDEF
:10E12000040B53EC102B00F075F941EC100B53EC81
:10E13000182B51EC100B00F06FFC94ED021B53EC0C
:10E14000112B00F067F953EC182B00F065FC94EDEF
:10E15000001B53EC112B00F05DF9BDEC028B41EC80
:10E16000100B70BD10B553EC102B51EC100B00F0E0
:10E1700051F941EC100B10BD10B553EC112B51ECC3
:10E18000100B00F047F941EC100B10BD000000002F
:10E190009FED050B10B553EC102B51EC100B00F05C
:10E1A0003BFC41EC100B10BD000000000000001013
:10E1B00030EE000A704730EE200A7047DFED020AA9
:10E1C00080EEA00A70470000000000009FED020AE8
:10E1D00020EE000A70470000000000102DE9F00159
:10E1E0004FF07F42B2EB410F9FBF4FF0FF31016014
:10E1F000BDE8F00170474FF0004242EA0123C1F34D
:10E20000C752783A551112F01F0C434CCCF120063E
:10E210007C44C1F3C752A2F178024FEA621204EBC8
:10E22000820254F8254008BFD2E9015612D0556841
:10E2300004FA0CF425FA06F73C43976805FA0CF546
:10E2400027FA06F8D26807FA0CFCF24045EA0805FE
:10E250004CEA0206A4FB034CA5FB0352A6FB036396
:10E260001D449D4234BF012600261319334416B1C4
:10E27000934202D903E0934201D2012200E000223E
:10E28000624402F1200C9206DC0C42EA443200EEB9
:10E29000102A5B03DFED210AF8EEC01A00EE103AF7
:10E2A0004FEA9C1C11F0004FB8EE400AC0F800C0C5
:10E2B00020EE201A00EE105ADFED190AB8EE400ADF
:10E2C00020EE200A71EE810A70EE800A10EE902A8C
:10E2D00002F500626FF30B0200EE902A70EEE11A75
:10E2E00031EEC11ADFED101A30EE411A9FED0D0A22
:10E2F00020EE800A01EE210A9FED0C1A00EE810A41
:10E3000004BFBDE8F0017047CCF180510160BDE869
:10E31000F001B1EE400A7047EC0F0000000000363B
:10E320000000802C22AAFD29DB0FC92F0000C92F75
:10E3300010B541EC100BFFF713F951EC100B10BDA9
:10E3400082B0CDE9000121F0004001909DED000B6D
:10E3500002B051EC100B704710B500EE100A2DED15
:10E36000028BB1EEC08A18EE100A20F00040C0F116
:10E37000FF40C00F0AD010EE100A20F00040C0F19C
:10E38000FF40C00F04BF0120F2F76AF918EE100A2F
:10E39000BDEC028B10BD81F00041704780F0004061
:10E3A000704721F00041704720F0004070470000A6
:10E3B00021F0004201F00043A2F16052B2F5801F4B
:10E3C00028BFD2F17F6C0BD95FEA001C43EAC2027E
:10E3D00042EB507018BF704728BF20F00100704713
:10E3E000B2F5801FBCBF184670474FEA410C1CF5C0
:10E3F000001F02D2084600F0ABBE70B500F0B6FBBD
:10E4000000000089FFF7F6BF4FF00040A0F5800044
:10E410007047000010B591EA030F48BF83F0004336
:10E4200000F1D884841A71EB030C05D2121943EB66
:10E430000C03001B61EB0C014FEA1154A4EB135CBD
:10E44000DFF81CE11EEA430F18BF9EEA445F00F0AC
:10E45000748021EA045123EA0E0343F48013DCF1B3
:10E46000200E32D322FA0CFE10EB0E0023FA0CFE23
:10E4700041EB0E01CCF1200E03FA0EFE10EB0E0064
:10E48000CCF1200E51F10001B1F5801F32D201EB29
:10E49000045112FA0EF2BDE8104058BF7047401CFC
:10E4A00038BF5FEA420218BF7047002814BF20F04F
:10E4B000010041F100014FEA410313F5001F38BF8D
:10E4C0007047A1F1C04100F09FBB012A43EB03025A
:10E4D000ACF1200CDCF11F0E32BF4FF0000E23FA1E
:10E4E0000CF310EB030041EB0451B4EB115FD0D0FF
:10E4F000A1EB045101F58011490801EB04515FEAD9
:10E5000030000ED350F1000038BF12FA0EFE08D1D1
:10E51000BDE81040C9E7401C38BF5FEA4202CAD1DB
:10E52000C3E7BDE810404FEA410313F5001F38BFB1
:10E530007047A1F1C04100F067BB9EEA445F08D07C
:10E5400011EA5E0FBDE8104004BF01F00041002059
:10E550007047BDE8104070B500F008FB64FBBE3E9C
:10E560000000E0FF491058BFC1F140415B1058BFA7
:10E57000C3F140438B42EFF3008070472DE9C04167
:10E5800030B4DFF8A4C23CEA111418BF3CEA1314FB
:10E5900000F0ED801CEA111481EA030544EAD57409
:10E5A00018BF1CEA131500F0C880A4EB050404F1A1
:10E5B0007F7404F500344FF0004545EAC12145EA77
:10E5C000C32341EA505143EA52534FEAC0204FEA75
:10E5D000C222994208BF904200F09D804FEA136525
:10E5E0000FF24416765D4FEA134506FB05F7C7F1B7
:10E5F000807706FB07F74FEAD737A7FB0368764219
:10E60000A7FB06CEC8F5803838BFA8F1010807FB84
:10E6100008E6A6FB028C4FF0000EE6FB03CEDCF111
:10E62000000CCEF1004E38BFAEF1010EA6FB0C5827
:10E630004FF00007E6FB0E87A1FB08C6A0FB07CE44
:10E6400016EB0E064FF0000545F10005E1FB0765EE
:10E6500015F1E04E7EBFA4F580345FEA46066D41B9
:10E6600016F1800745F100054FEA172747EA0567CD
:10E670004FEA15254FEA0666A6F1DE46B6F1805F41
:10E6800020D9384605EBC47124F0010C01EB0C11C4
:10E69000BCF1FE6F02D8F0BCBDE8008124425CBF33
:10E6A00001F5801E9EEAC47F02D4F0BCBDE8008163
:10E6B000244200F13980A1F1C041F0BCBDE8004125
:10E6C00000F0A2BA4FEAD02040EA41504FEAD121EF
:10E6D0004FEAD22242EA43524FEAD323A7FB0286F3
:10E6E00007FB036605FB02661EEA0E0F58BFA6EB8A
:10E6F0000056B6EB00564FEA520E4EEAC37E18EBB8
:10E700000E0E56EB530EBCD518EB02085E417F1C73
:10E7100055F10005B5E74FF480154FF000074FF0B5
:10E7200000064FF00008ACE701F1C04101F00041E4
:10E730004FF00000F0BCBDE800810CEA131511EAAF
:10E740000C1F00D00CE013EA0C1F00F026804FF0E5
:10E75000000081EA030101F00041F0BCBDE8008146
:10E76000F0BCBDE8004181EA030100F04DBAF0BC05
:10E77000BDE8004170B500F0F9F900BF097EFC3E2C
:10E7800000F007B84FF0000081EA030101F00041FA
:10E79000704781EA030100F037BAF0BCBDE80041E0
:10E7A00022494FF000007047FFFDFBF9F7F5F4F246
:10E7B000F0EEEDEBE9E8E6E4E3E1E0DEDDDBDAD81C
:10E7C000D7D5D4D3D1D0CFCDCCCBCAC8C7C6C5C47A
:10E7D000C2C1C0BFBEBDBCBBBAB9B8B7B6B5B4B391
:10E7E000B2B1B0AFAEADACABAAA9A8A8A7A6A5A47C
:10E7F000A3A3A2A1A09F9F9E9D9C9C9B9A99999840
:10E800009797969595949393929191908F8F8E8EE2
:10E810008D8C8C8B8B8A898988888787868585846F
:10E8200084838382828181800000FF070000F87F5B
:10E8300051EA030C17D41CF5801F58BFBCF5801F8C
:10E8400000F10680994218BF704708BF9042704798
:10E8500007D711F5801F58BF13F5801F19D49942AF
:10E860007047894270471CF5801F08D5BCF5801F92
:10E87000F7D58B4218BF704708BF824270474FF4EC
:10E88000001C1CEB410F38BF1CEB430F01D28B4225
:10E89000704770B500F06AF9922449004FF00051BA
:10E8A0004FF08053FFF75EBE4FEA1153A3F580632C
:10E8B000D3F11E03A8BFD3F1200C08DB4FF00042B8
:10E8C00042EAC12252EA505232FA03F0704709423A
:10E8D0000BD4102BC4BF0020704703F5787CBCF12B
:10E8E000FF3F05D04FF0FF3070474FF000007047FA
:10E8F00070B500F03BF900BF4992248000207047BA
:10E90000F0E7B0FA80F310FA03F10AD0C3F11D0367
:10E9100003F580634FEA03524FEA415002EBD121E5
:10E9200070474FF00000704751EA030C17D41CF5F4
:10E93000801F58BFBCF5801F00F10680994218BFA8
:10E94000704708BF9042704707D711F5801F58BF26
:10E9500013F5801F19D499427047894270471CF5FE
:10E96000801F08D5BCF5801FF7D58B4218BF7047B4
:10E9700008BF824270474FF4001C1CEB410F38BFA8
:10E980001CEB430F01D28B42704770B500F0EEF8DC
:10E99000922449004FF080514FF00053FFF7E2BD41
:10E9A00051EA030C17D41CF5801F58BFBCF5801F1B
:10E9B00000F10680994218BF704708BF9042704727
:10E9C00007D711F5801F58BF13F5801F19D499423E
:10E9D0007047894270471CF5801F08D5BCF5801F21
:10E9E000F7D58B4218BF704708BF824270474FF47B
:10E9F000001C1CEB410F38BF1CEB430F01D28B42B4
:10EA0000704770B500F0B2F8922449004FF0005101
:10EA10004FF08053FFF7A6BD70B5DFF848C11CEA80
:10EA2000111E1EBF1CEA13159EEA0C0F95EA0C0F6F
:10EA300000F06F8081EA03044EEAD47EAE4421EAFE
:10EA40004C1123EA4C1341F4801143F48013AEF1CE
:10EA50007F7EA1FB024CA0FB0365361955EB0C052C
:10EA6000A1FB034C4CF10003A0FB021C16EB0C06AF
:10EA7000654153F10003094218BF46F0010613F443
:10EA8000007F0BD14FEA03314FEA053041EA1551BF
:10EA900040EA165034036FF003020AE04FEAC32144
:10EAA0004FEAC52041EA555140EA5650F4026FF052
:10EAB000020202EB2E4201EB025585EACE710AD02A
:10EAC0005FEA440C18BF24F0004450F1000041F10B
:10EAD000000120EAD47040F2FE7C624500D270BD95
:10EAE000A84214BF4FF080444FF04044002E08BFAE
:10EAF0000024BEF1806FA8BFA1F1C041BDE8704005
:10EB000080F2828001F1C04101F000414FF000002D
:10EB100070470CEA13159EEA0C0F18BF95EA0C0F0C
:10EB200006D081EA030E4FF000000EF0004170BDE8
:10EB300000F01CF88900013E00F007B800F009B8A9
:10EB40004FEA430C5FEA5C5C08D081EA030100F005
:10EB50005BB84FEA410C5FEA5C5CF6D102494FF0CA
:10EB6000000070470000FF070000F87F0EF1020E62
:10EB70002EF0030E5EF8046B364205D4012A43EBF7
:10EB8000030515F5001F12D8012841EB010C1CF5F7
:10EB9000001F0CD80ED14FEAD17C0CEB4C0C0CF1C1
:10EBA000020C15F5001F08BF4CEBD37C04E04FF0BE
:10EBB000080C01E04FEAD37C0CEB4C0526FA05F675
:10EBC00006F00706B6F1040C06D20EEB860CBDE883
:10EBD00070404CF0010C6047DFE80CF0090B0202BA
:10EBE0004FF00041A1F500214FF0000070BD194623
:10EBF0001046012851EB010418BFD4F5001484BF5E
:10EC0000002001F0004170BD0808A0F500114FEA96
:10EC10003101704710B591EA030F81F000413FF5D3
:10EC200001AC83F0004300F0D5B800002DE9F041BD
:10EC300001F5801CBCF5001FC0F2A9804FEA115CF1
:10EC400021EA0C5141F480110CF1FD0C5FEA5C0CDF
:10EC50000CF5C07C01D340004941890241EA905142
:10EC600087022EA48E0EA45D0A0C04FB04F602FBA0
:10EC700006F6C6F14046A4FB0662F60D46EA4226B9
:10EC800006FB06F4A4FB01235242C3F1404338BF04
:10EC90005B1EA6FB02420024E6FB0324D20B42EAE1
:10ECA0004446A6FB0623A1FB02E2A3FB07E4E3FB29
:10ECB00061426442C2F1404E38BFAEF1010EA6FB84
:10ECC00004234FF00002E6FB0E32A2FB03463400A1
:10ECD000E2FB6264A1FB06E6A4FB07E8E4FB6168D3
:10ECE0007642C8F1405838BFA8F10108A2FB06E4FB
:10ECF000A3FB08E5E2FB6854A1FB05E6A7FB04E8DB
:10ED0000E1FB648618F1200556F10006A80940EAE7
:10ED10008660B109A8F11B0808F03F08B8F10A0F96
:10ED20001CD901EB0C51BDE8F08100BFFCF5EEE809
:10ED3000E2DDD8D3CFCBC7C3C0BDB9B6B4B1AEAC9A
:10ED4000A9A7A5A3A19F9D9B9A9896959392908F12
:10ED50008D8C8B898887868584838281A0FB00685F
:10ED600000FB01F208EB4208B8EB872807D53418FE
:10ED700058EB0104D5D5401C51F10001D1E7341AFC
:10ED800078EB0104CDD4401E71F10001C9E75FEAC0
:10ED90004C0C5FEA9C5C0DD105D301F000414FF0B3
:10EDA0000000BDE8F081BDE8F04170B5FFF7DEFE80
:10EDB0006DDBFFBEBDE8F04101494FF00000704738
:10EDC0000000F87F10B591EA030F48BF83F00043BD
:10EDD0003FF528AB841A71EB030C07D28CF0004C82
:10EDE000121943EB0C03001B61EB0C014FEA1154A9
:10EDF000A4EB135CDFF8A4E11EEA430F18BF9EEA00
:10EE0000445F00F0B48021EA045123EA6E035242C9
:10EE1000C3EB6E0338BF5B1EDCF1200E25D322FA54
:10EE20000CFE10EB0E0043FA0CFE41EB0E01CCF190
:10EE3000200E03FA0EFE10EB0E00CCF1200E51F165
:10EE4000000129D401EB045112FA0EF2BDE8104082
:10EE500058BF7047401C1CBFB2F1004F70470028DC
:10EE60000CBF491C20F00100704712EB020E43EB6F
:10EE7000030218BF4FF0010E4EEA4202ACF1200C23
:10EE8000DCF11E0E56D943FA0CFE10EB0E00CCF14D
:10EE90001E0E51F1FF31D5D50EF1010E12FA0EFE04
:10EEA000404141EB010101EB445C5FEA5C5C10D93D
:10EEB00001EB045110EBDE7038BFBEF1004FBDE82E
:10EEC000104018BF704700280CBF491C20F00100FB
:10EED000704734D24FEAD42C24F4006411F50011A9
:10EEE0001BD0B1FA81F20B3AA41AA41ED2F120036E
:10EEF000914030FA03F31943904001EBCC7101EBE0
:10EF00000451002CBDE81040A8BF704701F1C0417A
:10EF100001F000414FF000007047B0FA80F310FAA2
:10EF200003F102D1BDE810407047E41A173C4805D0
:10EF3000C90AE2E701EB0451BDE8104070474910EF
:10EF40004FEA300001EB0451BDE8104002E04FF001
:10EF5000000170474A0008BF0042F8D0B2F5001F18
:10EF600028BF704701F000414FF0000070479EEA53
:10EF7000445F07D011EA5E0FBDE8104004BF0021D6
:10EF800000207047BDE8104070B5FFF7EFFD00BFEF
:10EF900040DFF63E104683F0004170470000E0FF7E
:10EFA00043004FEAD30C4FEA3C0C43401FBF4007DD
:10EFB0000CF1605113F0FE4F70471CF0006F03D14D
:10EFC0000CF00041002070470CF0004343EA507001
:10EFD00040EACC0010B500F068F800BF00000092D5
:10EFE0004FEA0001FFF710BE4FF00041A1F50021EC
:10EFF0004FF00000704710B5FFF71AFC0CBF01205E
:10F00000002010BD10B5FFF713FC14BF0120002035
:10F0100010BD10B5FFF788FC8CBF0120002010BD8B
:10F0200010B5FFF781FC2CBF0120002010BD10B5EA
:10F03000FFF7B6FC94BF0120002010BD10B5FFF70C
:10F04000AFFC34BF0120002010BD4FF07E5209E01C
:10F0500011F0004204D54042C1F1000138BF491E01
:10F0600042F07E5202F170620B0012BF20235FEA71
:10F0700000017047B1FA81FC01FA0CF1A3EB0C031B
:10F0800020FA03FC41EA0C0102EBC352C3F1200356
:10F0900010FA03FC5CEA416C42EB112018BF5FF0F0
:10F0A000806C28BF20F0010070470EF1020E2EF098
:10F0B000030E5EF8044B244204D44FEA4102B2F13D
:10F0C0007F4F11D84FEA4003B3F17F4F0CD80ED1D8
:10F0D0004FEAD07C0CEB4C0C0CF1020CB2F17F4FE0
:10F0E00008BF4CEBD17C04E04FF0080C01E04FEA84
:10F0F000D17C0CEB4C0324FA03F404F00704B4F1C4
:10F10000040C06D20EEB840CBDE810404CF0010C50
:10F110006047DFE80CF0070802024FF00040A0F55E
:10F12000800010BD0846420018BFD2F1807288BF2F
:10F1300000F0004010BDF1EE100A4FF6FF71C0F272
:10F14000C03120EA010040F04070E1EE100A704743
:10F15000FF2141EAD050C0057047000000000000C8
:10F160004FBB610567ACDD3F182D4454FB21E93FDF
:10F170009BF681D20B73EF3F182D4454FB21F93FCE
:10F18000E2652F227F2B7A3C075C143326A6813C54
:10F19000BDCBF07A8807703C075C143326A6913CFF
:10F1A000C4EB98999999C9BF711623FEC671BCBF6B
:10F1B0006D9A74AFF2B0B3BF9AFDDE522DDEADBFD3
:10F1C0002F6C6A2C44B4A2BF0D5555555555D53FEB
:10F1D000FF8300922449C23F6E204CC5CD45B73F06
:10F1E000513DD0A0660DB13FEB0D76244B7BA93F7E
:10F1F00011DA22E33AAD903F000000000000000069
:10F20000000000006E83F9A22915444ED15727FC57
:10F21000C0DD34F5999562DB4190433CAB6351FE10
:10F2200000000000000000000102030406070809B6
:10F230000000000001020304010000000000024081
:10F240001000000000000240010000000004024025
:10F25000020000000004024002000000000802401A
:10F2600010000000000802402000000000080240DA
:10F270000800000000180240400000000018024092
:10F280003DF5000800000000000000000000000044
:10F290000000000000040000180000000000000052
:10F2A0000000000001F50008000000000000000060
:10F2B0000000000000000000000400001800000032
:10F2C000000000000000000004F50008000000003D
:10F2D000000000000000000000000000000400002A
:10F2E0001800000000000000000000001AF50008EF
:10F2F000000000000000000000000000000000000E
:10F3000000040000180000000000000000000000E1
:10F31000FDF40008000000000000000000000000F4
:10F3200000000000000400001800000000000000C1
:10F3300000000000F8F400080000000000000000D9
:10F3400000000000000000000004000018000000A1
:10F3500000000000000000000EF5000800000000A2
:10F360000000000000000000000000000004000099
:10F3700018000000000000000000000043F5000835
:10F38000000000000000000000000000000000007D
:10F390000004000030000000000000000000000039
:10F3A00027F5000800000000000000000000000039
:10F3B0000000000000040000180000000000000031
:10F3C0000000000032F5000800000000000000000E
:10F3D0000000000000000000000400001800000011
:10F3E00000000000000000007FDAEF420054E74117
:10F3F0008063504320C19643ECF4000800000000F5
:10F4000000000000000000000000000000020000FA
:10F4100018000000000000000000000000000000D4
:10F4200001000000000200000924000801000000A3
:10F430000200000000020000892300080200000012
:10F440000400000000020000212400080300000066
:10F450000800000000020000392400080400000039
:10F4600010000000000200006123000805000000F9
:10F470002000000000020000C52300080600000074
:10F480000000008000080000E923000807000000D9
:10F490000080000001080000F523000808000000BB
:10F4A0008000000000020000512400080900000054
:10F4B00000010000010C0000852300080A00000084
:10F4C0003040000001010000A12300089A99193E74
:10F4D0000000803F00000000000000000000803FAE
:10F4E0000000803F000000000000000064656661CD
:10F4F000756C745461736B006472313600636D64B3
:10F5000000616900617474695F657374690067699B
:10F510006D62616C5F6374726C00636861737369C0
:10F52000735F6374726C0073686F6F745F6374727F
:10F530006C00737465705F6D6F746F720045543149
:10F540003673005461736B5F496E6974000000008C
:10F5500090F50008000000203000000020020008A4
:10F56000C0F5000800C00120F8030000C401000835
:10F57000C0F500083000002020AA01003C0200086D
:10F5800030F70008F8C30120582600003C020008AC
:10F59000022B073DFEF7BBB8DD098A3BDE7772BC64
:10F5A0003DF50008000000000C030020752600084F
:10F5B000892500087D26000801000000AAAAAAAA41
:10F5C000112324F42A010312012A110991120112B4
:10F5D000123A021CE112011B09021871E59A99996D
:10F5E0003E1B803F044ABF04112240432242658FE4
:10F5F000C2F53D1AE0142FA041DB0FC9403C980929
:10F60000CDCCCC3E0AD7233C3CD9401A2004C14380
:10F6100020416940C980F94022C01A10301B804047
:10F62000681980291C29402B80BF4019DFFA02DFAE
:10F630004948193CC00B7A449A99193E1F856BBE04
:10F640001CAE47A1441AC0040112496401221CCD1A
:10F65000CC4CB4298C69B4214A061869C05B3F05BB
:10F660001C320349A4339B43191C3A01B429041CDE
:10F67000020201070914C201164B05023029641E5B
:10F68000C03F9A99998849902C6666667819F8293E
:10F6900004397C1A40D03920190C29B0290459208A
:10F6A0002B20404429F04D0AD7233D2839B83DBFCF
:10F6B000DB0FC91C9960192869F0A960013CCBF0E7
:10F6C0004104295C29685BCC3DB0296C79702980A4
:10F6D000CD3D0A573E20393819205BB443A0D920CC
:10F6E0000928B01201540102015A02085A03085AAB
:10F6F0000408540502025A06085A07085A0808E97D
:10F70000513302034A40843AC0DC1C030405172924
:10F7100003611305281B0835041A7D042964134569
:10F72000271B0871041AD904E954294DC13210006D
:040000050800018965
:00000001FF
